:020000040800F2
:1000000000000110E91C080891250008016302089E
:10001000891D0808891D0808891D080800000000BE
:100020000000000000000000000000005146000831
:10003000554600080000000059460008FDD700089A
:10004000891D0808891D0808891D0808891D0808D8
:10005000891D0808891D080829A800082DA800087E
:10006000891D080831A8000835A80008952800084F
:10007000A9280008BD280008D1280008E5280008A4
:10008000F92800080D290008891D0808891D08089D
:10009000891D0808891D0808891D080839A8000855
:1000A0004127000869270008912700082D2700082C
:1000B000B9270008CD270008E1270008891D080896
:1000C000891D0808891D0808891D0808891D080858
:1000D000891D0808891D080895250008A125000824
:1000E0003DA80008891D08085D4600081D28000875
:1000F000452800086D280008092800082129000863
:10010000891D0808891D0808F5270008891D0808A9
:10011000AD250008B9250008891D0808891D0808B3
:1001200035290008492900085D29000871290008BF
:1001300085290008891D0808891D0808891D0808E7
:10014000891D0808891D0808891D0808A946000896
:1001500099290008AD290008C1290008C525000813
:10016000891D0808891D0808891D0808891D0808B7
:10017000891D0808891D0808891D0808891D0808A7
:08018000891D0808891D08080B
:1001C000D0E907239A423CBFC1685218D01A704741
:1001D000D0E9092300699A4238BF1218D31A0138AE
:1001E000C01A7047D0E90902101AB0FA80F040092D
:1001F000704700BF0246036A4069D168C05C0133A2
:100200008B4228BF00231362704700BF436A826994
:10021000D154436A0169426B01338B4228BF0023EA
:100220004362D36843F08003D3607047436B188800
:1002300010F0100002D01A889B880120704700BF80
:10024000436B99891A88890610B504460AD592B27B
:10025000900607D5E26A002A2AD09888216B80B2DE
:100260009047636B99891A88090692B210D51006D7
:100270000ED5D4E909128A4215D0A1692069895C9A
:100280000132C9B29980B2FBF0F100FB1122A262E7
:10029000998A1A88C90592B204D5D20744BF4FF68D
:1002A000F7721A8010BDDA6822F08002DA60EFE798
:1002B0009B88E2696169DBB28B54E269E168636B38
:1002C0000132B2FBF1F001FB1022E261CAE700BF8C
:1002D000036942681F2B10B40AD95468A3F1200C9B
:1002E000202101FA0CF1214207D15DF8044B70473F
:1002F0001468202199402142F7D081690024C86800
:100300000C7480684C68016821F00101016020686C
:1003100094F805C00C4C818934F81C4089B221EA5C
:1003200004011F2B818107D9A3F1200120238B40D9
:100330005DF8044BD3607047202101FA03F35DF8A8
:10034000044B9360704700BFBC24080882B00922A8
:10035000274B8DF80720DA68D00319D4DA68D10664
:1003600040D4DA68D20541D4DA6812F0E00F3BD10C
:10037000DB6813F0020F0CBF092308238DF8073048
:100380009DF80730012B0AD09DF8070002B0704796
:1003900001238DF807309DF80730012BF4D1144A62
:1003A00012E0D368DB0519D4D36813F0E00F17D13E
:1003B000D36813F0020F0CBF092308238DF8073010
:1003C0009DF80730012BDFD1D168C8034FF001033E
:1003D000F4D4D368D906E4D50623EFE70223EDE78A
:1003E0000723EBE70623D4E70723D2E70223D0E76E
:1003F000003C0240704700BF704700BF704700BF1D
:1004000001207047034BD3E90003C01AC0F30A0070
:10041000704700BF20220020054AD2E9001399420C
:10042000FDD0D1180133C3F30A03087A5360704733
:1004300020220020064BD3F8080800B97047D3F8F3
:100440000808A0F10500B0FA80F04009704700BF2D
:1004500020220020012380F849307047044BD3E963
:100460000003C01AC0F30A00C0F50060704700BF67
:100470002022002010B5D0F8E83504461B699847C3
:10048000032384F81231002010BD00BF08B50422F8
:1004900090F81211D0F8E83580F8131180F8122185
:1004A000DB689847002008BD08B5D0F8E435DB6963
:1004B00003B19847002008BD08B5D0F8E4351B6AA1
:1004C0009847002008BD00BF08B5D0F8E4355B6A46
:1004D0009847002008BD00BF70B5037805460E465A
:1004E0001446DBB1013080F0EBFA431CDBB2013380
:1004F0005B00DAB223800323327073702C7864B10E
:100500002846022300215A1CD2B2F454B15410F8E8
:10051000014F0233DBB2002CF5D170BD022213462D
:10052000E8E700BF10B5074C2068FF2808D006494F
:10053000D1F80C2801F5016100F082F8FF23236057
:10054000002010BD0000002020220020432301488D
:100550000B80704704000020122301480B80704775
:1005600048000020042301480B8070475C000020F5
:1005700010B5044C04480A462146FFF7ADFF20465B
:1005800010BD00BF382A002074E0080810B5044CE4
:1005900004480A462146FFF79FFF204610BD00BFD2
:1005A000382A002080E0080810B5044C04480A46A8
:1005B0002146FFF791FF204610BD00BF382A0020DA
:1005C00088E0080810B5044C04480A462146FFF7A5
:1005D00083FF204610BD00BF382A002094E00808A1
:1005E00010B5044C04480A462146FFF775FF204623
:1005F00010BD00BF382A0020A0E00808704700BFE7
:10060000704700BF704700BF704700BF704700BF12
:10061000704700BF704700BF044B00200522C3F89D
:100620000828C3F81809C3F81C09704720220020C5
:10063000024B0020C3F80808704700BF20220020AA
:10064000212838B50C4625D0222816D0202812D1D2
:1006500089B1072A0FD1174DD5F81C3913B1096894
:10066000002098472168A288A379C5F82019A5F829
:10067000242985F82639002038BD0029FBD0022A1C
:10068000F9D10C4BD3F81839002BF4D0098800208D
:100690009847F0E70029EED0072AECD1054BD3F8B4
:1006A0002019B3F8242993F826392160A280A37178
:1006B000E1E700BF2022002010B4114CD4E9003241
:1006C0009A1AC2F30A020A44B2F5006F13D871B144
:1006D00001444A1E013810F801CFE118904203F19D
:1006E000010381F808C0C3F30A03F4D1236000209A
:1006F0005DF8044B704702205DF8044B704700BF63
:100700002022002010B58121044676F0A5F920466C
:10071000012176F0A1F92046822176F09DF9FFF7BC
:1007200087FF002010BD00BF034610B4D9691A69C5
:10073000002040F20114A3F844410860D1699C6D87
:1007400021F002014FF0010CD161A3F89CC320609D
:10075000D369044923F4003381F827095DF8044B79
:10076000D361704720220020202301480B8070476E
:1007700060000020122301480B8070478000002099
:10078000042301480B807047940000200A4608B5F6
:10079000054920B90548FFF79FFE034808BD0448F6
:1007A000FFF79AFE004808BD482B0020B0E008087B
:1007B000C8E0080810B5044C04480A462146FFF773
:1007C0008BFE204610BD00BF482B0020E0E008084B
:1007D0001C48D0F8E837D0F8EC2710B59B184FF03C
:1007E0001A040C8001D1184810BD174AD0F8EA0746
:1007F00002F1100411464FF0000E4FEA137CB3F1E2
:10080000204F34BF0CF1300C0CF1370C81F802C0D2
:1008100081F803E002318C424FEA0313EDD102F17B
:1008200008040021030FB0F1204F34BF30333733B9
:100830009374D174023294424FEA0010F2D102480C
:1008400010BD00BF00F0FF1F9800002010B5044C41
:1008500004480A462146FFF73FFE204610BD00BF70
:10086000482B0020F4E0080810B5044C04480A4660
:100870002146FFF731FE204610BD00BF482B002067
:1008800000E10808034BD3F8B42BB3F8B83B13834B
:1008900000207047202200204FF40070034B1060AE
:1008A000D3F8F03D0B600020704700BF20220020ED
:1008B00000207047012070470120704700207047DA
:1008C00010B41C6994420CD394460A4661448C428D
:1008D000996938BFA4EB0C0261445DF8044B7CF0CD
:1008E0001FBC5DF8044B7047704700BF704700BFE6
:1008F000D0ED007AD0ED036A30EE677AE6EE877AC3
:10090000B0EE670AC0ED007A704700BF90ED017A43
:10091000B5EE407AF1EE10FAF0EE407A09D19FED93
:100920000D7A60EE870AF7EE006A86EEA07A80ED17
:10093000017A31EE077A90ED000A80ED021AC1EEDD
:10094000076A77EEC07AC0ED036AA6EEA70A80EDCB
:10095000000A7047DB0FC940D0ED056AD0ED017A7F
:1009600090ED066AD0ED025A90ED035AC0ED066A8A
:10097000B0EE407A26EEA70AD0ED007A80ED057A37
:10098000A7EE870AD0ED077AA5EE860A90ED086AF1
:10099000D0ED045AC0ED087AA5EE670AA5EEC60AA6
:1009A00080ED070A704700BFF0EE406AD0ED007A94
:1009B00090ED050A90ED037A90ED016AD0ED025AB0
:1009C000A7EEA60AD0ED047A27EE407A67EEC07A49
:1009D000A6EE267AE5EEA67A90ED066AC0ED067AD6
:1009E00036EE076A80ED056A704700BF03685A1C3F
:1009F00002601970704700BF2DE9F04FD0E9003157
:100A000085684A1C00EB8104F1EE407A92FBF3F614
:100A1000002D03FB1622426089B084ED200AC4ED4C
:100A2000407A40F346815A189FEDA46A0692591EF7
:100A30006A1C079200F1800900F5807BF0EE466A9F
:100A400002224FF0010A884606998C1A94FBF3F1B2
:100A500003FB1144611C91FBF3F003FB101101EB4C
:100A60000A0009EB840E0BEB840C924590FBF3F427
:100A70009EED007ADCED007A03FB1400A3EB020686
:100A800080F2CD80CDE901ECCDE9032637460C4656
:100A90000546059031E0A34209EB850C0BEB85067A
:100AA00005F1010531DD09EB84000BEB840E2246D4
:100AB000013490ED006AD6ED005ADEED006AB4EE26
:100AC000C76AF1EE10FA07DD9CED005AB4EEC56A74
:100AD000F1EE10FA00F38680F4EEE76AF1EE10FA18
:100AE00004DDF4EEE56AF1EE10FA13DC0137474558
:100AF000B0EE467A2EDAF0EE667AAB42CBDCA34259
:100B00005E46CC464FF00105CDDCDE46484601246A
:100B10000022CEE7F4EEE75AF1EE10FA58BFF0EEFD
:100B2000657ABAF1010FCEED007A18BF01200CD022
:100B30000132934200F10100CEBF0BEB82065E460C
:100B400000228245C6ED007AF2D101374745B0EE6A
:100B5000677AD0DBDDE901ECDDE903260598DEEDFF
:100B6000006A9CED006A30E08B4209EB800C0BEBD5
:100B7000800700F1010030DD09EB81050BEB810EF0
:100B80000C46013195ED007AD7ED005ADEED007A82
:100B9000B4EEE67AF1EE10FA06D59CED005AB4EE0A
:100BA000C57AF1EE10FA4DD4F0EE476AF4EEC67A4B
:100BB000F1EE10FA04D5F4EEE57AF1EE10FA5DD418
:100BC000B0EE676A0136B04529DD8342CCDC8B424A
:100BD0005F46CC464FF00100CEDCDE464D4601219B
:100BE0000024CFE7B4EEC75AF1EE10FA58BFB0EECA
:100BF000457ABAF1010F80ED007A3FF46DAF1046EF
:100C000001260130834206F10106CEBF09EB800CBC
:100C1000CC46002056458CED007AF2D15CE707996E
:100C20000AF1010A8A4502F1020208F1FF387FF455
:100C30000BAF76EEC66AF6EE007A26EEA70A09B08A
:100C4000BDE8F08FB4EEE65AF1EE10FAD8BFF0EE40
:100C5000456ABAF1010FC5ED006AA7D02546012704
:100C60000135AB4207F10107CEBF09EB850CCC463D
:100C700000255745CCED006AF2D197E7F4EEC65A4D
:100C8000F1EE10FAD8BFB0EE656ABAF1010F8EED41
:100C9000006A97D001250134A34205F10105CEBFBA
:100CA0000BEB84075F460024554587ED006AF2D1BF
:100CB00088E79FED020A09B0BDE8F08F0000000050
:100CC00003685A1C02601970704700BF024BD3F8CA
:100CD000200E03681B681847202200200079704707
:100CE0000079C0F34010704700794009704700BF99
:100CF00090F83C20034602F0FF0012B1002283F876
:100D00003C2070472DE9F84345697DB90768C7F372
:100D10000D0804460E46B8F1000F0AD0D6F8008040
:100D2000FFF714FB09283BD06FF001052846BDE80A
:100D3000F883514B9F422AD303F580439F4224D32B
:100D400003F580439F427FD34C4B9F427FD903F5ED
:100D500080339F427ED903F500339F427DD903F54E
:100D600000339F427CD903F500339F4269D903F5D4
:100D700000339F4277D903F580239F4276D9B7F19C
:100D8000016F76D305200DF021FC4FF00808FFF726
:100D9000DDFA092821D04FF0FF352846BDE8F88359
:100DA000374E336923F440733361336943F400737E
:100DB0003361336943F001033361C7F80080FFF703
:100DC000C5FA3369092823F001033361ACD12368E4
:100DD000043323602846BDE8F883DFF8A490D9F8EF
:100DE000103023F44073C9F81030D9F8103043F4B0
:100DF0000073C9F81030D9F8103023F0F803C9F89F
:100E00001030D9F8103043EA080343F00203C9F860
:100E10001030D9F8103043F48033C9F81030FFF7A0
:100E200095FAD9F8103023F00203C9F81030D9F838
:100E30001030092823F0F803C9F810303FF46EAFE2
:100E4000A9E74FF03808A2E74FF010089FE74FF0EE
:100E500018089CE74FF0200899E74FF0280896E71C
:100E60004FF0300893E74FF0400890E74FF0480804
:100E70008DE74FF058088AE700400008FFFF0008A0
:100E8000003C02402DE9F0410446D0E90030134413
:100E900083421DD80D4601EB0208B2B104F10C07E4
:100EA000002601E0A84510D023695A1C2261234482
:100EB00015F8011B1973042AF4D139462046FFF7AF
:100EC00021FFA845C4E90460EED16069BDE8F08166
:100ED0004FF0FF30FAE700BF2DE9F0411F4E80468A
:100EE0000B4696F8242E002AFBD19BB343445F1E89
:100EF00008F1FF38D6F8283ED6F82C2E0133C3F37C
:100F00000A039A4216D10CF0C5FC04460D460CF0BB
:100F1000C1FC001B61EB0501B0F57A7F71F10001A6
:100F2000F5D3D6F8283ED6F82C2E0133C3F30A03A6
:100F30009342E8D0D6F8282ED6F8283E18F8011F9C
:100F400032440133C3F30A03B84582F8301EC6F8B1
:100F5000283ECFD10020BDE8F08100BF2022002034
:100F60000A4B10B5D3F8084804B910BDD3F80838B7
:100F7000052BFAD1064C002A0846D4F8383511461C
:100F8000F3DDFFF7A9FFD4F8383510BD202200208B
:100F90001833002090F84820531C0244DBB280F83C
:100FA000483082F8341090F849204AB1132B06D902
:100FB000002280F848200C4AD2F8081829B9704756
:100FC00080F84820002BF6D17047D2F80828052A6F
:100FD000F5D110B5054C19463430D4F83835FFF743
:100FE0007BFFD4F8383510BD2022002018330020B4
:100FF00090F848100023A0F8483001B97047094B19
:10100000D3F80828002AF9D0D3F80838052BF5D1F1
:1010100010B5054C3430D4F83835FFF75DFFD4F8FF
:10102000383510BD20220020183300202DE9F0476C
:10103000564E1F4606EB80039C68002C00F0A280F1
:1010400004F13E03A36104F59F73E3614FF48073E1
:10105000C4E904332836236866600546E16094F8E5
:101060003D00A363914609F0A1FC804694F8440238
:1010700094F83CA0261D002853D194F8450250BB9B
:10108000D4F840326BBB3B0731D419F0020F5FD16B
:1010900019F0010F48D1D4F8483294F9471294F866
:1010A00047221B010029DBB20DDB3949881880F883
:1010B00000335009012302F01F02934041F8203011
:1010C0003046BDE8F087334902F00F021144304644
:1010D0000B76BDE8F08773F053F8D4F84032002B5C
:1010E000D1D02D4A116B0B4313633B07CDD501358E
:1010F000EDB207F01003B8F1000FCCD040F2067249
:1011000088F80850A8F8062094F84622002B34D11D
:1011100017F0200F0CBF32211221404609F036FE95
:10112000B9E773F02DF8A8E7504609F03FFC6A1CB8
:10113000D2B20028AFD0027240F20662012DC28006
:1011400094F846220CBF3221022109F01FFEA2E7CB
:101150006B1CDBB2B8F1000F9AD088F8083040F26F
:101160000653A8F8063094F846224046022109F0BA
:101170000DFE19F0010F8ED0D6E70221404609F08E
:1011800005FE88E726463046BDE8F087BC240808FF
:1011900000E100E0FCEC00E0003802402DE9F047FF
:1011A000038A8489A4B21C4082B047D08146884615
:1011B0004FF0004501F14C0701F13406B4FA84F315
:1011C00025FA03F2D24391B2A9F8101014401B3B48
:1011D000B8F1000F5FD0042B2ED8DFE803F052489F
:1011E0003D320300D8F80C30D9F82CA033B19B68FD
:1011F00023B11FFA8AF108F104009847D8F8243087
:1012000033B19B6823B11FFA8AF108F11C0098479B
:10121000D8F83C3033B19B6823B11FFA8AF108F14A
:1012200034009847D8F8543033B19B6823B11FFA83
:101230008AF108F14C009847002CBFD102B0BDE8FC
:10124000F087D8F80C30D9F834105B6808F1040046
:101250009847002CB2D1F1E7D8F82430D9F83810EB
:101260005B6808F11C009847002CA7D1E6E7D8F886
:101270003C30D9F83C105B6830469847002C9DD133
:10128000DCE7D8F85430D9F840105B683846984706
:10129000002C93D1D2E7042B07D8DFE803F0190321
:1012A000140F0A00D9F83C300193019B002C85D122
:1012B000C4E7D9F82C300193019BF7E7D9F8343013
:1012C0000193019BF2E7D9F838300193019BEDE7D8
:1012D000D9F840300193019BE8E700BFF8B5264CF0
:1012E00094F8242E012A034603D0022A09D00020B4
:1012F000F8BD224ED6F83C558DB984F8245E002006
:10130000F8BD002540F20112C0E95455C0E9565518
:10131000A0F8442100F5A27175F09AFCEDE7402D8C
:1013200020D94027D4F82C1E154AC3F858710A4416
:10133000C3E9542240F20112A3F844210022C3F869
:101340005C2103F5A271184675F082FCD4F82C3E9E
:101350003B44ED1BC3F30A03C4F82C3EC6F83C55CE
:101360000020F8BDAAB2402A01D02F46DAE70222B7
:1013700084F8242ED5E700BF202200201833002057
:101380005030002001EB810138B500EBC1010F4D59
:10139000B1F88C1304462846FFF78EF9E378C4F8B9
:1013A000A853012083424FF000024FF04001C4E9EE
:1013B000EC12A4F89C0304F56771204608BFC4F83A
:1013C000AC5375F045FC002038BD00BF58380020F4
:1013D000F8B52A4CD4F880350F2B04D05A1CC4F829
:1013E00080250020F8BD264D95F8243E0022C4F843
:1013F0008025002BF5D1D5F82C2ED5F8283E9A4221
:10140000EFD0D5F82C2ED5F8283E9A422DD8D5F815
:10141000286ED5F82C3EF61A402E2BD8B3B2402BAE
:1014200013BF3746402702230123D5F82C2E85F819
:10143000243E144BC0F858711344C0E9543340F2B1
:101440000113A0F844310023C0F85C3100F5A2710B
:1014500075F0FEFBD5F82C3E3B44F61BC3F30A03A4
:10146000C5F82C3EC4F83C65BBE7D5F82C6EC6F534
:101470000066D1E701234027D7E700BF18330020DB
:10148000202200205030002010B5324B93F89025D8
:1014900093F8A4C5D3F88C35044613B152EA0C0274
:1014A00031D00123E06984F8463140F20112A4F8FA
:1014B000442102682849002AA8BFC2F380739B0315
:1014C00001EA124143F020030B4363F31F42BCF1D6
:1014D000020F026000D010BDE278204BC4F8A833A0
:1014E0001F200021C4E9EC01012A4FF00101A4F8FA
:1014F0009C1308BFC4F8AC3304F567712046BDE8FF
:10150000104075F0A5BB012175F06CFA0122E0696D
:1015100084F8462140F20113A4F8443101680029FF
:101520000A460CDBC1F380730B4C9B0343F0200392
:1015300004EA11410B4363F31F42026010BD064BE6
:1015400003EA114343F4804343F0200363F31F4253
:10155000026010BD18330020DFBFFFFF9C38002061
:101560002DE9F041B0F8CC15D0F8CE35B0F8D25511
:10157000B0F8D085C0F84051012284B080F8112124
:1015800001F01F02012A044600F2CC56ADF8081003
:10159000C1F3072ECDF80A30ADF80E504FEA134CC8
:1015A00051D0022A7746C9B29BB210D0002A55D139
:1015B000BEF1090F4BD8DFE81EF08900AD004A00EC
:1015C000C8004A005C01DF004A001301330101F04A
:1015D000600120295FFA8CF272D0012F00F0B881EF
:1015E000032F00F0A181AFBB90F81231022B00F065
:1015F000E381032B2BD11CF0800F40F0E98102EB3B
:10160000820200EBC20393F87623003A18BF01224E
:10161000C24D02234FF48071C4E94E3384F8113176
:10162000C4F83031A4F81C1105F2B4530021C4F8F9
:101630003411C4E94A3304F58E712046C5F8B42547
:1016400075F0A4FA06E090F81231032B0ED0204674
:1016500075F090F9002004B0BDE8F08101F0800140
:1016600075F0C0F9002004B0BDE8F0815FFA8CFC91
:10167000BCF1010FEBD8D0F8E43502A99B6898477C
:10168000BDF80E30002BE5D1C4E94A33C4E94C3330
:1016900004214FF4807284F81111A4F81C2104F580
:1016A0008E71204675F072FA636D9D4A1A61E27878
:1016B000012ACFD15E614FF0802219681A60C9E714
:1016C000D0F8E43502A99B689847C3E790F8123137
:1016D000023B012BBBD8914BD0F818210021C3F855
:1016E000AC1512B10222C3F8AC258E4A02234FF486
:1016F00080700021C4E94C31A4F81C01C4E94E33C8
:10170000C4E94A2284F8113104F58E71204675F03F
:101710003DFA9FE790F81221023A012A97D8012B4F
:1017200098D1D0F8E43500259B68C0F8185102A97B
:10173000984704224FF48073C4E94A55C4E94C55D4
:1017400084F81121A4F81C31A9E7012B00F03B819A
:10175000022B7FF47FAF5FFA8CF3002B7FF47AAF1C
:1017600003694FEA1C22023A5B68032A00F2BD813A
:10177000DFE802F0B6CED2D01E0A022EADF8065037
:1017800000F08A81032E00F04E81012E7FF45FAFBE
:10179000D0F8EC3580781B680DF106019847BDF84C
:1017A0000630002B3FF456AFBDF80E20002A3FF460
:1017B00051AF934228BF13464FF480720221A4F820
:1017C0001C210022C4E94A0084F81111C4E94E33F7
:1017D000C4E94C3204F58E71204675F0D7F939E72B
:1017E000012D7FF434AF90F81231022B00F0088104
:1017F000032B7FF42CAF4FF4807200F58873022125
:10180000A0F81C21002280F81111C0E94E55C0E952
:101810004A33C0E94C5200F58E7175F0B7F919E7FB
:10182000DDB23E4F012D87F8A5553FF610AF90F879
:101830001231022B00F0D880032B7FF408AF002D6B
:1018400000F0358190F81011012910D0D0F8E4355E
:101850005B68984797F8A515D4F8E43584F810111B
:101860001B6820469847D4F8E8359B6898470023C2
:101870000AE758EA05027FF4EAAE90F8121103294C
:101880003FF4E5AE03F07F0580F81451006911467E
:1018900063F30A11036819430423016084F81131CA
:1018A0004FF48073C4E94A22C4E94C22A4F81C31E5
:1018B00004F58E71204675F069F9636D184A1A6156
:1018C000E278012A06D0002D00F0FC80022384F883
:1018D0001231BFE65E614FF0802219681A60F2E7AC
:1018E00002210E4861F306130022C0F8B03504232C
:1018F000C4E94A22C4E94C2284F8113101224FF490
:10190000807304F58E7184F81621A4F81C31C8E6A2
:101910000321E6E70521E4E70421E2E7183300208C
:1019200018000860C438002090F81211022943D032
:1019300003297FF48CAE23B9510602D0114675F00D
:1019400051F8D4F8E4359B6802A9204698478EE701
:1019500090F8121102292FD003297FF478AE002BC2
:101960007FF478AE12F07F0181D01CF0800F40F040
:10197000AD8002EB820100EBC10181F8763381F882
:101980007533282381F8742303FB020300EB8201E3
:1019900093F87723496D0B68023A012A23F4001368
:1019A0008CBFC3F30072012262F31C73D4F8E425E8
:1019B0000B60936802A9C8E753063FF44BAE11468B
:1019C00075F010F846E6D0F8E425C0F81831F0E7D5
:1019D00002F07F0202EB820200EBC20393F81E21A9
:1019E000003A18BF012213E6002D3FF4A2AE0121F8
:1019F0000322D0F8E43580F8101180F812212FE787
:101A00003B4A80F811314FF480710023A0F81C117B
:101A1000C0E94E55C0E94A22C0E94C5300F58E7129
:101A200075F0B4F816E6DBB2052B3FF610AEDFE832
:101A300003F02B231B130B03D0F8EC3580789B6944
:101A40000DF106019847AAE6D0F8EC3580785B697D
:101A50000DF106019847A2E6D0F8EC3580781B69B5
:101A60000DF1060198479AE6D0F8EC358078DB68EE
:101A70000DF10601984792E6D0F8EC3580789B6826
:101A80000DF1060198478AE6D0F8EC3580785B685E
:101A90000DF10601984782E6D0F8E43580789B6A1C
:101AA0000DF1060198474670C4F8F00577E602226A
:101AB000D0F8E43580F8122180F810515B6829468F
:101AC000984736E6012384F81231C3E5282202FB49
:101AD000010080F81C1104EB810180F81E3180F8B0
:101AE0001DE190F81F21896955E70121F9E600BF42
:101AF000C038002010B5044629B990F81121032AF6
:101B00000DD0002010BDD0F8E4359B69002BF8D033
:101B100090F81221032AF4D19847002010BDD0F884
:101B200090230B46D0F87C138A4219D9521AC0F878
:101B3000902394F803C0D0F880038A4228BF0A4655
:101B4000BCF1010F92B234D0C4E9E22304F55D7117
:101B5000C4F88003A4F87433204675F017F8D0E772
:101B6000D0F8E4351B691BB190F81221032A1ED06E
:101B700000234FF480720421C4E94A33C4E94C3392
:101B800084F81111A4F81C2104F58E71204674F01C
:101B9000FDFF636D0D4A1A61E278012AB1D104F2AA
:101BA000CC545C614FF0802219681A60A9E798470D
:101BB000DEE70844C4E9E22304F55D71C4F880035C
:101BC000A4F87433C4F88403C6E700BF18000860A3
:101BD00038B5044649B990F81131022B11D094F868
:101BE0001631012B39D0002038BDD0F8E4355B69BF
:101BF000002BF8D090F81221032AF4D19847002046
:101C000038BDD0F83831D0F8242193422FD990F83C
:101C100003C09B1ABCF1010F0D46C0F83831D0F853
:101C200028116ED09BB2C0F830314FF48073C0E9F8
:101C30004A11C0F8345100F58E71A0F81C3174F0CF
:101C4000A5FFC4E9E255C4F8805304F55D71A4F81A
:101C50007453204674F09AFFC1E73F4B2269D3F8D2
:101C6000B0155160002384F81631002038BDD0F83B
:101C70003C31B3FBF2F502FB15350DBB9A421FD880
:101C8000D0F8402193421BD24FF48073A0F81C314E
:101C900000F58E71C0E94A55C0E94C5574F076FFE5
:101CA000E378C4F84051012BC4E9E255C4F88053ED
:101CB000A4F8745308BFC4F8845304F55D71C8E7F1
:101CC000D4F8E435DB681BB194F81221032A15D04F
:101CD000E27800230521012A84F81111C4E9E233D6
:101CE000C4F88033A4F8743304F55D7124D0204621
:101CF00074F04CFF636D194A1A6170E720469847EB
:101D0000E6E79BB21144C0F830314FF48073C0E96C
:101D10004A11C0F8345100F58E71A0F81C3174F0EE
:101D200035FFC4E9E255C4F8805304F55D71A4F8A9
:101D30007453C4F884538CE7C4F88433204674F099
:101D400025FF636D0548186104F2CC525A614FF0CB
:101D500080211A68196042E71833002018000860D3
:101D600070B50B7813F060020D46044624D0202A8B
:101D700004D0204674F0FEFD022070BDCA88487869
:101D80001AB31B0640D5324E3146FEF759FCEB889C
:101D90004FF480720221A4F81C21002284F8111152
:101DA000C4E94E33C4E94A66C4E94C3204F58E7185
:101DB000204674F0EBFE06E04B780A2B10D00B2B7C
:101DC00008D0062BD5D0002070BD02221144FEF7AA
:101DD00037FCF8E78B78C3BB1E4AC2F8B835F2E788
:101DE000022180F811114FF48071A0F81C111A49DA
:101DF0000123C0E94A11C0E94E33C0E94C3200F575
:101E00008E7174F0C3FEDEE71449154B0860E0786C
:101E1000C3F80C28002103F5016301284FF00305E6
:101E2000C4F88C13A4F87413C4E9E42284F81151A3
:101E3000C4F88823C4F8803304F55D7108BFC4F882
:101E40008433204674F0A2FEBDE774F093FDBAE738
:101E5000302A002018330020D03800200000002055
:101E600020220020002310B519460446402274F0B9
:101E700023FE802120460023402274F01DFED4F86A
:101E8000E835A078012284F812215B689847002089
:101E900010BD00BF10B5022304464022812174F01A
:101EA0000BFE204602234022012174F005FE20464D
:101EB00003230822822174F0FFFD104B0222A3F8B5
:101EC0004C20FEF7A9FBE2780D4BC4F8A833402163
:101ED000C4F8B013012A4FF000004FF00101C4F81C
:101EE000B403A4F89C13204604F5677108BFC4F836
:101EF000AC3374F0ADFE002010BD00BF0000002028
:101F00005838002030B5812183B0044674F0A4FD18
:101F10000121204674F0A0FD2A4900250223402219
:101F200081F827592046812174F0C6FD0121022342
:101F30004022204674F0C0FD234BD3F8BC2583F823
:101F4000A4551268284690470095009AE1681F4BF7
:101F500042F010020092009A0A610A690092013B65
:101F600002D0009AD006F8D400230193019B43F0DD
:101F700020030193019A154B012060F38A1201920C
:101F8000019A0A610A690192013B02D0019A920604
:101F9000F8D4E2780E4BC4F8A8331F200021C4E91E
:101FA000EC01012A4FF00101A4F89C13204604F52E
:101FB000677108BFC4F8AC3374F04AFE002003B068
:101FC00030BD00BF2022002018330020410D030047
:101FD0009C3800202DE9F843DDF820800F46154697
:101FE0000021202204461E467CF0B2FCB8F1000F0E
:101FF0000CD0D8F80030E3811B0C2382D8F80430D1
:10200000B8F80A20E3821B0C6282238338467EF0F4
:1020100057FDEB0619D4431EB8B107EB000C01E0E5
:10202000013B12D31CF801EDBEF12E0FF8D1C01AFE
:10203000421E032AA8BF0322082B03F10109A8BFEF
:1020400008239046B9441A4606E008280246B946D5
:10205000A8BF08224FF000084FF020333946236014
:10206000636020467BF05CF804F10800154B238187
:102070004246494683707BF053F8611EE21D11F819
:1020800001CFACF16103192B9CBFACF1200C81F89E
:1020900000C09142F3D104F10A0011F8013FA3F10D
:1020A0006102192A9CBF203B0B708142F5D1182395
:1020B0002373330CA382E572099B6683E361BDE859
:1020C000F88300BF202020002DE9F04FDFF858B43E
:1020D000DBF8B40B0C46BBF8B81B418385B0002B72
:1020E00063D01344174604F5FE7A99461FE0002F8B
:1020F00069D0DBF8FC3DBB4200F0CB80DBF8F83D5B
:10210000BB4200F0FD80DBF8003EDBF8041EBB4262
:1021100050D8B94200F27581791A204671F02CFF2F
:1021200001374F4504F500740AF5007A39D0DBF821
:10213000083EBB42DBD8DBF8185EFB1A296BDA08D5
:1021400002328A4203F0070602D3AB6B9A420BD9E4
:1021500029461046029271F0DFFE029A05460028D9
:1021600000F06F81CBF8180E2B79002B40F0238103
:10217000D5F82880B8F1000F00F05C812B6BD21AE3
:10218000EB6806EBC20203EB422220462B464FF4DB
:1021900000710137C0474F4504F500740AF5007A15
:1021A000C5D1DBF8B40BBBF8B81B0183002005B028
:1021B000BDE8F08FB942AFD94FF40072002120463C
:1021C0007CF0C6FBACE74FF40072394620467CF049
:1021D000BFFB802384F8BE310C2384F8C231DBF8C6
:1021E000F81DC54ADBF8F03DC4F8C6119142C4F8A9
:1021F000CA3100F30B81C14AC14D82FB010285FB4C
:1022000001050A44C817C0EB6212C0EB2530BD4D72
:1022100084F8C10185FB0265C2EB82168010891B20
:10222000013120F03F0015440843D117C1EBE511FF
:102230000A4484F8BF21B04A84F8C001013B9342AC
:1022400000F3F080AD4AAE4882FB031280FB03101E
:102250001A44D917C1EB6212C1EB2031A94884F8A6
:10226000C51180FB0250C2EB821589105B1B013344
:1022700021F03F0110441943D317C3EBE0131A4474
:1022800084F8C41184F8C3214AF65523A4F8FE311A
:1022900046E74FF0FF3384F8EC3184F8ED3184F8F1
:1022A000EE3184F8EF315223237063706123A37001
:1022B00084F8E7314123E37084F8E6317223002586
:1022C00084F8E43184F8E531DBF8103EC4F8E831F5
:1022D0004FF4F0722946201D7CF03AFB552384F818
:1022E000FE316FF05503C4F8F051C4F8F451C4F84E
:1022F000F85184F8FC5184F8FD5184F8FF310FE760
:102300004FF40072002120467CF022FB7E4B03CB71
:1023100045F6EB0323809023C4F80710A370022234
:102320000821F823C4F80300617322746375DBF895
:10233000F03D2273A27384F82C20DBF8F82D9B1A51
:102340002362DBF8002EDBF8043E9B1A6362002355
:10235000E372E3736377A377E37784F82D3084F82F
:102360002E3084F82F3084F83130684BA361684BED
:10237000C4F842303E232377012384F83030654A85
:10238000802384F8403084F846104AF65521A4F89A
:10239000FE1103CA604BC4F84700C4F84B1003CBCE
:1023A0001388A4F84F309378C4F85200C4F856103C
:1023B00084F85130B4E64FF40072002120467CF0DE
:1023C000C7FA002E44D12B6C04F12008002B7BD0DF
:1023D0002B6B52491122CDE900662046FFF7FAFD2A
:1023E0002B6C1A6C002A7ED01B6B4D49CDE9006620
:1023F00040461122FFF7EEFD04F140084FF4E07370
:102400006DE0F91A204671F0B7FD89E6FF2284F8E5
:10241000C1214FF6FF72A4F8BF21374A013B934216
:102420007FF710AFFF2384F8C5314FF6FF73A4F890
:10243000C33129E741464FF4007220467CF088FA08
:102440006EE6384A231F43F8042F9A45FBD167E60E
:10245000D5E910253301002A43D0023B002D3FF47B
:102460005FAE013BAD6CF9D1A0464FF40073002D77
:102470003FF456AECDE9027A08EB0306A24608E027
:102480000024CDE900C4FFF7A5FDAD6CBDB1B0459A
:1024900015D02C7929682B6B404605F11C0C1122B4
:1024A00008F12008002CEBD16A792C6942F0210256
:1024B000CDE900C4FFF78EFDAD6C002DE7D1544689
:1024C000029FDDF80CA02BE6CDE900663346DBF871
:1024D000F41D08222046FFF77DFD4FF4F0736D6C6C
:1024E000C5E7013BBAE7CDE900660D4933464046F2
:1024F0001122FFF76FFD7FE7FF03FB0083200882B7
:10250000975545418180808010E108083F00FF0019
:1025100029940E0D1CE1080828E1080810E80808B5
:1025200074E90808DEADBEEF202200208C46134679
:102530000146624618464CF0ADBC00BF1049114B35
:10254000D1F8882042F4700210B4C1F888201A68CB
:102550000D4C002042F001021A6098601A6822F0C7
:10256000847222F480321A605C601A68074C22F48C
:1025700080221A60D8608C605DF8044B704700BF01
:1025800000ED00E000380240103000240000000898
:10259000704700BF0148FDF753BE00BFB8000020E0
:1025A0000148FDF74DBE00BF040300200148FDF7C0
:1025B00047BE00BF500500200148FDF741BE00BFE7
:1025C0009C0700200148FDF73BBE00BFE809002042
:1025D000704700BFB0B130B443688D685A791C6849
:1025E000022393404A689BB26AB1A2899DB192B21C
:1025F00013438160A381A3899BB243F00103A381AC
:1026000030BC70477047A28992B222EA0303A381CB
:1026100065B18160EFE722F001021204120CA28181
:10262000A289816092B21343A381E9E7A38923F0D1
:1026300001031B041B0CA3818160E1E738B5D0E9DD
:10264000004007EE902A0068324A334B2468D3F8E2
:10265000303C2468013990428DB210D002F580627E
:1026600090420CD002F57052904208D002F5806280
:10267000904204D002F58062904218BF5B0807EEDA
:10268000103AF8EE677AB8EE477ADFED246A87EE03
:10269000270A30EE260A76F0C7FD1E492388421E1F
:1026A0008C4292B29BB21AD01D498C4217D0B4F121
:1026B000804F1FD0A1F580318C421BD001F5806185
:1026C0008C4217D001F580618C4213D015498C42A1
:1026D00019D123800123E5622285A38238BD23F42A
:1026E0005C739BB223800023E5622285238601234D
:1026F000A38238BD23F45C739BB223800123E5627F
:102700002285A38238BD08498C42E2D023F440736D
:102710009BB2DEE700000140000000200AD7233C06
:10272000000401400010004000140040024B034828
:10273000D3F8C015FEF732BD183300200000014069
:1027400010B5064C0648D4F8C015FEF727FDD4F89E
:10275000E0150448BDE81040FEF720BD1833002006
:10276000000001400040014010B5064C0648D4F876
:10277000C015FEF713FDD4F8E4150448BDE8104079
:10278000FEF70CBD1833002000000140004401405A
:1027900010B5064C0648D4F8C015FEF7FFFCD4F877
:1027A000E8150448BDE81040FEF7F8BC18330020D7
:1027B0000000014000480140034B4FF08040D3F837
:1027C000C415FEF7EBBC00BF18330020024B0348D2
:1027D000D3F8C815FEF7E2BC18330020000400400F
:1027E000024B0348D3F8CC15FEF7D8BC18330020B1
:1027F00000080040024B0348D3F8D015FEF7CEBCCA
:1028000018330020000C0040024B0348D3F8DC15BD
:10281000FEF7C4BC183300200004014010B5064C7C
:102820000648D4F8DC15FEF7B9FCD4F8EC150448DA
:10283000BDE81040FEF7B2BC183300200004014090
:102840000018004010B5064C0648D4F8DC15FEF719
:10285000A5FCD4F8F0150448BDE81040FEF79EBC76
:102860001833002000040140001C004010B5064C45
:102870000648D4F8DC15FEF791FCD4F8F4150448AA
:10288000BDE81040FEF78ABC183300200004014068
:10289000002000400348D0F8403C13B100F634401B
:1028A00018477047000000200348D0F8603C13B17F
:1028B00000F6544018477047000000200348D0F845
:1028C000803C13B100F674401847704700000020A8
:1028D0000348D0F8A03C13B100F694401847704765
:1028E000000000200348D0F8C03C13B100F6B4400B
:1028F00018477047000000200348D0F8E03C13B1AF
:1029000000F6D44018477047000000200348D0F874
:10291000003D13B100F6F440184770470000002056
:102920000348D0F8203D13B100F614501847704703
:10293000000000200348D0F8403D13B100F63450A9
:1029400018477047000000200348D0F8603D13B1DD
:1029500000F6545018477047000000200348D0F894
:10296000803D13B100F674501847704700000020F6
:102970000348D0F8A03D13B100F6945018477047B3
:10298000000000200348D0F8C03D13B100F6B45059
:1029900018477047000000200348D0F8E03D13B10D
:1029A00000F6D45018477047000000200348D0F8C4
:1029B000003E13B100F6F4501847704700000020A5
:1029C0000348D0F8203E13B100F614601847704752
:1029D0000000002002683649002310B422F00102F2
:1029E000212488420260036043608360C360036106
:1029F000446138D02F4B98422ED02F4B98423CD078
:102A00002E4B984240D02E4B984232D02D4B9842BC
:102A100041D02D4B984246D02C4B984217D02C4B8E
:102A200098423CD02B4B984216D02B4B984224D046
:102A30002A4B984228D02A4B98421AD0294B9842C8
:102A400029D0294B98422ED0284B984208D14FF0DC
:102A50003D5243F8AC2C03E04FF4746243F8202C51
:102A60005DF8044B7047224B5DF8044B3D229A60A1
:102A70007047204A43F8642CF2E74FF474125DF873
:102A8000044B43F8382C70474FF074625DF8044BE8
:102A900043F8502C7047184A43F87C2CE0E73D225D
:102AA00043F8082CDCE7154A43F8942CD8E700BF1C
:102AB00010600240286002404060024058600240BE
:102AC0007060024088600240A0600240B86002402E
:102AD000106402402864024040640240586402408E
:102AE0007064024088640240A0640240B8640240FE
:102AF000006002403D000020400F002000003D200B
:102B0000214A936803F00C03042B10B43AD0082B2D
:102B10001FD01E4B1C4C0360A1681D4AC1F303115A
:102B2000114491F85C10CB404360A168C1F382214D
:102B3000114491F85C1023FA01F18160A1685DF8FD
:102B4000044BC1F342310A4492F85C20D340C36085
:102B500070475368516813F4800F536814BF0D4ACF
:102B60000A4AC3F3881301F03F01B2FBF1F202FB02
:102B700003F3054A5268C2F3014201325200B3FB2B
:102B8000F2F3C7E7034BC5E7003802400024F40026
:102B9000BC24080800127A0070B5446B8668A389CB
:102BA00023F400531B041B0CA381857990F805C006
:102BB0002B0303F40051C5F380000CF001032A023B
:102BC0009B001CF0020F4FEA003002F4806218BF35
:102BD00043F0080302431A43238A9BB223F4405371
:102BE0000B432382A38923F4B05323F00C031B046B
:102BF0001B0C1343A381A38A23F440731B041B0CF7
:102C000084B0A3826846FFF77BFF234B9C4205D02C
:102C100003F580639C4201D0029B00E0039BA289E4
:102C20001E49120403EB83034CBF7600B60003EB8E
:102C30008303B3FBF6F3A1FB0302A08952096426C8
:102C4000000406FB12334FEA02121CD41B0132337C
:102C5000A1FB0313C3F3431313439BB223812A073E
:102C6000A38A0AD59BB243F00803A382A3899BB22F
:102C700043F40053A38104B070BD23F008031B0488
:102C80001B0CA382F2E7DB003233A1FB0313C3F377
:102C900042131343E1E700BF001001401F85EB51D1
:102CA0002DE9F8431D46344B9DF820609DF8249093
:102CB00098428846174646D0304B98424BD0304B0E
:102CC000984250D02F4B984235D02F4B98422ED15E
:102CD0004B46324629460520FEF7A8F90446002354
:102CE000C4E90B87C4E90733C4E909336671A560F9
:102CF00084F806902046FFF74FFFF107626B0ED471
:102D0000B30707D493899BB243F4005393812046C1
:102D1000BDE8F883D36843F08003D360F2E74FF651
:102D2000DF731380D36843F02003D360E8E7002407
:102D30002046BDE8F8834B46324629460420FEF77C
:102D400075F90446CBE74B46324629460120FEF78B
:102D50006DF90446C3E74B46324629460220FEF78A
:102D600065F90446BBE74B46324629460320FEF789
:102D70005DF90446B3E700BF00440040004800404E
:102D8000004C00400050004000140140816003E707
:102D9000417101E78171FFE62DE9F043794F07EBBF
:102DA000C00985B005464FEAC00899F8380E07F00B
:102DB000FDFD044699F8390E07F0F8FD064699F82E
:102DC0003A0E71F0DDF96B1CDBB2002C00F0AB8029
:102DD00040F60C122372E280002E00F0B6803372AF
:102DE00040F60C232046F38004223A2107F0CEFF60
:102DF000042230463A2107F0C9FF07EB0803624A74
:102E0000D3F8344E944200F09680604B9C4200F020
:102E1000A2805F4B9C4200F0A980474497F83B3E5C
:102E2000022B32D0032B7CD05A495B4F012B08BFB9
:102E30000F46A6886846FFF763FE26F03F06029B12
:102E4000564AB3FBF7F13604A2FB0323360C46EADD
:102E50009346A680228822F001021204120C2280DE
:102E60008AB2C1F30B019B0C09B942F001024FF485
:102E7000967101FB03F34A49A1FB03139B0901333C
:102E80009BB242F4004223841FE0A6886846FFF705
:102E900037FE26F03F06029A404B3604A3FB02138E
:102EA000360C46EA9346A680218821F001010904E8
:102EB000090C21803B499209A1FB021292099B0C4B
:102EC0000133042A238438BF0422A2832388364A8C
:102ED0009BB243F001032380238823F4816323F012
:102EE00002031B041B0C4FF4804143F480632380D6
:102EF0002181238823F080031B041B0C238023885B
:102F00009BB202EB451243F0010323800121002311
:102F100082F8F85582F8F91582F8FA3505B0BDE85F
:102F2000F083224F85E7002E3FF467AF337240F6FF
:102F30000C23F3805CE71E4B1A6A42F400121A62FB
:102F40001A6A22F400121A6267E7042220463A2124
:102F500007F01CFF51E703F5F0331A6A42F48002D0
:102F60001A621A6A22F480021A6256E703F5EE33F7
:102F70001A6A42F400021A621A6A22F400021A6201
:102F80004BE700BF00000020005400400058004004
:102F9000005C0040009F2400804F120083DE1B4332
:102FA000D34D6210632D3E0518330020C027090061
:102FB000003802402DE9F047924E90F9001080460B
:102FC000807806EBC1050138CC0090B0D5F8341EEE
:102FD00014282DD8DFE810F04C0120011500550011
:102FE0005F009E00A600C301B6017A0084003C0287
:102FF0000402D701C000D0002F003700A3019501C3
:103000005401888A0C8B81B27F4841EA044188438D
:1030100000F02081D8E90201101A42F2107263EB2D
:103020000101904271F1000102D3152388F80230AA
:1030300010B0BDE8F08798F813000882C8E90223B1
:10304000122088F80200888A0C8B80B240EA044083
:103050006E4C844300F0B28000200E900F9001204F
:103060000F910E900E99002900F017820F991431DC
:103070000F910F9909684905CCD5142388F80230BF
:10308000D6E798F8110000F0FE000882C8E9022394
:10309000052088F80200888A0C8B80B240EA044040
:1030A0005B4C844300F0A18000200090019001203F
:1030B000019100900099002900F0FB8101991431E1
:1030C0000191019909684F05D7D4A3E798F8110039
:1030D00040F001000882C8E902230B2088F80200B2
:1030E000888A0C8B80B240EA04404A4C84436DD0FD
:1030F0000020049005900120059104900499002976
:1031000000F0D181059914310591059909684D05A3
:10311000B3D47FE798F813000882C8E90223072098
:1031200088F80200888A0C8B80B240EA0440374C51
:1031300084435ED00020029003900120039102900E
:103140000299002900F0C181039914310391039978
:1031500009684E0591D45DE7088820F4806000047A
:10316000000C088098F8110000F0FE000882C8E901
:103170000223102088F80200888A0C8B80B240EA73
:103180000440234C844312D000200C900D90012069
:103190000D910C900C99002900F091810D9914313A
:1031A0000D910D99096848053FF567AF32E798F82A
:1031B0001330FF2B06D198F810301BB1132388F879
:1031C000023035E7112388F8023031E7D8F81400CF
:1031D000012800F08F81022800F04382098B0E2124
:1031E000C8E9022388F8021022E7062388F8023093
:1031F0001EE7D8F81400002800F06D81082388F835
:10320000023015E7000000200100030084000700E1
:103210008200070002000300088820F40060000418
:10322000000C0880088880B240F48060088008881C
:1032300080B240F480700880032088F80200888AF9
:103240000C8B81B2A94841EA04418843C8E90223B2
:103250007FF4EEAE98F81230002B40F0CE8198F853
:103260001330FF2B00F03F82042388F80230DFE6A2
:10327000098889053FF5CEAE002388F80230D7E6ED
:10328000344494F8380E07F091FB064694F8390E52
:1032900007F08CFB964AB2F8583601339BB282464F
:1032A000A2F8583616B13368B2881A83BAF1000F03
:1032B00004D0DAF80030BAF804201A83112130461D
:1032C00005F056FC1121504605F052FC4FF009095B
:1032D00065272EB13368B28819690A4240F023810C
:1032E000013F00F01D810AF0D5FA04460D460AF0B0
:1032F000D1FA001B61EB0501052871F10001F6D33D
:10330000E7E7088880B240F4007008804FF6FF308D
:1033100088820121C8E9022388F8021088E6D8F8DB
:103320001400002800F06D81D8F8184014F8016BE3
:103330000E8201381225C8E90504C8E9022388F87D
:10334000025075E6888A0C8B81B2684841EA0441D4
:1033500088437FF45FAE0A2388F8023068E6088865
:1033600080B240F480700880092088F80200888AC2
:103370000C8B81B25D4841EA04418843C8E90223CD
:103380007FF456AEE7E7002401250A940B940B91D5
:103390000A950A98002800F047810B9814300B908A
:1033A0000B98006846077FF535AED8F8140003285F
:1033B00000F06D81022800F24381088820F48060CB
:1033C0000004000C0880088880B240F40070088077
:1033D000098A88F81C40C8E9022388F8025027E6C9
:1033E0000020012408900990099108940898002869
:1033F00000F0148109981430099009980068470773
:103400007FF508AEEFF31185102080F3128808884D
:1034100080B240F400700880D8F818000E8A471C6B
:10342000C8F81870EDB2067085F311880D8AD8F8C7
:1034300018106FF001004E1CC8F818600D70C8E934
:103440000223C8F8140088F81C4088F80240EFE511
:10345000002006900790012007910690069C002C02
:1034600000F0E880079C14340794079C24686406E5
:103470007FF5D0AD0C8AD8F818104D1CC8F818503C
:103480000C70D8F8141088F81C000139C8E9022320
:10349000C8F8141088F80200CAE50F9918310F9186
:1034A0000F990968B6E505991831059105990968DC
:1034B000B0E501991831019101990968AAE50D99C2
:1034C00018310D910D990968A4E5039918310391FC
:1034D000039909689EE5088880B240F4007008806E
:1034E0000121C8E9022388F80210A1E501000300C8
:1034F00018330020088820F480600004000C088045
:10350000EFF31184102080F31288088B088880B2B2
:1035100040F40070E4B2088084F311880C215FE667
:1035200016B13368B2885A830AF0B4F904460D46DE
:103530000AF0B0F9001B61EB0501052871F10001EB
:10354000F6D316B13368B2881A830AF0A3F9044699
:103550000D460AF09FF9001B61EB0501052871F18A
:103560000001F6D3B9F101097FF4B2AE16B13368A8
:10357000B2885A830AF08EF904460D460AF08AF999
:10358000001B61EB0501052871F10001F6D3BAF1CA
:10359000000F04D0DAF80030BAF804205A830AF099
:1035A00079F904460D460AF075F9001B61EB050137
:1035B000052871F10001F6D316B13368B2881A8379
:1035C0000AF068F904460D460AF064F9001B61EB45
:1035D0000501052871F10001F6D3BAF1000F04D0FE
:1035E000DAF80030BAF804201A8398F90000441C75
:1035F0003FF442AEFFF7D0FB3EE60F2388F80230DF
:1036000016E5088880B240F4007008800121C8E9FE
:10361000022388F81C1088F8021009E5099918316E
:10362000099109990968F5E40B9918310B910B99E7
:103630000968EFE407991831079107990968E9E4E7
:10364000D8F81800098A441CC8F818400170D8F846
:103650001410C8F808200139C8F81410C8F80C3044
:10366000E6E4088880B240F400600880EFF311843B
:10367000102080F31288088B088820F480600004F2
:10368000000CE4B2088084F311880D21A8E50888B5
:1036900020F480600004000C0880EFF311841020F7
:1036A00080F31288D8F818000D8A461CC8F81860F4
:1036B0000570088880B240F40070E4B2088084F39A
:1036C0001188D8F81800098A441CC8F818400170FD
:1036D000D8F814100C200239C8E90223C8F81410D5
:1036E00088F80200A4E498F81030002B3FF4BCAD39
:1036F00031E600BF38B5184D9DF814E005EB4014D5
:103700004FEA401C94F8F90500B938BD490084F827
:103710000B26C4F80C3684F809160023049984F8A3
:1037200008E6022205F5BF6584F80A36C4F81016CB
:1037300084F8143684F8FA2565440AF0ABF802469A
:103740000B462846FFF736FC94F8FA35002BF4D1E7
:1037500094F8140638BD00BF18330020F0B50446B5
:1037600083B00D461746061D20680379012B1AD039
:10377000022B02D0002003B0F0BD8368DB07324685
:103780004FF0FF015CBF3246FF2106F0CBF9002865
:10379000F0D015B12379DB07E6D4002FEBD02379E5
:1037A0003B7003B0F0BD8268417C90F9100002F0DC
:1037B0000102CDE90062FF22FFF79CFFE7E700BFAF
:1037C00030B50446051D20680379012B83B017D05E
:1037D000022B02D0002003B030BD8368DB072A46ED
:1037E0004FF0FF015CBF2A46FF2106F09BF900283D
:1037F000F0D02379DB07EED520680379012BE7D1E0
:103800008268417C90F9100002F00102CDE900527B
:10381000FF22FFF76FFFEAE730B50246044652F891
:10382000040B0379012B83B00ED0022B01D00020B2
:1038300008E0FF2106F076F90028F8D02079C0438F
:1038400000F0010003B030BD8568417C90F91000A4
:10385000009205F001050195FF22FFF74BFFEBE712
:1038600030B5B42283B00446FF21006805F072FA37
:1038700010B9002003B030BD20680379012B04F19A
:10388000040514D0022BF4D18368DB072A464FF0DD
:10389000FF015CBF2A46FF2106F044F90028E8D06A
:1038A0002379DB07E6D520680379012BEAD182680A
:1038B000417C90F9100002F00102CDE90052FF2294
:1038C000FFF718FFEAE700BF30B50A4683B00446A9
:1038D000A521006805F03EFA10B9002003B030BD04
:1038E00020680379012B04F1040514D0022BF4D1D4
:1038F0008368DB072A464FF0FF015CBF2A46FF21A1
:1039000006F010F90028E8D02379DB07E6D5206817
:103910000379012BEAD18268417C90F9100002F012
:103920000102CDE90052FF22FFF7E4FEEAE700BF03
:1039300070B582B0CDE900230446FFF791FF10B9BE
:10394000002002B070BD20685522A52105F002FAC2
:103950000028F5D0251D20682A46FF2106F034F9FD
:103960000028EDD02379DB07F5D40DF1FF350DF1FB
:10397000070615F8011F2046FFF7A6FF0028DFD035
:10398000B542F6D1DDE700BF002A35D0F0B50446D8
:1039900083B00E468F18051D16F8012B2068A5214F
:1039A00005F0D8F990B9002003B0F0BD8268417CE1
:1039B00090F9100002F00102CDE90052FF22FFF75A
:1039C00099FE0028EFD02379DB0710D52068037912
:1039D000012BEBD0022BE6D18368DB072A464FF0A0
:1039E000FF015CBF2A46FF2106F09CF8E9E7B742D9
:1039F000D2D1012003B0F0BD0120704770B59622EE
:103A000082B004460E460068FF2105F0A3F910B904
:103A1000002002B070BD251D20680379012B1FD046
:103A2000022BF5D18368DB072A464FF0FF015CBF0C
:103A30002A46FF2106F076F80028E9D02379DB0733
:103A4000EAD4E1222068114605F084F90028DFD08D
:103A500020683246FF2102B0BDE8704006F0B4B8DD
:103A60008268417C90F9100002F00102CDE9005219
:103A7000FF22FFF73FFEDFE7002A43D0F0B5044600
:103A800083B00E468F18051D20689622FF2105F091
:103A900061F990B9002003B0F0BD8268417C90F9D3
:103AA000100002F00102CDE90052FF22FFF722FED2
:103AB0000028EFD02379DB0710D520680379012B8C
:103AC000EBD0022BE6D18368DB072A464FF0FF01DB
:103AD0005CBF2A46FF2106F025F8E9E7E1222068CD
:103AE000114605F037F90028D4D020683246FF216E
:103AF00006F06AF80028CDD00136B742C4D10120C3
:103B000003B0F0BD0120704770B505460B46044672
:103B1000164655F8040B82B087211A4605F01AF9AB
:103B200020680379012B1AD0022B02D0002002B0AA
:103B300070BD8368DB072A464FF0FF015CBF2A4651
:103B4000FF2105F0EFFF0028F0D02379DA07E7D452
:103B5000002EECD0C3F34013337002B070BD826806
:103B6000417C90F9100002F00102CDE90052FF22E1
:103B7000FFF7C0FDE7E700BF70B5782182B00446CB
:103B800016460068002205F0E5F810B9002002B0E2
:103B900070BD251D20680379012B14D0022BF5D1AF
:103BA0008368DB072A464FF0FF015CBF2A46FF21EE
:103BB00005F0B8FF0028E9D02379DA07EAD45B09D9
:103BC000337002B070BD8268417C90F9100002F041
:103BD0000102CDE90052FF22FFF78CFDEAE700BFAA
:103BE00030B5CC2283B00446A521006805F0B2F8B8
:103BF00010B9002003B030BD20680379012B04F117
:103C0000040514D0022BF4D18368DB072A464FF059
:103C1000FF015CBF2A46FF2105F084FF0028E8D0A1
:103C20002379DB07E6D520680379012BEAD1826886
:103C3000417C90F9100002F00102CDE90052FF2210
:103C4000FFF758FDEAE700BF30B5B42283B0044661
:103C5000FF21006805F07EF810B9002003B030BDE8
:103C6000251D20680379012B22D0022BF5D1836812
:103C7000DB072A464FF0FF015CBF2A46FF2105F013
:103C800051FF0028E9D02379DA07EAD4CC21204675
:103C9000FFF71AFE0028E0D002E02379DB07DDD52C
:103CA00020682A46FF2105F08FFF0028F5D1D4E7D0
:103CB0008268417C90F9100002F00102CDE90052C7
:103CC000FF22FFF717FDDCE72DE9F04F8BB0CDE9C0
:103CD00007230446002004908A460390251D049B78
:103CE000079A2046DE0002EBC30BFFF7B9FD20B9AF
:103CF00035E0237913F0010207D020682A46FF211E
:103D000005F062FF0028F4D129E005929A07099096
:103D100040F1D880F0212046FFF7D6FDF8B1079B8F
:103D2000DDF81480083E3344012606933746BAF185
:103D3000000F54D0082F52D807F1FF394AFA09F979
:103D400009F0010920684FEAC912782105F002F84C
:103D500028B120680379012B50D0022B06D0002017
:103D6000089B049A1A700BB0BDE8F08F8368DB07DC
:103D70002A464FF0FF015CBF2A46FF2105F0D2FE24
:103D80000028ECD0237913F00102E2D1C3F3801CA8
:103D9000D9099B0646D5BCF1000F60D1BAF1000FDE
:103DA0005AD0082F58D8894540F08880B9F1000FC3
:103DB00048D01BF8083033430BF808307600013741
:103DC00016F0FF06FFB2B2D108F101085FFA88F8D9
:103DD000B8F1080F43D00126BAF1000FAAD1049B15
:103DE000C3B1039BBB4215D9069B13F808301E4292
:103DF00014BF4FF001094FF00009A3E78268417C2E
:103E000090F9100002F00102CDE90052FF22FFF705
:103E100071FCB5E7039BA3EB0709B9FA89F94FEAEF
:103E200059198FE7BAF1000F13D0082F11D889451F
:103E300096D1B9F1000FBCD1059BBCF1000F08BFB2
:103E40003B4605931BF8083023EA06030BF80830BD
:103E5000B4E70029ADD1EFE70029AAD1F2E7402F5E
:103E600006D8089B049A1B7893423FF638AF77E751
:103E70009BF807700BF1FF360BF1060B16F801CF1C
:103E8000082182EA0C0343F30003013923F0730392
:103E900083EA520211F0FF01D2B24FEA5C0CF0D17A
:103EA000B345EBD19742DCD1049B0133DBB20493E1
:103EB000059B002B3FF454AF0393D2E7DDF8248039
:103EC00040464DE7804640464AE700BF10B50068CF
:103ED0000379012B84B00C461AD0022B02D00020AB
:103EE00004B010BD836813F0010F03AA4FF0030361
:103EF00014BF2221A22105F0EDF80028EFD0BDF972
:103F00000D3003EB83031B12E633238004B010BD96
:103F10008368417C90F9100003F00103019303AB27
:103F2000009322220323FFF7E5FBE6E738B5184D9F
:103F30009DF814E005EB40144FEA401C94F8F90595
:103F400000B938BD84F80B26C4F80C3601220023D2
:103F5000490005F5BF6584F80A2684F81436049AEA
:103F600084F808E6022384F80916C4F8102684F8B9
:103F7000FA35654409F08EFC02460B462846FFF7E9
:103F800019F894F8FA35002BF4D194F8140638BDDA
:103F90001833002000680379012B0BD0022B01D0CD
:103FA000002070478368DB074FF0F00219D5FF212E
:103FB00004F07ABE00B5826890F910C0417C85B0EB
:103FC00002F0010201920DF10F0200926046FF2201
:103FD0004FF0F00C8DF80FC0FFF7A8FF05B05DF8AB
:103FE00004FB7F2104F060BE70B505682B79012BBE
:103FF00084B004460E4617D0022B02D0002004B035
:1040000070BDAB68E122DB074CBF11466121284639
:1040100004F04AFE0028F1D020683246FF2104B0A7
:10402000BDE8704005F0D0BDAA68697C95F9100024
:1040300002F001020DF10F0501920095E1228DF8C9
:104040000F20FFF773FFE5E770B505682B79012BAB
:1040500084B004460E4618D0022B02D0002004B0D3
:1040600070BDAB68DB074FF0C3024CBFE12161219B
:10407000284604F019FE0028F0D020683246FF21BF
:1040800004B0BDE8704005F09FBDAA6895F9100026
:10409000697C02F0010201920DF10F020092C3222D
:1040A0008DF80F20E122FFF741FFE4E70068037974
:1040B000CA4341EA0211012BCAB209D0022B01D036
:1040C000002070478368DB0717D5D22104F0ECBDD0
:1040D00000B585B090F910C08DF80F208268417C42
:1040E00002F001020DF10F00CDE90002D22260467C
:1040F000FFF71CFF05B05DF804FB522104F0D4BDAE
:1041000070B505682B79012B84B004460E461CD08F
:10411000022B02D0002004B070BDAB68DB074FF06B
:10412000F0024CBFE1216121284604F0BDFD0028CA
:10413000F0D02246FF2152F8040B05F045FD00287F
:10414000E8D02379337004B070BDAA6895F91000E7
:10415000697C02F0010201920DF10F020092F0223F
:104160008DF80F20E122FFF7E1FEE0E70068037918
:10417000012B0BD0022B01D0002070478368DB0796
:104180004FF0B40219D5FF2104F08EBD00B582684E
:1041900090F910C0417C85B002F0010201920DF14E
:1041A0000F0200926046FF224FF0B40C8DF80FC052
:1041B000FFF7BCFE05B05DF804FB7F2104F074BD81
:1041C00000680379012B0AD0022B01D00020704730
:1041D0008368DB070A4617D5A52104F065BD00B545
:1041E000826890F910C085B002F001028DF80F10BE
:1041F000417C0DF10F00CDE90002A5226046FFF7DA
:1042000095FE05B05DF804FB252104F04DBD00BF0F
:1042100000680379012B0BD0022B01D000207047DE
:104220008368DB074FF0960219D5FF2104F03CBDEF
:1042300000B5826890F910C0417C85B002F001029F
:1042400001920DF10F0200926046FF224FF0960C92
:104250008DF80FC0FFF76AFE05B05DF804FB7F2103
:1042600004F022BD00680379012B0AD0022B01D093
:10427000002070478368DB070A4617D5872104F0C2
:1042800013BD00B5826890F910C085B002F001023C
:104290008DF80F10417C0DF10F00CDE9000287224F
:1042A0006046FFF743FE05B05DF804FB072104F00C
:1042B000FBBC00BF00680379C901012BCAB206D05C
:1042C000022B01D000207047782104F0EDBC00B52E
:1042D00085B090F910C08DF80F208268417C02F003
:1042E00001020DF10F00CDE9000278226046FFF7D0
:1042F0001DFE05B05DF804FB00680379012B0BD0AF
:10430000022B01D0002070478368DB074FF0550275
:1043100019D5A52104F0C8BC00B5826890F910C079
:10432000417C85B002F0010201920DF10F02009272
:104330006046A5224FF0550C8DF80FC0FFF7F6FD33
:1043400005B05DF804FB252104F0AEBCF0B589B0E2
:104350000023904A02930393136843F4803313605D
:1043600003E0029BB3F5A04F09D0136803F40033B8
:104370000393029B01330293039B002BF1D0854BE7
:104380001B6813F4003318BF01230393039B012B15
:1043900001D000BFFDE77F4B7F491A6C7F4842F098
:1043A00080521A640A6842F440420A609A689A602D
:1043B0009A6842F400429A609A6842F4A0529A6065
:1043C00058601A6842F080721A601A689001FCD531
:1043D000734A40F205711160996821F003019960F8
:1043E000996841F00201A2F580629960936803F038
:1043F0000C03082BFAD1936803F00C03042B00F094
:10440000C680082B00F0AB80664A624B664998680C
:10441000664D674E674FC0F303100144002491F8C6
:104420006C10CA406449E9606449586FA960596BCF
:10443000C6F8302C21F080015963596F604A6148F9
:1044400041F080715967196B0A431A635A6B5A63BA
:104450009A6B9A631A6C5C490A431A64596C5B4AFA
:104460000A435A6448F2FF7123462246CDE90044CC
:1044700072F08AFF5648234622464FF6FF71CDE977
:10448000004472F081FF5348234622464FF6FF71E5
:10449000CDE9004472F078FF4F48234622464FF69C
:1044A000FF71CDE9004472F06FFF4C48234622466D
:1044B0004FF6FF71CDE9004472F066FF484823468D
:1044C00022464FF6FF71CDE9004472F05DFF45488A
:1044D000234622464FF6FF71CDE9004472F054FFA7
:1044E0004148234622464FF6FF71CDE9004472F061
:1044F0004BFF234622464FF6FF713C48CDE900446E
:1045000072F042FF04A8FEF7FBFAD5F8FC200499EC
:10451000D6F8303C364842F08072C5F8FC20354A67
:10452000C2F8B00F5460106840F0010010604FF402
:104530007A72B3FBF2F3013BB3F1807F2E4AB1FBF9
:10454000F2F2C7F85C2608D24FF0E022F021536166
:10455000072385F823109461136109B0F0BD5168F9
:10456000536852684902C2F388124CBF23490D496F
:1045700003F03F03B1FBF3F303FB02F2054B5B686F
:10458000C3F3014301335B00B2FBF3F23DE71B4A87
:104590003BE700BF0038024000700040085440076D
:1045A000003C02400024F400BC24080800ED00E0B8
:1045B00000000020183300200003FA050000000866
:1045C000FF91670000000240FFC9FE10335707004B
:1045D0000004024000080240000C024000100240AB
:1045E0000014024000180240001C0240002002405B
:1045F00055CEACC5001000E040420F0000127A001A
:1046000082B0064B002201920193019B03EB8003D1
:104610000193019B196002B0704700BF5028004011
:1046200010B51C2006F0C2F91121044604F0A0FACE
:104630004CB12368A2885A83C82009F059F923682D
:10464000A2881A8310BDBDE81040C82009F050B9F7
:10465000704700BF704700BF704700BF10B5104CD7
:1046600094F86A3623B90F4B4FF480225A6110BD7B
:104670004FF0E022D2F8103D23F00603C2F8103DBF
:10468000FDF75CFFD4F870369B68DB07EBD5D4F8F8
:104690006C27136823F0030161F307031360E2E75B
:1046A00018330020003C01402DE9F04FA34CD4F812
:1046B0006C365A69D5078BB002D50BB0BDE8F08FC8
:1046C0005A699B6912EA0301F7D0C1F30743080353
:1046D000019300F1E180019B5D073FD48807CEB2D2
:1046E00003D5D4F86C3602225A610029C0F24A82FE
:1046F0000A05C1F3072500F19981370708D5904BCA
:104700009048D3F8583E9847D4F86C3608225A613E
:10471000F60600F10F82E80600F1BE81A80600F15E
:104720001781019BDA0609D5854B8648D3F8683E88
:104730009847D4F86C364FF480125A61019B9B065F
:10474000BBD57F4B7F48D3F86C3E9847D4F86C3686
:104750004FF400125A610BB0BDE8F08FD4F87036F8
:104760009E69DB691E40B6B2002EB7D0754D4FF082
:10477000000B05F118080F46F00740F18280D4F8CD
:104780007016D8F8002008694B6B23FA0BF3DB0195
:10479000DBB203439068034013F00109D8B200F084
:1047A0000F824B6B012000FA0BF023EA00034B63EE
:1047B00001239360624B6348D3F8503E5FFA8BF15C
:1047C000984794F86336012B00F07E8219F0800F31
:1047D00057D0D5E94CC1D5F82431D8F800E0ACEB7E
:1047E00001029342DEF8180028BF134680B203335B
:1047F000B0EB930F45D9D4F8703694F86396CDE9B1
:10480000026BBA4667469C46B94237D2D5F8243186
:10481000781A984228BF184600F1030BD5F82831C2
:104820004FEA9B0BB9F1000F10D182B20332921004
:10483000D8F8B8600AD04946013153F8047B376094
:104840008A42F9D1D5E94C71D5F8283101440344A5
:104850008F42C5F82831C5F83411DEF818300AD176
:1048600095F81C01012202FA00F0DCF8342022EA5B
:104870000002CCF834209BB29B45C5D3DDE9026B26
:10488000574676080BF1010B05F1280508F10408DD
:104890007FF472AF394621E7D4F870369D69DB6941
:1048A0001D402D0C3FF417AF04F5CC68DFF890B035
:1048B000029104F2B46600274FF00109C24608E0F5
:1048C0006D0807F1010706F1040608F1280800F059
:1048D0009181EA07F4D53068D4F870168368496985
:1048E0000B40D9B2DB0740F1708194F86336C0F811
:1048F0000890012B07D10169D8F87C33C1F312016C
:104900005B1AC8F88C33DBF84C3EF9B25046984736
:1049100094F86336012BD3D1002FD1D194F871379D
:10492000052BCDD1D4F8B43607491961074959612F
:1049300019684FF080211960C2E700BF18330020CA
:10494000000000207839002018000860443F002053
:10495000D4F87056D4F87826AB68C3F34103022B21
:10496000136814BF0021032161F30A0313606B680D
:1049700043F4807306A86B60FEF7C2F8D4F86C2687
:10498000079ED36823F47053D360A86810F0060F15
:10499000C0F3410100F03C819F49A048314481426D
:1049A00040F2AE819E48A6F57401A1F510518142F6
:1049B00040F2AA819B499C4831448142C0F0A881C1
:1049C0009A48A6F18C71A1F54341814240F2A4813D
:1049D0009749984831448142C0F0A281964997484E
:1049E00031448142C0F0A0819548A6F1B771A1F58C
:1049F00058518142C0F0A08192499348314481428C
:104A0000C0F09681914892493044884234BF0620D4
:104A100005204025012160F38D23D3604FF400531E
:104A200084F86216A4F8645653617AE600238DF880
:104A3000133094F872378DF81330864B8648D3F8CC
:104A4000603E9847D4F87036D4F86C26986894F88D
:104A50006A364FF400615161002B3FF44EAEC3073C
:104A60007FF54BAE94F87537012B7FF446AE9DF879
:104A70001330032B7FF441AED4F86C3777491A68B2
:104A800042F001021A601A6842F003021A600B69D0
:104A900043F006030B6130E6D4F87066D4F86C1668
:104AA0007368002723F0010373600597059B43F0AB
:104AB00020030593059B67F38A130593059B0B6100
:104AC000674BBC460A690592013B02D0059A9206E3
:104AD000F8D494F8612652B1624B03EB820EFF22A8
:104AE00053F8040F8260D86B73458260F8D10B23B2
:104AF00063F3070763F3070C4FF0FF33B3614FF025
:104B00000113F3617761C6F810C03368564823F487
:104B1000FE63336094F86326D4F8B436012A186132
:104B20006FD04FF480534B614A4B4B48D3F85C3EF7
:104B30009847F3E5D4F86C369A6922F010029A612E
:104B40001A6AC2F34340022802F00F0100F090807D
:104B5000062812D101EB810104EBC101D4F83067C2
:104B6000D1F8EC09C2F30A1210443268C4F82C2CB4
:104B70003268C4F8302CC1F8EC099A6942F010028E
:104B80009A61C8E594F86A363BB1D4F86C2713688B
:104B900023F0030060F307031360D4F870262D4B55
:104BA0002D48D3F8645E5368029123F001035360EB
:104BB000A847D4F86C3602994FF000425A6197E545
:104BC000010707D5082393605BE68A0707D5022310
:104BD000836075E6C3060FD51023936051E60B077B
:104BE0007FF56EAEDBF8543E504698473368082197
:104BF000996065E602996EE5410679D54023936098
:104C00003FE61A4A5A611A684FF080221A6088E714
:104C10004FF400750920FEE6401E1BFF3F420F00C7
:104C2000DFC810002013FBFE20D61300FF69180018
:104C300000D3CEFE40771B00C05BB3FEC0912100C5
:104C400040AC2700C01D6AFE40E13300803C36FEC8
:104C5000E09C4100000000207839002000ED00E0D9
:104C6000410D03008C39002018000860443F0020EB
:104C700047F6F070104280D0C2F30A1201EB8100B7
:104C800004EBC00002F1030C5FEAAC0CD0F8E06961
:104C9000D4F830E74FEA810818BF002006D0013071
:104CA000DEF8007046F8047B8445F8D1414404EBFB
:104CB000C101D1F8E0091044C1F8E009D1F8EC09CC
:104CC0001044C1F8EC0958E7BBF1000F7FF47EAD4A
:104CD00094F87137042B7FF479ADD4F8B436184AC0
:104CE0001A61184A5A611A684FF080221A606DE5FD
:104CF000830758BF81467FF569AD02239360C0E505
:104D0000012140250E2086E6012140250D2082E666
:104D1000012140250C207EE6012140250B207AE66A
:104D2000012140250A2076E601214025092072E66E
:104D30000121402507206EE60121402508206AE672
:104D400018000860443F002070B5194D194BC5F894
:104D5000543C194B85F8601C002683F8276905F63A
:104D60005443C0E954330D23C0F8583140F20113C5
:104D70000446C0F85C6100F5A271A0F8443171F0FE
:104D800067FF1F23C4E9EC36E378012205F284555E
:104D90009342C4F8A853A4F89C2308BFC4F8AC53AA
:104DA00004F567712046BDE8704071F051BF00BF47
:104DB000183300205553425320220020F0B50B78C1
:104DC00013F0600283B004462BD0202A30D14A78F9
:104DD000FE2A39D0FF2A2DD14A88002A3BD1CA8821
:104DE000002A38D11F0636D46148624B80F8272943
:104DF000C4F8B423E278012183F8A415A4F89C1325
:104E000003F284531F21012AC4F8B013C4F8A83355
:104E100004F5677108BFC4F8AC33204671F018FF81
:104E200006E04B780A2B1AD00B2B08D0012B2AD086
:104E3000002002E071F09EFD022003B0F0BD4D4B5A
:104E40004A8883F8652CF3E74F8827B9CD88012D70
:104E500001D11B0642D4204671F08CFDECE7022103
:104E600080F811114FF48071A0F81C114249012300
:104E7000C0E94A11C0E94E33C0E94C3200F58E71E9
:104E800071F084FED4E78B88C0681E06DDB244D47E
:104E90000192019A394B42F010020192019A02618B
:104EA00002690192013B02D0019AD206F8D4314E38
:104EB0002946204671F0D0FD294696F8A4550223D4
:104EC0004022204671F0F8FD022DB1D1812120460B
:104ED00071F088FD002386F8A435A9E7254ED6F8A1
:104EE000BC359B699847C0B286F8640C0028B2D0E4
:104EF000022306F6644684F811314FF48073C4E946
:104F00004E55C4E94A66C4E94C57A4F81C3104F56F
:104F10008E71204671F03AFE8AE70092009A174B94
:104F200042F020020092009A65F38A120092009AE1
:104F3000026102690092013B02D0009A9106F8D406
:104F40000C4E2946204671F087FD294696F8A45557
:104F500002234022204671F0AFFD022DB6D0012D74
:104F60003FF466AF01212046FFF7EEFE60E700BF89
:104F700020220020183300207D3F0020410D030037
:104F800010B50D4B93F82739022B07D0033B012BAB
:104F900002D80021FFF7D8FE002010BD074B93F880
:104FA0009115044671F008FF0028F5DA012120462A
:104FB000FFF7CAFEF0E700BF2022002018330020D0
:104FC000F8B53F4C94F8276905467EB1012E01D013
:104FD0000020F8BD3B4B93F8911571F0EDFE0028D1
:104FE000F6DA31462846FFF7AFFEF1E7354FB0F865
:104FF000B433D7F88C25C7F85C2C1F2BD7F888253D
:10500000C7F8582C08D1304BD7F884259A4203D1E1
:1050100097F89115012919D997F8663C5A1CD2B214
:1050200007EBC303042A18BF1646052283F8682C31
:105030004FF400522846C3F86C2C022387F8666CA4
:1050400087F8A435FCF720FA0020F8BD97F89235D0
:10505000013B0F2BE0D871F0AFFE002827DB94F85E
:105060002739013B022BB3D9B7F8883C1BB3042284
:1050700084F82729154AC5F85C61C5E95422D7F898
:105080008C2587F8606C934228BF1346D7F85C2CB8
:10509000C5F8583140F20111A5F84411D21A05F5AE
:1050A000A2712846C7F85C2C71F0D2FD90E7284623
:1050B000FCF7EAF98CE719462846FFF745FE87E733
:1050C000202200201833002055534243306E002028
:1050D00010B54FEA511E024400EB8E0C624529D9EF
:1050E00001F01F034FF0FF3450F82E1004FA03F3C1
:1050F0000B4093FAA3F3B3FA83F3DBB2202B16D160
:105100000CF104018A4202D817E08A4212D98C4677
:105110000431DCF8003093FAA3F3B3FA83F3DBB283
:10512000202BF2D0ACEB000C03EBCC0010BD03EB5A
:105130004E1010BD4FF0FF3010BD204610BD00BF17
:105140000369416890ED067AF0B4C56A3B4E876802
:1051500053EA010204BFD6F8381541606A1C30EEEC
:10516000077A0133012A80ED067A0361C26241D0D9
:1051700090ED075AD0ED096AD6F8384507EE902A27
:1051800070EE455AB8EEE76A611AC5EE867AB94202
:1051900077EE857A30EE670AC0ED087AE5EE806A30
:1051A000C0ED077AC0ED0A6AC0ED096A01D8F0BC0B
:1051B0007047012A2ADD07EE905AF8EEE77A86EE6C
:1051C000A76AB5EEC06AF1EE10FA1FDBF1EEC67AFF
:1051D000F4EE677AF1EE10FA18D6D0ED056AF4EE27
:1051E000E76AF1EE10FA14D5037BF3B10323F0BCA8
:1051F00003707047D6F8382580ED080A521ABA4273
:105200004FF0000180ED070A4162D0D9DFED0C7A42
:10521000E3E707EE903AF8EE677A0223C7EE276AD3
:10522000F0BC0370C0ED066A7047D6F838154160CF
:10523000002203618261C362B9E700BF1833002016
:1052400000000000DFED504A10B5844600F1480E22
:105250000346B1EC017AD3ED067ADA6A77EE877A03
:105260000132012AC3ED067ADA6255D093ED075A6E
:1052700093ED096A07EE902A77EE455AF8EEE77A41
:10528000C5EEA76A76EE857AF0EE466A37EE677A63
:10529000C3ED087AE5EE876AC3ED0A6AC3ED077AC3
:1052A000C3ED096A18337345D3D1384C4168D4F83B
:1052B00038250369521A816801338A4203612AD969
:1052C00090ED056A00F1300EDCF82C20DCED0A6A66
:1052D000012A02F1FF3126DD07EE901AF8EEE77A97
:1052E00086EEA77AB5EEC07AF1EE10FA1BDBF1EE8E
:1052F000C77AF4EE677AF1EE10FA14D6E645B4EE0A
:10530000E76A0CF1180C16D0F1EE10FADCD5037B2D
:105310006BB30323037010BDF0EE477AF0EE646ABE
:1053200083ED087ABAE7DFED187AE645B4EEE76A6E
:105330000CF1180CE8D1F1EE10FAE8D407EE903A2F
:10534000D0ED066A90ED0C7AD0ED125AF8EE677A3D
:10535000022386EEA76A0370C7EE276A85EEA77A56
:1053600080ED066AC0ED0C6A80ED127A10BD002255
:10537000D4F83815416003618261C36202634364FB
:105380008264C36510BD00BF000000001833002018
:10539000B0EEC06AF0EEE05AF4EEC65AF1EE10FA42
:1053A000F0EE407A0EDCB5EE400AF1EE10FA4BD08A
:1053B000F4EEC65AF1EE10FAF0EE466A50D5B0EEB1
:1053C000655A03E0F0EE656AB0EE465A85EE267A3D
:1053D0009FED252A9FED253A9FED254ADFED254AD1
:1053E000DFED252ADFED253ADFED256AA7EE023A4B
:1053F000E7EE223AA7EE034AB7EE005AE7EE044A78
:10540000A7EE235AE7EE246AF4EEC65AB1EE667AA6
:1054100087EE050AF1EE10FA48BF9FED1A7AF5EE15
:10542000C00A48BF37EE400AF1EE10FA48BF9FEDC0
:10543000167AF5EEC07A48BF37EE400AF1EE10FA60
:1054400048BFB1EE400A7047DFED107A9FED100AB9
:10545000F5EEC00AF1EE10FA58BFB0EE670A7047D9
:10546000B0EE465AB2E700BF39094E3DE3B59EBEE5
:1054700088FA16BE45FE7FBF99FB243F69A2163EFF
:10548000A7DFA8B4DB0FC93FDB0F4940A7DFA83473
:10549000DA0F494091ED007AD0ED047A90ED054A9B
:1054A000D0ED064A90ED075AD0ED085A90ED096A02
:1054B000D0ED0A6AE7EE077AF7EE003AC0ED047A1B
:1054C00091ED007AD1ED017AA7EE274A90ED0B7AA3
:1054D00080ED054A91ED024A91ED003AD0ED0C7A4B
:1054E000E3EE044AC0ED064AD1ED004A35EE245AF7
:1054F00080ED075AD1ED014A91ED005AE4EE855A4C
:10550000C0ED085AD1ED015AA5EEA56A80ED096AF1
:10551000D1ED015A91ED026AE5EE866AC0ED0A6AA4
:10552000D1ED016A37EE267A80ED0B7AD1ED026A71
:1055300091ED007AE6EE877AC0ED0C7A91ED026A81
:10554000D1ED016AD0ED0D7A90ED0E7A90ED0F4A13
:10555000D0ED104A90ED115AD0ED135AE6EE267AAE
:1055600075EEA35AC0ED0D7AD1ED026AD0ED127A34
:1055700090ED006AA6EEA67AD0ED016A80ED0E7A73
:1055800091ED027A34EE074A90ED027A80ED0F4AEF
:1055900091ED004A74EE844AC0ED104AD1ED014A03
:1055A00035EE245A80ED115A91ED025AC0ED135A8E
:1055B00077EE857AC0ED127AD1ED017AD1ED005AFD
:1055C00091ED025A67EEA77AE5EEA57AE5EE057A47
:1055D000A5EEA76A80ED006A91ED016AE6EE276A02
:1055E000C0ED016AD1ED026AA6EEA77A80ED027ADB
:1055F00090ED037A77EE277AC0ED037A704700BF0B
:105600002DE9F04F4FF0000989B0864600F11005F2
:105610000646034600F13008074648462C46CDF8BA
:105620000CE08B469C46B24600283CD10CF1040CA1
:10563000A445FBD1032800F1010151D09C46AA46A4
:10564000029398B1DCED047A0192AAEB0903B64605
:105650007246F3EC016A92ED007AE6EEC77A5345A2
:105660000EF1100ECCED047AF2D1019ADCED046A51
:1056700015ED047AC6EE877A0CF1100CC4450AF1D8
:10568000100ACCED007ADCD1029B043614330846B4
:1056900008F1040814351034103709F104099C4648
:1056A000B2460028C2D0DCED007A0192D6463946D7
:1056B0007246F1EC016A92ED007AE6EEC77A994201
:1056C0000EF1100ECCED007AF2D10CF1040CA445D1
:1056D000019A0AF1040AE6D1032800F10101ADD1D3
:1056E000DDF80CE0002359460493059306930793D5
:1056F0007646774604AD0020F2EC017AE5EC017ABB
:10570000B0B104AC3B46B4EC017AF3EC016AE6EECE
:10571000C77AB34245ED017AF5D1013004280BD0A8
:10572000F2EC017A10371436E5EC017A0028E8D162
:10573000103714360120DFE708AD75ED017A10311E
:105740000EF1400E04287446A1F1040241ED017AE5
:105750001ED07346F3EC016AB1EC017AE6EEC77A2B
:10576000A342C2ED007AF5D15EED016A87EEA67A1A
:10577000013882ED007A17D0AEF1140E103C1146BC
:1057800075ED017A0428A1F1040241ED017AE0D11E
:105790005EED016A87EEA67A103CAEF1140E03208E
:1057A00001ED017A1146EBE709B0BDE8F08F00BFCB
:1057B000DFED297AB4EEE70AF1EE10FA28DD9FED6D
:1057C000277A30EE470AB4EEE70AF1EE10FAF8DC79
:1057D000DFED237AB4EEE70AF1EE10FA2FDD30EEBA
:1057E000670A37EEC00A60EE007A9FED1E7A9FEDE1
:1057F0001E6ADFED1E6AA7EE876A9FED1D7AE7EE4F
:10580000866A60EE275AA7EEA67AA5EE870A704749
:10581000DFED187AB4EEE70AF1EE10FAD8D59FED75
:105820000F7A30EE070AB4EEE70AF1EE10FAF8D478
:10583000DFED0B7AB4EEE70AF1EE10FACFDC9FED64
:105840000E7AB4EEC70AF1EE10FA44BF30EE270A22
:1058500037EE400AC7E700BFDB0F4940DB0FC94006
:10586000DB0FC93F9A7C2E36FAAF4FB93587083C1B
:10587000A4AA2ABEDB0F49C0DB0FC9BF10B5404C3C
:10588000B4FBF2F4A14219D3DFED3E7AF7EE005AF1
:10589000B0EE677AB0EE676AF0EE676A0023C0ED9B
:1058A000005AC0ED017A80ED027A80ED036AC0ED06
:1058B000046A836143610362C36110BD07EE902AED
:1058C000B8EE677ADFED307A27EE277AB7EE006A16
:1058D000C6EE076A07EE901A9FED2C7AF8EE677A0B
:1058E000B0EE405A67EE877AC7EEA64AFDEEE47A3C
:1058F00017EE902A2032402A3FD8B0EE640AFFF714
:1059000057FFB0EE404ADFED227A34EEA70AFDEEF3
:10591000C07A17EE902A2032402A29D8FFF748FF94
:10592000F8EE006A60EE266A012B1CD0B7EE006A22
:1059300036EE406AF6EE004A66EE244A35EE055A27
:10594000F7EE007A84EE057A77EE275A37EEC75ADB
:1059500084EEA57AC6EE257A86EEA56AC5EE256A9E
:10596000F0EE475A9AE7B0EE666AF7EE004AE5E7CE
:10597000DFED086A9FED030AD6E79FED024AC2E712
:1059800020A1070000000000BD378635DB0FC940AD
:10599000DB0FC93F00000080DFED077A30EE270AF9
:1059A000FDEEC07A17EE903A2033402B00D8FFE688
:1059B0009FED020A704700BFDB0FC93F00000000E7
:1059C0002DE9F84FDDF82CB09DF828408946002CD1
:1059D0001BF8011B0CBF4FF020084FF030081C1EB5
:1059E0000546174608463ADB00295CD0002C55D006
:1059F0004FF0000A5B4600E064B313F8016B013C12
:105A0000002EF9D1BAF1000F2FD1264644B14D45F1
:105A10004146284600D2B847013CF8D10B9B187884
:105A20000146A0B14FF0FF344FF0000A00E09B4662
:105A30004D45284600D2B8475B4613F8011B0029A4
:105A4000F5D10B9BF61A5E44BAF1000F10D1304627
:105A5000BDE8F88FBAF1000F1BD15646E0E763426C
:105A600029B31C464FF0010AC4E70028E0D10646DE
:105A7000002C04F1FF3AEADD54464D4541462846E4
:105A800000D2B847013CF8D2013656443046BDE852
:105A9000F88F06460028DAD02646C9E72646A246F1
:105AA0004FF0FF34C4E72646002CB0D1CFE76FEAB1
:105AB000040A0E46E0E700BF0FB430B583B006AB72
:105AC0000C4853F8042BD0F8241ED0F8200E019374
:105AD00071F0C2FF084C0546D4F8200E03685B69DC
:105AE00098470028F8D0284603B0BDE8304004B0FD
:105AF000704700BF18330020202200200EB410B5DC
:105B000083B005AB044653F8042B0749009301A862
:105B1000019471F0A1FF019B00221A7003B0BDE84F
:105B2000104003B0704700BFC10C00080CB470B542
:105B3000334CD4F8283EA4B0002B5BD094F8303E10
:105B400099420AD9D4F8342E01238340134204D158
:105B500024B0BDE8704002B07047D4F83835294A07
:105B6000A2FB030292094FF47A7101FB123304A8DD
:105B70002549FFF7C3FF04AA29AB0244CDE902324D
:105B80002249289A064603A871F066FF039B0A2261
:105B9000591C03911A70039B0022591C03911A701F
:105BA000D4F8285EADB12B685B6A1BB128469847D4
:105BB000D4F8285E9DF810100029C9D00DF1110409
:105BC0002B6828461B68984714F8011B0029F7D159
:105BD000BEE7D4F82C3E002BBAD03044022200920B
:105BE00004A98218FD2039F067FB24B0BDE870409D
:105BF00002B07047D4F82C3E002B9FD1A8E700BF1D
:105C000018330020D34D621034E10808ED09000874
:105C1000194A10B5D2F8384E033004EB9003B3F5AF
:105C2000007F19D8C2F8383E02F63C6202EB8404C9
:105C3000124A02EB810120F00300D1F84425C3F59C
:105C400000731044C1F844050D4A9B000421002054
:105C5000FFF76CFF204610BD00210846094AFFF7F8
:105C600065FF094AD2F8A830002443F00073C2F857
:105C7000A830204610BD00BF18330020104400207B
:105C800040E1080864E10808000000102DE9F04137
:105C90000268214D0746002455F834309A4209D055
:105CA00001340E2CF8D11D4A00210520FFF73EFFDC
:105CB000002013E01A4B03EB8408D8F8C0657EB1CE
:105CC000797901EB410306EBC30300221820C3E9F5
:105CD000032200FB01609F601A750430BDE8F0816B
:105CE00007216420FFF794FF0146C8F8C00568B19A
:105CF0003146642278F02CFED8F8C06505EBC40567
:105D0000C6E90056F6617663F664D9E7054A0520D0
:105D1000FFF70CFFCCE700BF4825080874E108082E
:105D2000183300209CE1080870B50668F46982B059
:105D30000546002C3FD03379012B04F103022DD00E
:105D4000022B26D1B36813F0010F30464FF00D033C
:105D500014BF0C218C2103F0BDF9A070D8B1B4F9A7
:105D60000A3007EE903AF8EEE77AC5ED077AB4F913
:105D70000C3007EE903AF8EEE77AC5ED087AB4F900
:105D80000E3007EE903AF8EEE77AC5ED097A02B0E8
:105D900070BD0023A370002002B070BDB368717C99
:105DA00096F91000009203F0010301930C220D23D9
:105DB000FDF7A0FCD1E709211420FFF729FFF061CE
:105DC00004462E68B7E700BF38B50568EB6904469E
:105DD000E3B1987800B938BDB3F9042007EE902AF2
:105DE000F8EEE77A0120C4ED047AB3F9062007EE55
:105DF000902AF8EEE77AC4ED057AB3F9083007EE99
:105E0000903AF8EEE77AC4ED067A38BD09211420FD
:105E1000FFF7FEFE0346E861DBE700BF03685A1C9C
:105E200002601878704700BF03681A46591C016069
:105E300012F8021B0260587841EA0020704700BF48
:105E400010B402681346511C016013F8021B036072
:105E5000D31C5478036093781B0443EA0423141D75
:105E60000460D0785DF8044B0B4343EA0060704750
:105E700012B370B50446864604E0981B17D114EBA4
:105E80000C0C15D01EF8013BA3F14100192811F8A4
:105E9000010BA0F1410598BF2033192DA2EB0E0C88
:105EA00000F12006E9D91B1A04D10028E7D170BD02
:105EB000604670BD184670BD1046704710B4028829
:105EC0008378184C02F0030101EB4101013B03EB25
:105ED000810304EB4303C178B3F8FC30A2F5FA6206
:105EE000920840F2B55404FB02334A1E1344017970
:105EF00042798479008903EB430301EBC301C1EBD1
:105F00000111094B02EB8102C2EB0212234403EBA5
:105F1000820300214FF47A72C3FB02015DF8044B47
:105F2000704700BFBC24080880436D38F8B516469A
:105F30001F460446394630464FF47A7200237BF000
:105F4000F7FC3C4D3C4B054483FB05602844E917B6
:105F5000C1EB601183FB01030B44384EC817C0EB43
:105F6000631086FB003CC317354EC3EBAC0386FBC6
:105F700003764FEAE37ECEEBE61EC1EB0116A5EBFE
:105F8000860CC0EB0015A1EB8501617103EB4301A9
:105F9000A0EBC10040F2B55101FB1E33B3F5896F90
:105FA00084F806C020714FEA8E0637DA40F2DA2113
:105FB0008B4239DCB3F5B77FB4BF4FF0000E4FF022
:105FC000010E20490EEB4E0001EBC0017546B1F801
:105FD00012014FEA4E071C4907EB0E0C01EBCC0CEB
:105FE0000CF1160C0B2101E03CF8020D984212DD79
:105FF0000139F9D11349774401EBC701B1F8FC002D
:106000000121013306F5FA6E1B1A7544A170E37085
:1060100022812580F8BD0131C9B2F2E7032540F2A3
:106020009650AE460627D6E7022540F22940AE46F6
:106030000427D0E780BC92C789888888ABAAAA2A9F
:1060400073B06D16BC240808B825080830B52F4C6D
:1060500086460D460FCC8DB0EC46ACE80F000FCC59
:10606000ACE80F0094E80F001EF0030F8CE80F005F
:106070000FD1274B274A03FB0EF3B2EBB30F43D3E9
:10608000254AB2EB331F34BF01220022C2F11D02A8
:1060900000E01C220EF1FF33002B019240F26D1242
:1060A000194602FB0EF2B8BF0EF1020102EBA1028B
:1060B0001A491B4C81FB0301DB17A3EB611002445F
:1060C000C3EBE1131A44253284FB02311144D31788
:1060D000C3EBA103C3EBC303D31AADF10402EE4635
:1060E00002EB85015EF8040FC21884FB023C944465
:1060F000D317C3EBAC03C3EBC3037145A2EB03039C
:10610000F0D1C01A0DB030BD1D22C3E71826080813
:10611000295C8FC2285C8F020AD7A3001F85EB5130
:10612000932449920E4B10B5D3F8D045D3F8D4350B
:1061300054EA030209D1014640F201130020C1F8DC
:10614000023088710880088110BD064AD2F83825CF
:10615000121943F10003FFF7E9FE012010BD00BF53
:10616000104400201833002088422DE9F0414FF000
:1061700001043DD301FB04F4B0FBF4FC8C45F9D2DF
:106180003CB3002616E0BCF1090F274698462C4682
:1061900023DD002A0CBF4FF0570E4FF0370EF444AA
:1061A000B94288F800C003F1010306F1010610D8D6
:1061B000B0FBF5FCB4FBF1F504FB1C00002EE2D1B2
:1061C000BCF1000FDFDCA1420AD90CF1300C03F85E
:1061D00001CB00221A70BDE8F0814FF0300EDEE7EF
:1061E000B0FBF5FC2C4605FB1C00B5FBF1F5E7E721
:1061F0008446C6E72DE9F041044694421546084618
:1062000009D2B4FBF2F6154B05FB16441B5D00F8F2
:10621000013BBDE8F081B4FBF2F69642B6FBF2F723
:106220000CD20E4B05FB176705FB1644DA5D00F830
:10623000012B1B5D00F8013BBDE8F081BA42B7FBC2
:10624000F2F807D9054B05FB187813F8082000F879
:10625000012BE7E74046FFF7CDFFF3E7B8E1080879
:10626000B5EEC00ADFED347AF1EE10FACCBF30EEB5
:10627000270A30EE670ADFED317A20EE270A30B5C3
:10628000FDEEC07A87B017EE904A054684EAE470C6
:10629000002303A9A0EBE470CDE9003302936DF075
:1062A00091FF002CB4BF2D23202303A88DF80030CC
:1062B0007AF006FC012829D0022833D003281DD00B
:1062C00003A968467AF03CFB68467AF0F9FBC41EE5
:1062D000E4B222466946284676F022FF00232B5579
:1062E00028467AF0EDFB2E232B5401300DEB0401F0
:1062F00028447AF045FB284607B030BD302303A977
:1063000068468DF801307AF01BFBDDE743F230027E
:10631000302303A96846ADF801208DF803307AF0E8
:106320000FFBD1E743F2300303A96846ADF8013013
:106330007AF006FBC8E700BF6F12033A00007A4408
:106340000278202A034600F10100F9D0092AF7D08B
:106350002D2A29D02B2A03BF5A78B7EE000A03460C
:10636000B7EE000AA2F13001C8B20928DFED4C7A7D
:1063700010D8F2EE046A07EE101AB8EEC77A13F8D6
:10638000012FA7EEA67AA2F13001C8B20928F0EEDB
:10639000477AF0D92E2A49D0197801F0DF01452932
:1063A00007D020EE270A70475A78BFEE000A03464E
:1063B000D8E710B459782D2962D02B2954D0A1F1F7
:1063C0003002092A03F1010355D80024002202EB10
:1063D000820201EB420213F8011FA1F130000928EB
:1063E000A2F13002F3D9B2F59A7F134628BF4FF4D9
:1063F0009A73072A50D9DFED2B6A1A46B7EE007A56
:10640000083A072A27EE267AFAD803F007032BB1B9
:10641000F2EE046A013B27EE267AFBD16CB3C7EE9D
:10642000877A5DF8044B20EE270A70475978A1F16E
:106430003002D0B2092803F10103AED8F2EE046AAB
:10644000F0EE665A07EE102AB8EEC77A13F8011F6D
:1064500087EE266AA1F13002D0B2092866EEA56A5D
:1064600077EE867AEED998E79978A1F13002092A79
:1064700003F10203A9D9B7EE007A67EE877AD0E775
:106480009978A1F13002092A03F1020388BFB7EE1F
:10649000007AC4D8012499E7B7EE007AB7E700BFC5
:1064A0000000000020BCBE4C0378202B024600F107
:1064B0000100F9D0092BF7D02D2B08BF5378A3F199
:1064C0003001CBB206BF02464FF0FF3C4FF0010C4B
:1064D000092B4FF0000000D9704712F8013F00EB84
:1064E000800001EB4000A3F13001CBB2092BF4D9BD
:1064F0000CFB00F0704700BF2DE9F04F91B048F061
:106500007BFD48F03DFDB0F1000A40F33C810024E2
:10651000DFF80C93B54D27462646A04604E006F565
:106520000066B24540F3958020220DEB0201304613
:1065300048F0B0FCAE49122208A877F02BF9834648
:106540000028ECD1BE4222D0AA4BAB4908EB48024E
:1065500003EB820308F10108424601931846F31B3E
:106560000293FFF7CBFA4A46019B42F84C3B029B51
:10657000C9F80C70C9E90433D9F81C30C9E90833EB
:106580009E4BC9F828300123C9F8083091469C4B2E
:10659000D3F8F035C9F81C303746122202F1400317
:1065A0000DEB03012B5D11F8201C994202F1010251
:1065B0000BD00024202AF1D12037BA4508A938464B
:1065C0003EDB48F067FC0022E8E70134152CF1D1EE
:1065D000D01920220DEB020148F05CFC894907AA82
:1065E00008A876F029FD58B30023CDE90133CDF892
:1065F00014B0039304931F469B467B1E042B00F2AA
:10660000BA81DFE803F082728A860300CDF814B005
:10661000FFF74AFF059B8346049989B1DDE9012014
:1066200042EA401203985B0143EAC023A1F2BC7125
:1066300043EA6B0342EA412243EA0243C9F81C30B1
:10664000B8F1640F6DD0374606F50066B2453FF7E6
:106650006BAFB8F1640FC34663D0BE421BD0654C2C
:1066600065490C2303FB084408F1010B5A462046F8
:10667000FFF744FA614BC9F82830F61BD9F81C30F3
:10668000C9F80040C9E90376C9E908330123C9F80C
:106690001460C9F80830BBF1000F0BF1040143DCB2
:1066A000594C574A4FEA4A03B3F1805FD2F8F0558C
:1066B0006EDB564954484FF4987276F031FD544BD6
:1066C000A3F11C0203F598719D60C3E900554C339A
:1066D0008B42F9D1A06828B923791BB12368002B1C
:1066E00040F0A28011B0BDE8F08FFFF7DDFE019011
:1066F0004449002007AA013776F09EFC00287FF469
:106700007CAF5B46DDF814B086E7FFF7CDFE029064
:10671000EEE7FFF7C9FE8346EAE7FFF7C5FE039001
:10672000E6E74FF0640B6821374C354AD4F84C61EA
:10673000C2F8F0654C2707FB01F563193A460021C2
:10674000184678F005F93A46002178F001F9314A07
:10675000625105F11002DFF8CC80284FC0F820808C
:106760004FF00109C0F80890876244F802A0224463
:106770001835C2F804A0221D0BF10501565115442D
:106780006E6046628DE71E4B1F4CD3F8F055042116
:106790004FF04C0808FB01F6A71942460021384685
:1067A00078F0D6F842460021384678F0D1F81A4BF6
:1067B000A3514FF0010906F11002DFF86880C7F815
:1067C0000890CAF1006303FA09F34FF0020BC7E91E
:1067D000078887F805B01148A35006F11801224434
:1067E0005360455001444D607D6262E704E2080851
:1067F000E0E10808E8490020F4E108082D25000838
:10680000F81000201CE20808B84E002048260808AE
:10681000D44E002024E2080834E20808BC4E0020D0
:10682000E84F00200068994F002600275449A064D3
:10683000C4E91067E063064607469646CD6C01F151
:106840004C036DB39D689F6406F1FF3C6545C1E94B
:106850002377DF630ED006F1010C65451DD113F8D7
:10686000486C002E3FF43EAF196443F8083C2E46B6
:106870001946E3E7002E3FF435AF53F80C1C2E46C3
:10688000002E3FF42FAF0D6CEA6B02F1010CC5F83E
:106890003CC01D648B641946D0E7B542F0D021E7B7
:1068A000724602272E46A64615E0D36B17635B019E
:1068B00018BF03F6FF73C2E9046614BF01EB13337C
:1068C0003B4653631946916352F84C4FCB1A1D4413
:1068D0004F1C0130CCB11379791E002BE5D113691F
:1068E00017635BB103F6FF73546901EB1333536312
:1068F0004CB104F6FF7C01EB1C31E4E754693B46E4
:106900005363002CF5D13946DDE71E4A1E4BC2F811
:106910001C0E013902F55F60C2F8F43D3E264023AB
:106920003F27C2F8105EC2F8003EC0E90267744615
:10693000C2F80C1E8D0F8B00D9B140F2FF169B19C7
:1069400045F100055B0A43EAC553C0E9094403F178
:106950004004234403EBC101C2F8083EC2F8F01D15
:10696000CB0D490240F8043CC2F8044E40F8081C24
:10697000B8E60123E9E7FFF797FD0490B8E600BF0A
:10698000B84E00202022002044E2080870B5344DA3
:106990002B787E2B01D0002070BD08224FF4FC43E1
:1069A00041F2210019B200294FEA4303B6BF80EA41
:1069B00041019BB28BB2013AF4D1B5F8011069B331
:1069C0002848294CA042E6D206384618A642E2D210
:1069D00041F2210C0529DED9864214D0013806F196
:1069E000FF3E10F8012F082183EA02231AB2002A81
:1069F0004FEA4303B6BF8CEA42029BB293B201391D
:106A0000F4D17045EDD1318849B1B21DA242C2D254
:106A10007218A2423046BED21646DBE7134E741EF1
:106A200041F22100A44614F8012F082183EA022331
:106A30001AB2002A4FEA4303B6BF80EA42029BB271
:106A400093B20139F4D16645ECD17288D01A084A64
:106A5000331D5B1BB0FA80F04009A2F8883A70BD84
:106A600000000E0807000E080000100801000E08C4
:106A7000104400202DE9F04F914B924A8BB000203A
:106A8000D21ACDE90600CDE90800D11805928E4A48
:106A90000393049110690028C0F281818A4AF3208F
:106AA000D060002008908948012288428DF8242077
:106AB00000F271817E2007928DF818004FF4FC429D
:106AC000082041F2210514B2002C4FEA4202B6BF61
:106AD00085EA440492B2A2B20138F4D17C48ADF800
:106AE00002207C4A90427CD2804641F22105B8F8CF
:106AF0000200B8F80020C0F30B07C2F30B04120B1E
:106B0000BE1D4FF000098DF808200204ADF80460A6
:106B1000ADF806408DF8099000F1C38006338B4232
:106B200000F2398101AE0DF10A0B344601E0A345B4
:106B300013D0079B14F8011B03F128026A440133A8
:106B4000042B079302F8101CF1D106A903A8FAF749
:106B5000D9F8A345CDE90790EBD1089B002BC0F2F3
:106B60001A81BDF8024016F8013B082284EA03248A
:106B700023B2002B4FEA4404B6BF85EA4303A4B214
:106B80009CB2013AF4D1B345EDD1D8F804603A464D
:106B9000314603A8FAF776F90028C0F2FC80F01914
:106BA000864213D0711E013811F8013F082284EA91
:106BB000032423B2002B4FEA4404B6BF85EA430303
:106BC000A4B29CB2013AF4D18142EDD1DDE90302D5
:106BD000ADF8024011463F4A08F1140890450346BB
:106BE00085D302334FF000089942ADF80480C0F01D
:106BF000D28001AD2E460DF106042F4601E0BC42C5
:106C000013D0079B17F8011B03F128026A440133D4
:106C1000042B02F8101C0793F1D106A903A8FAF778
:106C200071F8BC42CDE90780EBD1089B002BC0F284
:106C3000B280BDF8023041F2210016F8012B83EA40
:106C40000223082219B200294FEA4303B6BF80EAA3
:106C500041019BB28BB2013AF4D1B442EDD1039918
:106C6000ADF80230049B0231994200F294800DF19C
:106C70000206144602E0B54200F08A80079B16F82F
:106C8000011B03F128026A440133042B02F8101C93
:106C90000793F0D106A903A8FAF734F8CDE9074025
:106CA000E9E7CB460BF1010B06335FFA8BFB994208
:106CB0008DF809B06FD301AE0DF10A0A34460DE02C
:106CC00000000E0800001008003C024001000E0801
:106CD00088560908EC5B0908A24515D0079914F8F5
:106CE00001CB01F128030DEB0300013104290791C9
:106CF00000F810CCF0D106A903A8FAF703F8002396
:106D0000A24508900793E9D1089A002A43DBBDF811
:106D1000024016F8012B082184EA022422B2002A3C
:106D20004FEA4404B6BF85EA4202A4B294B20139E4
:106D3000F4D1B245EDD1D8F8041001EB09063A467A
:106D4000314603A8FAF79EF8002824DBF0198642A2
:106D500013D0711E013811F8013F082284EA032480
:106D600023B2002B4FEA4404B6BF85EA4303A4B222
:106D70009CB2013AF4D18142EDD1DDE90302BBF1CD
:106D8000030FADF8024003461146B9448AD121E70A
:106D9000089B002B09DA00200BB0BDE8F08F1548E6
:106DA000506000F18830506078E6079840B9124989
:106DB0000A6942F000420A61B3FA83F04009EBE746
:106DC000DDE9033203449342E5D806ABC0F1040287
:106DD0000021184477F0BCFD06A903A8F9F792FF3B
:106DE000002803460890D6DB9DF82420002AE3D033
:106DF000DDE700BF23016745003C024008B5FFF70F
:106E000039FE40B9FFF736FE28B9FFF733FE10B957
:106E1000052007F0DBFBFFF7B9FD0028F8D008BD1F
:106E200070B545880B460446C5F30B052A4600217C
:106E3000184677F08DFD0A4A21699142034606D330
:106E4000084A914206D3BDE8704018460847002919
:106E5000F9D170BD2A46BDE8704076F061B900BF37
:106E6000EC5B0908FF6009082DE9F04103EB4306DC
:106E7000964602EB460612F9067B86B00346754637
:106E800092F80080A3EB0804A3EB070C002CB8BF1A
:106E90006442BCF1000FB8BFCCF1000C6445B8BF30
:106EA000154602F10602B8BF4FFA88F7B242E7D1A1
:106EB0006A889EF80000B842144614D1BEF8020059
:106EC000A1EB0008A1EB020CB8F1000FB8BFC8F1AC
:106ED0000008BCF1000FB8BFCCF1000CE045BEBF0C
:106EE0007546024604460EF1060E7645E1D16A79F2
:106EF00004922A79CDE902422878054ACDE90010AA
:106F000003210120FEF712FE284606B0BDE8F081FD
:106F10004CE208084FF40063838170474FF400632C
:106F200083817047074B10B403F11001002453F81C
:106F3000042B824208BF43F8044C8B42F7D15DF822
:106F4000044B7047307E00200120704701207047BD
:106F50002DE9F04F734D2869AB8AB5F920E0B5F9FA
:106F60001CC0B5F81A80B5F9226085B0C3EB2014B7
:106F7000009204FB04F4B5F91820CDF80CE02413BA
:106F800002FB04F45B00B5F916200296C3EBE003A4
:106F900002FB03F3A41304EBE3242B6B0193A4F58E
:106FA000FA30B5F91E30EC6280FB00EA4FEAE37B71
:106FB00003FB0AF98CFB00C20EFB0B99A3FB0E3BF3
:106FC000CB4412031B0A42EA1C5243EA0B634FEA0A
:106FD0000C3C13EB0C0342EB2B22A3FB083C02F509
:106FE000004208FB02CC4FEAEC734FEA6C0953EA0B
:106FF0006C0C0F46B5F9241000F09180029E019AA6
:1070000086FB0008C2F5801C01FB0AFA4A464FEADB
:1070100048484FEAE17948EAD0380EFB09A9400414
:10702000A1FB0E1E4118F14449EB080900200CF0A9
:107030000048039E411848EA5C084FEACC7CBCEB50
:10704000010C09EBC60968EB09081CEB0C0E48EBB8
:1070500008011EEB0C0E48EB010188014FEA8E1966
:1070600040EA9E601EEB090E41EB0001890041EAF7
:107070009E714FEA8E0E1EEB0C0E48EB01014FEA9B
:107080008E00890010EB0C0041EA9E7148EB010173
:107090007AF04EFCB5F92A304FEA61384FEA503E9B
:1070A0004EEAC14EDA1703FB08F984460EFB02993B
:1070B000B5F92800B5F92620A3FB0E35A94403FB3A
:1070C00008F50EFB0955A3FB0E3E75445B0E43EA23
:1070D000C51313EB0C0341EB65654FEAE07E00FB43
:1070E00001F10EFB0C11A0FB0C0C6144C00C40EA3A
:1070F00041301B1845EBE1451B0A43EA056303EBEE
:1071000002130FB11B0A3B60009B23B104EB840404
:10711000803424121C60012005B0BDE8F08F0023EC
:10712000EFE700BF307E002031B10A4BD3ED147A77
:10713000FDEEE77AC1ED007A52B1064B9FED067A7B
:10714000D3ED157A67EE877AFDEEE77AC2ED007A25
:1071500001207047307E00200000C84201207047A7
:1071600010B40E4B0E4C1B68A06D1B1AFA2B09D8DD
:1071700009B1236E0B600AB1636E136001205DF8E4
:10718000044B7047074A1368002023F0040384F877
:107190005C0013605DF8044B704700BF503800205E
:1071A000307E0020AC00001001207047044B00220C
:1071B00000219A66DA661A6759670120704700BF96
:1071C000307E00200F4B104A1B68516F5B1AFA2B60
:1071D00016D8D2ED1A6A92ED1B7AD2ED1C7AFDEE2A
:1071E000E66ABDEEC77A16EE903AFDEEE77AC38600
:1071F00017EE103A038717EE903A43870120704745
:107200000020704750380020307E00200048704732
:10721000EC16002000487047A87E002030B50F4AC9
:1072200083B092F888500191B5B9D2F88C509DB1D5
:107230002B681A6882B19B6873B104462846984748
:1072400050B12B68019922461C6828460B462146FE
:1072500003B0BDE83040084703B030BD307E0020A9
:107260000B4B70B5D3F890608EB133681A6872B169
:107270009B6863B1054630460C46984738B1336881
:107280002A46196830462346BDE87040084770BD5D
:10729000307E0020437913F0010306D0D0E9073196
:1072A000C268581A531E184070471846704700BFEE
:1072B000437913F0020307D0D0E909130269581E7D
:1072C000401A531E184070471846704743790246CB
:1072D00013F0010014D0106AD168D36901F1FF3CAA
:1072E0001B1A13EA0C030AD053691B5C00F1010C52
:1072F000D8B2BCFBF1F301FB13C31362704718460D
:10730000704700BF43799B070AD5436A8269D1540D
:10731000436A02690133B3FBF2F102FB11334362AA
:10732000704700BF4171704781717047D0E90920F3
:10733000101AB0FA80F04009704700BF024BD3F832
:1073400094305B68184700BF307E0020024BD3F8B2
:10735000943008309B681847307E00200120704729
:1073600001207047012070470120704701207047BD
:1073700031B10C4BD3ED267AF8EEE77AC1ED007A05
:107380007AB1084BDFED086AD3F89C30A3F5D543FA
:10739000333B07EE903AF8EEE77A87EEA67A82ED75
:1073A000007A7047307E00200000C84201207047FC
:1073B0000120704710B4754C0023224692F9041046
:1073C000012902F10C023AD00133072BF6D12246F3
:1073D000002392F90410022902F10C0245D0013376
:1073E000072BF6D12246002392F90410032902F15B
:1073F0000C0255D00133072BF6D12246002392F917
:107400000410042902F10C025ED00133072BF6D1DF
:10741000002394F90420052A04F10C0468D00133F8
:10742000072BF6D15A4B5B685B067BD401795DF87C
:10743000044B203901298CBF002001207047554A98
:1074400003EB430302EB8303D3F8A03003B3524AA8
:10745000037992F83DC09C4503D092F83C209A42B3
:10746000B5D101205DF8044B70474A4A03EB430352
:1074700002EB8303D3F8A03063B1484A037992F852
:107480003D109942EDD092F83C209A42AAD1E8E70B
:1074900022469EE722460C3212F9081C0329A9D184
:1074A0003C4A03EB430302EB8303D3F8A030002BE9
:1074B00036D03B4A037992F83D109942D1D092F8E8
:1074C0003C209A4299D1CCE7324A03EB430302EBCA
:1074D0008303D3F8A030002B9BD0324A037992F873
:1074E0003D109942BDD092F83C209A4290D1B8E725
:1074F000284A03EB430302EB8303D3F8A030002BAD
:1075000090D0294A037992F83D109942A9D092F877
:107510003C209A42A5D01E4B5B685B0686D501E0F5
:1075200022466CE7214B00229C4619460C791A2C06
:1075300001F1140104D001320C2AF7D1002403E038
:1075400002EB82020CEB820400221979192903F163
:1075500014030BD001320C2AF7D1002C3FF466AF94
:10756000226803689A427FF461AF7AE701681CB130
:1075700023688B423FF475AF0D4B02EB820203EBA5
:1075800082031B698B427FF451AF6AE7D07E0020F3
:10759000AC000010307E0020B4000020000300206A
:1075A0004C05002098070020E4090020FC1600206C
:1075B000EC1600200C4B10B5844603F1F00E0020B1
:1075C00002E014339E450ED01A686245F9D1DA689C
:1075D0008A4218BFD96000F1010403F1140318BFF7
:1075E000E0B29E45F0D110BDFC160020704700BFF0
:1075F000044B40F2FF7203EBC0039142A8BF114657
:1076000099807047E83F0020112807D8044B03EB0E
:107610008003D3F8F8300BB19B68196031F026BABB
:10762000307E0020112807D8044B03EB8003D3F8E9
:10763000F8300BB19B681960704700BF307E0020A6
:107640000D4A92F8003183B10C4B93F8401161B1AF
:1076500093F8411161B1D2F804010022FA2883F8AD
:107660004121A8BF4FF0FF3070476FF00100704715
:107670006FF00200704700BFEC160020307E002043
:107680000C4B93F842218AB193F843215AB10A492D
:10769000D1F808010022B0F5967F83F84321A8BFF6
:1076A0004FF0FF3070476FF0020070476FF001003D
:1076B000704700BF307E0020EC160020024BD3F84C
:1076C00044315B68184700BF307E0020024BD3F87E
:1076D00044319B68184700BF307E0020024BD3F82E
:1076E0004431DB68184700BF307E0020014BD3F8DF
:1076F0000C017047EC160020054B93F848311BB184
:10770000044BD3F8100170476FF00100704700BFC1
:10771000307E0020EC160020014BD3F84C0170475E
:10772000307E00204B1EDBB2062B98BF214A30B5BD
:1077300098BF32F81350204BA3F1580488BF4FF480
:107740008075002808BF1C46A44620893CF8082BF9
:1077500087B04FFA82FE90B1A5EB0E022B1A002AD9
:10776000B8BF5242002BB8BF5B429A42C4BF6446C6
:107770004FFA80FE3CF8080F0028EDD122880F4B0D
:107780000F4893F850C1A3790593A38804930D4B38
:10779000BCF1000F18BF0346A078CDE90015CDE974
:1077A00002200321084A0120FEF7C0F9204607B055
:1077B00030BD00BF7032080858180020307E00200D
:1077C00088FB080884E3080888E3080870B50668A1
:1077D000F0690D461446A0B3D0F80130CDB1D0F811
:1077E00005209FED1B7ADFED1B5ADFED1B6A07EECC
:1077F000902AF8EE677AB7EE006A77EEC77A77EEEE
:10780000A77A87EEA57A77EE467A67EEE67AC5ED37
:10781000007AACB107EE903A9FED107ADFED106A76
:107820009FED106AF8EEE77A67EE877A87EEA67A20
:10783000DFED0D6A77EE467A77EEA67AC4ED007A30
:1078400070BD09211420FEF7E3F9F061C4E700BF21
:107850009AC9CC449AC94C460E76D7450000484395
:1078600000E0FF44000048423393884370B5066847
:10787000F06982B00D461446002848D0D0F8053093
:10788000DFED266A9FED267A07EE903AF8EE677AEA
:10789000D0F8013077EEE67AF3EE096A67EE877A80
:1078A000B2EE047A67EEA67AF4EEC77AF1EE10FA39
:1078B00020DCBAEE047AF4EEC77AF1EE10FA19D4AD
:1078C0002DB19FED187A67EE877AC5ED007A7CB10D
:1078D00007EE903A9FED146ADFED146AB8EE677A0E
:1078E000DFED137AE7EE067A77EEA67AC4ED007A3A
:1078F00002B070BD17EE900A79F036FB0D4ACDE963
:10790000000104210320FEF711F902B070BD092126
:107910001420FEF77DF9F061B0E700BF00000046DB
:10792000000080380AD778430319C83D3393884351
:10793000000048C2D4E30808244B254A30B5D3F8E8
:10794000544194F91030A16803EB830302EB8302E6
:1079500083B08DF80700D2F8CC018A070AD501233D
:107960000DF1070200216FF04FFFA3689B0714D5AC
:1079700003B030BD636913B11A689B885383154BFC
:1079800015491A68154B4D68D200A3FB02329209C3
:107990004B685B1B9A42FBD2E1E70E4B0E491A681B
:1079A0000E4B4FF4FA7000FB02F2A3FB0232486860
:1079B00092094B681B1A9A42FBD26369002BD7D0FD
:1079C0001A689B88138303B030BD00BF307E00204F
:1079D000EC16002074390020001000E0D34D621036
:1079E00070B52B4C94F8583182B023B9012084F83B
:1079F000583102B070BDD4F85451264A95F9103070
:107A0000A96803EB830302EB83030522ADF8002092
:107A10008A07D3F8CC0111D502236A4601A96FF079
:107A2000F3FEAB689B071CD59DF8053003F00103FE
:107A300083F0010084F8583102B070BD6B6913B156
:107A40001A689B885383144B14491A68144B4E6868
:107A5000D200A3FB023292094B689B1B9A42FBD2D5
:107A6000DAE70D4B0D491A680D4B48684FF4FA766A
:107A700006FB02F2A3FB023292094B681B1A9A42E0
:107A8000FBD26B69002BCFD01A689B881383CBE79E
:107A9000307E0020EC16002074390020001000E039
:107AA000D34D62102DE9F04782B060B9364D95F89C
:107AB0005831D5F85C7173B900230120C5F85C31E9
:107AC00002B0BDE8F087314B2F4D1F6895F8583153
:107AD0000744002BF0D0DFF8BC802D4CDFF8B8A0B5
:107AE000DFF8B890D5F8546196F9103003EB8303B2
:107AF00008EB83030522D3F8CC01B368ADF800206E
:107B00009A072FD502236A4601A96FF07DFEB3685C
:107B10009B0712D59DF8053013F0010302D185F8BB
:107B20005831C9E7194B1B6801229F4285F858213B
:107B3000D8D8002002B0BDE8F087DAF800206168EC
:107B40004FF4FA7303FB02F2A9FB02329209636855
:107B50005B1A9A42FBD27369002BDBD01A689B88B0
:107B60001383D7E7736913B11A689B885383DAF8D4
:107B700000206168D200A9FB0232920963685B1A97
:107B80009A42FBD2BEE700BF307E00205038002072
:107B9000001000E0EC16002074390020D34D621074
:107BA00010B50020FFF77EFF00B910BD084C06207D
:107BB000FFF7C2FE0123C72084F85831FFF7BCFE4F
:107BC000044B1B6803F5A4430833C4F85C3110BDB3
:107BD000307E002050380020F0B5044689B00020E7
:107BE0000E461546FFF75EFF10B9204609B0F0BDFE
:107BF0001D4F0620FFF7A0FE012387F8583197F8A4
:107C00006021CDF80CD00223009300238DF80430BE
:107C10000293E2B1CDE9066505930522230E8DF8A6
:107C2000013004920DF10203220C1A70D7F85401AE
:107C30009C70220A5A700379022B10D00B4B1B68E0
:107C40002C4406332046C7F85C3109B0F0BDCDE9BD
:107C50000526042207950DF101030492E4E702A929
:107C60006FF022FEEAE700BF307E0020503800208F
:107C700070B5054688B000200E461446FFF712FF87
:107C8000E8B103220092164ACDF80CD092F86011A8
:107C9000059600238DF80430029391B9CDE90614BE
:107CA00004210DF101030491D2F854019D702A0CB6
:107CB0001A702A0A5A700379022B0CD0204608B099
:107CC00070BD290E8DF801100521CDE9063404910F
:107CD0000DF10203E8E702A96FF0E6FD2046EEE7AA
:107CE000307E0020F0B5064683B00020FFF7DAFEB4
:107CF00008B903B0F0BD324C0620FFF71DFE01228B
:107D000094F8603184F85821D82100228DF804209D
:107D1000D4F854510091C6F307420BBB70BA8DF8EA
:107D20000120ADF80200042395F91020254902EB4B
:107D3000820201EB8202A968D2F8CC018A0714D52D
:107D40006A4600216FF060FDAB689B0720D51E4B93
:107D50001B6803F59C530833C4F85C3103B0F0BDD5
:107D600030BACDF801000523DEE76A6912B1116867
:107D700092884A83154A164E1168164A7768C900D8
:107D8000A2FB012189097268D21B9142FBD2D7E77D
:107D90000E4B0F491A680F4B48684FF4FA7606FBF2
:107DA00002F2A3FB023292094B681B1A9A42FBD2E1
:107DB0006B69002BCBD01A689B881383C7E700BF81
:107DC000307E0020EC16002050380020743900204E
:107DD000001000E0D34D6210244B254A30B5D3F893
:107DE000644194F91030A16803EB830302EB830232
:107DF00083B08DF80700D2F8CC018A070AD5012399
:107E00000DF1070200216FF0FFFCA3689B0714D55A
:107E100003B030BD636913B11A689B885383154B57
:107E200015491A68154B4D68D200A3FB023292091E
:107E30004B685B1B9A42FBD2E1E70E4B0E491A6876
:107E40000E4B4FF4FA7000FB02F2A3FB02324868BB
:107E500092094B681B1A9A42FBD26369002BD7D058
:107E60001A689B88138303B030BD00BF307E0020AA
:107E7000EC16002074390020001000E0D34D621091
:107E8000274B284A30B5D3F8644194F9103003EBFE
:107E9000830383B002EB8302A3688DF804000025FE
:107EA000D2F8CC018DF8055049BA9A07ADF8061002
:107EB0000AD504230DEB030200216FF0A5FCA36893
:107EC0009B0714D503B030BD636913B11A689B8852
:107ED0005383154B15491A68154B4D68D200A3FB07
:107EE000023292094B685B1B9A42FBD2E1E70E4BD0
:107EF0000E491A680E4B4FF4FA7000FB02F2A3FB16
:107F00000232486892094B681B1A9A42FBD2636995
:107F1000002BD7D01A689B88138303B030BD00BFF5
:107F2000307E0020EC16002074390020001000E0A4
:107F3000D34D621070B52D4D2D4AD5F8644194F99A
:107F4000103003EB830302EB8303A26882B00020AE
:107F50004CF2050192078DF80200ADF80010D3F83D
:107F6000CC0119D503236A4601A96FF04DFCA36823
:107F70009B0724D595F868319DF806203BB102F0A7
:107F8000010383F0010085F8683102B070BD012063
:107F900085F8683102B070BD636913B11A689B88B7
:107FA0005383144B14491A68144B4E68D200A3FB38
:107FB000023292094B689B1B9A42FBD2D2E70D4BCF
:107FC0000D491A680D4B48684FF4FA7606FB02F229
:107FD000A3FB023292094B681B1A9A42FBD26369D7
:107FE000002BC7D01A689B881383C3E7307E00201C
:107FF000EC16002074390020001000E0D34D621010
:1080000070B55A4D5A4E82B0FF20FFF7E5FE2C683E
:10801000012304F5FA74C6F86C4186F8683103E070
:108020002B681B1B002B06DAFFF784FF0028F7D014
:108030000023C6F86C31D6F864414E4D94F91030E7
:10804000A2684AF2010103EB830305EB8303ADF859
:10805000041000218DF806109107D3F8CC0120D52B
:10806000032301AA00216FF0CFFBA3689A0743D531
:1080700094F9103003EB830305EB83034BF2010209
:10808000ADF80420D3F8CC0118228DF80620032384
:1080900001AA00216FF0B8FBA3689B0714D502B0BA
:1080A00070BD636913B11A689B885383324B33499F
:1080B0001A68334B4E68D200A3FB023292094B6818
:1080C0009B1B9A42FBD2CBE72B4B2C491A682C4BBB
:1080D0004FF4FA7000FB02F2A3FB023248689209E7
:1080E0004B681B1A9A42FBD26369002BD7D01A68DF
:1080F0009B88138302B070BD1F4B20481A68204B29
:1081000046684FF4FA7102FB01F1A3FB01318909C2
:1081100043689B1B9942FBD294F91030616903EBD1
:10812000830305EB8305D5F8CC01B1B10B688988D1
:10813000198359834BF20103ADF8043018238DF8ED
:1081400006300E490E4B4D68D200A3FB0232920955
:108150004B685B1B9A42FBD299E74BF20103ADF8E7
:10816000043018238DF80630EBE700BF50380020AC
:10817000307E0020EC16002074390020001000E052
:10818000D34D621070B50B4D0B4E2C680123044487
:10819000C6F86C4186F8683103E02B681B1B002B86
:1081A00006DAFFF7C7FE0028F7D00023C6F86C31C7
:1081B00070BD00BF50380020307E00202DE9F04F08
:1081C000DFF8C48198F870918BB007468B4616464D
:1081D000B9F1000F00F0A480D8F87451684CA8429F
:1081E0003AD1FFF7A7FE48B92268D8F86C11521AA5
:1081F000002A06DAFFF79EFE0028F5D00022C8F814
:108200006C210620FFF7E8FD0122ABB288F8682157
:108210000193C5F30A0AB9F1000F4FD105E02268B6
:10822000D8F86C11521A002A03DAFFF783FE0028EF
:10823000F5D08DF80EA04FEA1A2AD8F86401CDF8CF
:1082400020B08DF80DA00996022248E02268D8F8E7
:108250006C11521A002A06DAFFF76CFE0028F5D0DE
:108260000022C8F86C210620FFF7B6FD012288F82D
:108270006821D8F878214FEAD22905E02268D8F899
:108280006C11521A002A03DAFFF754FE0028F5D0C9
:1082900049461020FFF7F4FD226802324FF0000932
:1082A000C8F86C21012288F8709188F86821A1E74C
:1082B0002268D8F86C11521A002A03DAFFF73AFE46
:1082C0000028F5D0019BCDF820B0D8F864018DF8D6
:1082D0000EA0C3F3022B8DF80DB0099684228DF801
:1082E0000C20017900220492079203AA0592022928
:1082F0004FF0030206923ED022680232C8F86C2189
:108300000122354488F86821012288F87021C5F3DC
:108310000A02C8F8745142B1B8190BB0BDE8F08F29
:10832000C8E95D00164C054664E7D8F878214FEAA5
:10833000D229144AC2F81C9205E02268D8F86C11C0
:10834000521A002A03DAFFF7F5FD0028F5D0494656
:108350001020FFF795FD2268C8F878510232C8F85E
:108360006C2101210022B81988F8681188F8702161
:108370000BB0BDE8F08F04A96FF096FABCE700BF20
:1083800050380020EC160020307E002070B5134CD1
:1083900094F8703103B970BDD4F87861104B114D69
:1083A000F60AC3F81C6205E02B68D4F86C219B1A0E
:1083B000002B03DAFFF7BEFD0028F5D03146102070
:1083C000FFF75EFD2B6801210022023384F868115B
:1083D000C4F86C3184F8702170BD00BF307E00207D
:1083E000EC16002050380020F0B5314D314C83B0F0
:1083F000064605E02B68D4F86C219B1A002B03DAA3
:10840000FFF798FD0028F5D0D4F864712A4A0623B6
:108410008DF8073097F9103003EB830302EB8303E9
:10842000D3F8CC01BB689A0715D501230DF10702DB
:1084300000216FF0E9F9BB689B0721D5F10AD8202C
:10844000FFF71EFD2B6801220F3384F86821C4F862
:108450006C3103B0F0BD7B6913B11A689B885383FC
:10846000164B17491A68174BD1F804C0D200A3FB6A
:10847000023292094B68A3EB0C039A42FAD2D4E77A
:108480000E4B0F491A680F4B4FF4FA7000FB02F2C3
:10849000A3FB0232486892094B681B1A9A42FBD22E
:1084A0007B69002BCAD01A689B881383C6E700BF7C
:1084B00050380020307E0020EC1600207439002057
:1084C000001000E0D34D62102DE9F04F5D4DB5F87E
:1084D000783083B0002B55D0D5F864715A4EDFF850
:1084E00074A15A4CDFF870B14FF000094FEA4948C7
:1084F00005E03368D5F86C219B1A002B03DAFFF7EF
:1085000019FD0028F5D097F91030BA6803EB830302
:1085100006210AEB83038DF804109107D3F8CC01F0
:108520007ED5012301AA00216FF06EF9BB684FEAE6
:10853000D8209A07C8F3C748C0B23CD5D823ADF8B5
:10854000043097F910308DF8070003EB83030AEB32
:1085500083038DF80680D3F8CC0104230DEB0302CE
:1085600000216FF051F9BB689B070ED501213368DC
:10857000B5F8782085F8681189440F334A45C5F865
:108580006C31B3D803B0BDE8F08FDBF80030616820
:108590004FF4FA7203FB02F22D4BA3FB0232920955
:1085A00063685B1A9A42FBD27B69002BDED01A68A3
:1085B0009B881383DAE7DBF80020254BD4F804C04E
:1085C0004FF4FA7102FB01F1A3FB013189096368E1
:1085D000A3EB0C039942FAD24FF0000368F30703B0
:1085E00060F30F23ADF8063097F91030796903EB8B
:1085F00083030AEB8303D3F8CC0119B10B68898894
:1086000019835983D823ADF80430114B6168D20027
:10861000A3FB0232920963685B1A9A42FBD29CE781
:108620007B6913B11A689B885383DBF8003061685B
:10863000DA00074BA3FB0232920963685B1A9A4285
:10864000FBD26EE7307E002050380020001000E0A2
:10865000D34D6210EC160020743900202DE9F04F44
:10866000DFF8AC81D8F81C32B3EBD02F8BB00546C5
:108670008946174661D1614C614ECDF81C90D6F801
:1086800064910023C5F30A05C5F5006003228DF847
:108690000F300493089399F804308DF80C20B842F9
:1086A00003AAB4BF87B2BFB28DF80E5005922D0A4F
:1086B0000422022B8DF80D500997069200F0998044
:1086C000256801230235C6F86C5186F8683103E04D
:1086D00023685B1B002B2CDAFFF72CFC0028F7D05B
:1086E0004CF20503ADF8043099F9103003EB830325
:1086F00008EB8308D9F80830D8F8CC010022C6F876
:108700006C218DF806209A075FD5032301AA02A9E0
:108710006FF07AF8D9F808309B073ED59DF80A30FB
:10872000C3F30113013B022B33D938460BB0BDE82C
:10873000F08F00200BB0BDE8F08F304C304E4FEA88
:10874000D02A05E02368D6F86C219B1A002BF0DABA
:10875000FFF7F0FB0028F5D04FF0FF335146132010
:10876000C8F81C32FFF78CFB012386F868312368B8
:1087700003F1020BC6F86CB104E02368A3EB0B0312
:10878000002BD6DAFFF7D6FB0028F6D0C8F81CA2DB
:1087900073E7FFF735FC3846C8E71A4B1A491A68E1
:1087A0001A4B48684FF4FA7404FB02F2A3FB02323E
:1087B00092094B681B1A9A42FBD2D9F81430002B4D
:1087C000ACD01A689B881383A8E7D9F8143013B18A
:1087D0001A689B8853830B4B0B491A680B4B4C68E8
:1087E000D200A3FB023292094B681B1B9A42FBD2B8
:1087F0008BE704A948466FF057F861E7503800202E
:10880000307E002074390020001000E0D34D62104B
:10881000EC1600202DE9F0410C4E356873691D40BF
:1088200011D0DFF82C800127B5FA85F4C4F11F04BC
:1088300008EB840307FA04F4D3F87C010368984733
:10884000A5437461F0D1BDE8F08100BF003C014058
:10885000307E002070B583681C686379DB0748D5DB
:10886000A37994F85C22E06B03F001010E461ABB79
:1088700094F85F32012B3DD0002B3FD194F85E324B
:1088800094F85DE29E450ED9B4F86622012505FAFA
:1088900003FC013342EA0C025FFA83FCE64592B224
:1088A000F5D8A4F86622012384F85F3286EA030132
:1088B000BDE870406BF0AEBB43681A68D36AC3F37F
:1088C0004E03536294F86D32012B07D094F8613255
:1088D00023B1B4F868320133A4F8683286F001019C
:1088E0006BF098FB00224FF08073A4F86622C4F866
:1088F0005C3270BD94F85D3284F85E32002384F8F7
:108900005F32BDE870406BF085BB00BFF0B52DED68
:10891000028B4E4E16F83C3C022B83B00D4614469B
:1089200019D0DFED4B7A7DB19FED4A7A9FED4A6A0F
:10893000DFED4A6A67EEA77A67EE877A87EE867A76
:1089400077EE267AC5ED007A0CB1454B236003B073
:10895000BDEC028BF0BD434B96F820109B6803F0F2
:10896000020239BB5B0525D42AB3B6F9463007EEBF
:10897000903AB6F94430F8EEE77A06EE903A27EEF0
:10898000A77AF8EEE66AB6F94830A6EEA67A07EEC0
:10899000903AF8EEE77AA7EEA77AB5EEC07AF1EE54
:1089A00010FABEDBF1EEC77AF4EE677AF1EE10FA58
:1089B000B9D7B6E71AB9336ED3ED337AB3E72A4F96
:1089C0000DF106002EF030FEBDF80630D7F8AC25CC
:1089D0009FED266ADFED266A9FED267A9B1A07EE49
:1089E000903AF8EEE77AB0EE408A67EE867AA7EE24
:1089F000A67AFDEEC77AB0EE470A17EE903A20331A
:108A0000402B1FD8FCF7D4FE1B4B97F8D211D6EDA4
:108A10000B7AA3F12C021846443B002918BF1346D9
:108A200093ED057AD0ED006A77EE877AE8EE406A3A
:108A300027EEA77AA6EEA67AB5EEC07AF1EE10FA86
:108A4000B0DA6EE79FED020ADEE700BF288F002054
:108A500000000000CDCC9C3F00409C4682E6C5470C
:108A600033139043AC000010307E00200AD7233C23
:108A700035FA8E3CDB0FC93FF083002010B50B4B5D
:108A800082B053F8304001916CB107EE901A94ED2A
:108A9000047A94ED030AF8EEE77AA7EE870A70F0FD
:108AA000C3FBA368186002B010BD00BFE83F002000
:108AB000184B53F8200048B310B5174C00EB40009A
:108AC00004EB800393F965C0BCF1FF3F1FD093F81E
:108AD0006D00D0B104EB0C0293F86C0092F8B8E092
:108AE0008C23142103FB0CFC00220CEB000304EB91
:108AF00043030139B3F8BC30704412FA83F2F4D165
:108B0000064BA3FB0230C0F30F1010BD70470020CE
:108B100010BD00BF307E0020288F0020CDCCCCCCF3
:108B200030B5032083B00D461446FFF7C1FF019016
:108B30009DB107EE900A9FED0B7AF8EE677AF0EEA2
:108B4000006A67EE877AB8EE047AA7EEA67ADFEDC0
:108B5000067A67EE277AC5ED007A0CB1034B2360E5
:108B600003B030BD6740533A00007A44331390435A
:108B7000E8B170B506680E4B06F13F4202F57E0281
:108B800003EB92230C4682B00546187C6BF0F8FA92
:108B90006209C4F30013A9883046CDE90032C4F35A
:108BA000810304F003026EF0EFFB02B070BD70476A
:108BB0007032080870B5104B104CA3421AD205460B
:108BC00002E00C33A34215D293F805C08C45F8D1CE
:108BD00093F804C0AC4501D0002DF2D1D879904271
:108BE000EFD1186890F804E0E645EAD106689E42A5
:108BF000E7D170BD002070BD00610908B0620908AE
:108C00000379022B00D0704710B490F910201D4852
:108C10001D4C83B002EB82020831694400EB8202F2
:108C20000094D2F8CC2111F8084C18498A4225D07A
:108C3000A1F578418A4223D001F580618A4219D199
:108C4000118821F04001090403EB8303090C118012
:108C500000EB83001388D0F8D81123F0380331F8E3
:108C600024101B041B0C0B43138013889BB243F08E
:108C70004003138003B05DF8044B70470023DFE727
:108C80000123DDE7EC160020000102030030014063
:108C900010B50446C06900B110BD09211420FCF7CD
:108CA000B7FFE06110BD00BF034690F910002DE949
:108CB000F041244C00EB800016469A6804EB8000DB
:108CC0009207D0F8CC8109D540466EF083FE31463C
:108CD00040466EF07FFE0120BDE8F0815D690846E8
:108CE00015B12B68AA885A83174B184F1C68184B6C
:108CF0007A684FEAC40CA3FB0C3C4FEA9C1C7B68CF
:108D00009B1A9C45FBD2014640466EF063FE3146FD
:108D100040466EF05FFE0E4B78680C494FF4FA72D5
:108D200004FB02F2A3FB023292094B681B1A9A421F
:108D3000FBD2002DCFD02B68AA881A830120BDE872
:108D4000F08100BFEC16002074390020001000E014
:108D5000D34D621010B50379012B84B08E460DD02F
:108D6000022B02D0002004B010BD8368DB0758BF7F
:108D700001F07F0104B0BDE8104095E71446826819
:108D80008DF80F4002F0010201920DF10F020092E6
:108D9000417C90F910007246FBF7C8F804B010BD92
:108DA00010B50446002221210068FFF7D3FF206898
:108DB000FC222021FFF7CEFF206840222421FFF76C
:108DC000C9FF20680C222321FFF7C4FF206800227E
:108DD0002221FFF7BFFF012010BD00BF10B50446E0
:108DE00094220B210068FFF7B5FF20687122012152
:108DF000FFF7B0FF206800220421FFF7ABFF2068D7
:108E0000C8220521FFF7A6FF206800220621FFF7F0
:108E1000A1FF2068C8220721FFF79CFF20680022DD
:108E20000821FFF797FF2068C8220921FFF792FF6A
:108E3000012010BD00B500680379012B85B012D068
:108E4000022B03D0012005B05DF804FB8368DB072B
:108E50004FF031024CBFF4217421FFF725FF0120B0
:108E600005B05DF804FB826890F910C0417C02F007
:108E7000010201920DF10F0200926046F4224FF0C0
:108E8000310C8DF80FC0FBF751F8012005B05DF8EB
:108E900004FB00BF10B5044600680379012B84B0C1
:108EA00011D0022B02D0002004B010BD01220B21F2
:108EB000FFF7FAFE0028F6D020681D22092104B031
:108EC000BDE8104046E7826890F910C0417C8DF8FB
:108ED0000F3002F0010201920DF10F020092604684
:108EE0000B22FBF723F8E5E72DE9F04105461F4685
:108EF00095F91030244803EB830300EB8300AB6843
:108F0000D0F8CC8116469A070ED540466EF062FD29
:108F10003B463246002140466EF076FCAB689B072C
:108F200018D50120BDE8F0816B6913B11A689B88E0
:108F30005383164B164A1B684FEAC30E154BA2FB10
:108F40000E2E5A684FEA9E1E5C68A4EB020CE645A2
:108F5000FAD2DAE70D4B0F491A680D4B4FF4FA704D
:108F600000FB02F2A3FB0232486892094B681B1A0D
:108F70009A42FBD26B69002BD3D01A689B8813836B
:108F80000120BDE8F08100BFEC16002074390020FC
:108F9000D34D6210001000E030B50579012D83B08B
:108FA0008E460DD0022D02D0002003B030BD846863
:108FB000E40758BF41F0800103B0BDE8304093E7BB
:108FC00014468268009402F00102417C90F910007E
:108FD00001927246FAF7AAFF03B030BD10B5164CE5
:108FE00084F80514017984F8062401294FF0000261
:108FF00082B084F8042410D0022903D06FF00C0052
:1090000002B010BD032304F20442FF21FFF76CFFFE
:109010000028F3D0002002B010BD8268417C90F996
:10902000100004F2044402F00102CDE900420323DF
:10903000FF22FAF77BFFEBE7288F00200068037917
:10904000012B0AD0022B00D0704783680D4A13F021
:10905000010314D00023512146E700B58368094A73
:10906000417C90F9100083B003F00103CDE90023A7
:1090700000235122FAF75AFF03B05DF804FBD12117
:1090800032E700BF2C94002000680379012B0BD03D
:10909000022B00D0704783680D4A13F0010F4FF088
:1090A000010312D000211FE700B58268417C90F9CE
:1090B000100083B002F001020192054A00920022E2
:1090C000FAF734FF03B05DF804FB80210CE700BF22
:1090D0002C9400202DE9F04105461F4695F91030EB
:1090E000244803EB830300EB8300AB68D0F8CC810A
:1090F00016469A070ED540466EF06CFC3B460022A1
:10910000314640466EF080FBAB689B0718D50120C6
:10911000BDE8F0816B6913B11A689B885383164BC5
:10912000164A1B684FEAC30E154BA2FB0E2E5A6857
:109130004FEA9E1E5C68A4EB020CE645FAD2DAE721
:109140000D4B0F491A680D4B4FF4FA7000FB02F2F9
:10915000A3FB0232486892094B681B1A9A42FBD261
:109160006B69002BD3D01A689B8813830120BDE85C
:10917000F08100BFEC16002074390020D34D62103E
:10918000001000E030B50579012D83B08E460DD07A
:10919000022D02D0002003B030BD8468E40758BF20
:1091A00041F0800103B0BDE8304093E71446826887
:1091B000009402F00102417C90F910000192724685
:1091C000FAF798FA03B030BD10B504460068037989
:1091D00082B0022B0CBF4321032106236A46FFF70E
:1091E000D1FF68B1BDF80010BDF80220BDF8043011
:1091F00049BA52BA5BBAE1866287238702B010BDD2
:10920000C4F83600608702B010BD00BF70B50668B4
:10921000F56982B00446002D59D000232B70042339
:109220000DEB03023046FF21FFF7ACFF10B9002021
:1092300002B070BD206804236A46FF21FFF7A2FF39
:109240000028F4D09DF804309B09023B012BEED995
:10925000BDF80430BDF80620BDF80010BDF802606E
:109260005BBA43F6FF74C3F30D03A342DFD0002BB8
:10927000DDD052BAC2F34A1240F2FF7C6245D6D02A
:10928000002AD4D049BAC1F30D01A142CFD00029A0
:10929000CDD076BAC6F34A166645C8D0002EC6D0E1
:1092A0005C1A002CB8BF6442FF2CC0DC941B002C5D
:1092B000B8BF6442FF2CBADC0B445B10324452103E
:1092C000C5F805300123C5F801202B70B0E709214E
:1092D0001420FCF79DFCF061054626689DE700BF61
:1092E00070B50668F46982B0F4B1002323700423DA
:1092F0000DEB0302FF213046FFF744FF10B39DF84A
:1093000004309B0919D1BDF80420BDF8063052BACB
:109310005BBA92B2C3F34A1301212170C4F805204D
:10932000C4F8013002B070BD054609211420FCF7D5
:109330006FFCF06104462E68D7E7044A042103203D
:10934000FCF7F4FB002002B070BD00BFF8E3080892
:109350002DE9F041104C04F2044884F80514174636
:10936000002502234246FF21064684F80454FFF7F5
:1093700013FE68B1424630460223FF21FFF702FF89
:1093800030B1B4F804345BBA28463B80BDE8F081C4
:109390006FF00C00FAE700BF288F002030B51A4D9F
:1093A00095F8423183B00BB903B030BD04460DF1DE
:1093B000050100686CF0A6FA9DF8053083B9134AE0
:1093C000206801214FF4064482F80614A2F80444F0
:1093D000032302F20442FF2103B0BDE83040DBE585
:1093E0000DF1060296212068FFF7B2FF084ABDF88A
:1093F00006300849A2FB0323DB080122C1F808312B
:1094000085F84321DBE700BF307E0020288F002055
:10941000CDCCCCCCEC16002070B5334C05460323E4
:10942000006804F204520021FFF7ACFE60B92F4B34
:109430006FF00102C3F84C212D4AD4F808351168A9
:1094400032338B4246D370BDB4F80435274894F8C4
:1094500006C55BBA9BB207EE903AF8EEE77AF2EEF9
:10946000046A87EEA67A94F804350821BDEEC77A1F
:1094700080ED537A4FFA83FEBEF1000F4FEA4E02A1
:10948000A8BF5B0082F00702B4BFD3B2DBB20139E0
:10949000F0D194F80525082153405AB2002AB8BFEC
:1094A00052004FEA4303B6BF82F00702DBB2D3B2E9
:1094B0000139F2D19C45BFD1D0F84C312BB1D0F855
:1094C0004C214FF6FF739A42B6D14FF0FF33C0F8EC
:1094D0004C31B1E7C4F808152868064ABDE8704069
:1094E0000123312158E500BF288F0020307E002065
:1094F000503800202C94002010B5044600680379F1
:10950000012B84B02DD0022B01D0002027E08368EE
:1095100013F0010F02AA4FF0060314BF1F219F2171
:10952000FFF7D8FD0028F0D0BDF80810BDF80A20DC
:10953000BDF80C30C9BA07EE901AD2BAF8EEE76A55
:1095400007EE902ADBBAB8EEE77A07EE903AF8EE2B
:10955000E77AC4ED046A84ED057AC4ED067A04B0B6
:1095600010BD8368417C90F9100003F00103019362
:1095700002AB00931F220623FAF7BCF8D2E700BF24
:1095800010B5044600680379012B84B02DD0022B5E
:1095900001D0002027E0836813F0010F02AA4FF0EA
:1095A000060314BF2521A521FFF794FD0028F0D064
:1095B000BDF80810BDF80A20BDF80C30C9BA07EE96
:1095C000901AD2BAF8EEE76A07EE902ADBBAB8EE44
:1095D000E77A07EE903AF8EEE77AC4ED076A84ED91
:1095E000087AC4ED097A04B010BD8368417C90F913
:1095F000100003F00103019302AB00932522062320
:10960000FAF778F8D2E700BF10B500680379012BAC
:1096100084B00C4625D0022B01D000201FE08268C8
:1096200012F0010F18BF1D2103AA08BF9D21FFF7EB
:1096300051FD0028F1D0BDF80C309FED116ADFED2F
:10964000116ADBBA07EE903AB8EEE77AC7EE067A0F
:1096500077EEA67AFDEEE77A17EE903A238004B013
:1096600010BD8368417C90F9100003F00103019361
:1096700003AB00931D220223FAF73CF8D9E700BFA1
:10968000CFF7534100007A4300B500680379012BFE
:1096900085B030D0022B0BD01E4AD2F80C35D2F850
:1096A000102500201C490A610B6305B05DF804FB1E
:1096B000062302AAF721FFF70DFD0028ECD09DF844
:1096C00009309DF808C09DF80C209DF80A109DF8FF
:1096D0000BE01B0143EA0C3312019DF80DC043EA75
:1096E000111342EA0E320B4942EA1C12C1F80C3542
:1096F000C1F81025D6E78368417C90F9100002AAD2
:1097000003F00103CDE900230623F722F9F7F2FF66
:10971000D3E700BF288F0020307E002010B504461C
:1097200000680379012B84B043D0022B07D00022BC
:1097300013461046C4F83620638704B010BD836812
:1097400013F0010F02AA4FF0060314BF112191215B
:10975000FFF7C0FC0028EAD0BDF90820BDF90A30A7
:1097600006EE902A5B42BDF90C2007EE103AF8EEA7
:10977000E66AB7EE086A07EE902A66EE866AB8EEE9
:10978000C77AFDEEE66A27EE067AF8EEE77A16EE7D
:10979000903A67EE867ABDEEC77AFDEEE77AE38609
:1097A00017EE103A238717EE903A1BB2638704B086
:1097B00010BD8368417C90F9100003F00103019310
:1097C00002AB009311220623F9F794FFC2E700BF12
:1097D00010B5044600230068C4F836306387037967
:1097E000012B84B022D0022B01D000201CE0836822
:1097F00013F0010F02AA4FF0060314BF03218321C7
:10980000FFF768FC0028F0D0BDF90A30BDF8081059
:10981000BDF80C205B4201EB410103EB430302EB7B
:109820004202E1862387628704B010BD8368417CD1
:1098300090F9100003F00103019302AB009303229F
:109840000623F9F757FFDDE710B504464FF0000C8B
:109850000068C4F836C0A4F83AC00379012B84B07C
:1098600018D0022B01D0002012E0836813F0010F02
:1098700002AA4FF0060314BF61468021FFF72AFCBD
:109880000028F0D0029ABDF80C30C4F83620638767
:1098900004B010BD836890F910E0417C03F001032F
:1098A000019302AB0093624606237046F9F722FF4C
:1098B000E6E700BF10B584B00023044600680293B9
:1098C000CDF80B300279012A1ED0022A19D1836803
:1098D00013F0010F02AA4FF0070314BF4E21CE214F
:1098E000FFF7F8FBBDF80910BDF80B20BDF80D30EF
:1098F000C9BAD2BADBBA0120E1862287638704B0F5
:1099000010BD1A461946F6E7836890F910C0417CED
:1099100002AA03F00103009201934E22072360463E
:10992000F9F7E8FEDEE700BF00B500680379012B18
:1099300085B00DD0022B07D1012303AAFF21FFF729
:10994000C9FB05B05DF804FB002005B05DF804FB21
:109950008268417C90F9100002F00102019203AA92
:109960000092FF22F9F7C6FE05B05DF804FB00BFC8
:1099700030B5044600680379012B85B02DD0022B49
:109980000ED0224B6FF00102C3F80C212049214A6E
:10999000D1F8143515683233AB422CD305B030BD45
:1099A000826812F0010F18BF512103AA08BFD1210C
:1099B000FFF790FB0028E4D0BDF80C30134A5BBAE7
:1099C0009BB2C2F80C31D2F80C31B3F5C87FDDDDA3
:1099D0004FF0FF33C2F80C31D8E78368417C90F92F
:1099E000100003F00103019303AB00935122022303
:1099F000F9F780FEDEE701F20452C1F81455206841
:109A000000235121FFF7C8FA05B030BDEC16002045
:109A1000288F00205038002000B500680379012B02
:109A200085B02DD0022B24D1826812F0010F18BF0F
:109A3000002103AA08BF8021FFF74CFB1B4B83F8D2
:109A4000480198B1BDF80C305BBA9BB2B3F5FA6F20
:109A500024D2174A1749A2FB0323DB0807EE903AEA
:109A6000F8EEE77AFDEEE77AC1ED447A05B05DF8ED
:109A700004FB0E4B002283F8482105B05DF804FB7F
:109A80008368417C90F9100003AA03F00103CDE93B
:109A9000002302230022F9F72DFECFE7054B4FF0FC
:109AA000FF32C3F8102105B05DF804FB307E0020C2
:109AB000CDCCCCCCEC16002010B500680379012B7E
:109AC00084B00C461FD0022B02D0002004B010BD81
:109AD000826812F0010F18BF002103AA08BF80217D
:109AE000FFF7F8FA0028F0D05CB19DF80D309DF931
:109AF0000C20DB0903EB830302EB820203EB42033E
:109B0000238004B010BD8368417C90F9100003F0FD
:109B10000103019303AB009300220223F9F7EAFD4E
:109B2000E0E700BF70B50446234894F9103003EB1A
:109B3000830300EB8300A368D0F8CC6115469A0735
:109B40000DD530466DF046FF0123002229463046F0
:109B50006DF05AFEA3689B0716D5012070BD63699E
:109B600013B11A689B885383144B154A1B685068BD
:109B70004FEAC30C134BA3FB0C3C4FEA9C1C5368ED
:109B80001B1A9C45FBD2DCE70C4B0D491A680D4BA8
:109B90004FF4FA7000FB02F2A3FB0232486892090C
:109BA0004B681B1A9A42FBD26369002BD5D01A6806
:109BB0009B881383012070BDEC16002074390020AF
:109BC000001000E0D34D621010B50379012B82B074
:109BD0008E460DD0022B02D0002002B010BD83684B
:109BE000DB0758BF41F0800102B0BDE8104099E7A3
:109BF00014468268009402F00102417C90F9100042
:109C000001927246F9F776FD02B010BDF0B583B04F
:109C100015460DF107021C4606460F46FFF7D4FF16
:109C20009DF8072005EA0203A34201D103B0F0BD6D
:109C300022EA050222433946304603B0BDE8F0402F
:109C4000FFF788B810B582B004466A46006808215C
:109C5000FFF7BAFF9DF80030DB0602D4002002B007
:109C600010BD206806236A460021FFF78BFA002802
:109C7000F4D09DF801309DF800109DF802209FED72
:109C80004B6A1B0203EB01439DF804101C029DF874
:109C900003401A444FEA01219DF8053001EB0441CD
:109CA00048BF02F17F420B4407EE902A090248BFE9
:109CB00003F17F43B8EEE77A07EE903AF8EEE77AE1
:109CC000C7EE066A3A4BB3F94020B3F94610C7EE27
:109CD000863A07EE102A374A93ED0F6A92F8184534
:109CE000B3F94220D3ED0E7AF8EEC65A06EE102AEA
:109CF000B3F9442005EE102AB3F9482004EE901A77
:109D000004EE102AB8EEC77A112CF8EEE77AB8EE16
:109D1000C66AB8EEC55AF8EEE44AB3F94A10B3F988
:109D20004C20B8EEC44A27EE237A26EEA32A23D08D
:109D3000A6EE845AA6EEA46AE5EE265AE5EEA67AC9
:109D400077EE877AE6EE027AB3F9362007EE102A2C
:109D5000B3F93420C3ED147A06EE902AB8EEC77A30
:109D6000F8EEE66A27EE237AB6EE006AA6EE867A69
:109D700083ED157A02B010BD03EE102AF8EEC32A67
:109D800003EE101AA6EEA24AB8EEC33AA4EE265A83
:109D9000E6EE834AE5EE265AA4EEA66AE5EEA67A3A
:109DA00077EE877AE6EE027ACEE700BF00007848C9
:109DB000307E0020288F002030B5002385B0044677
:109DC000C0F8363043870DF1070200680221FFF723
:109DD000FBFE18B19DF80730DB0703D400252846A9
:109DE00005B030BD062302AA03212068FFF7CAF997
:109DF00020680DF107020921FFF7E6FE054600285D
:109E0000ECD09DF8073013F00C0FE7D1BDF8082017
:109E1000BDF80C30BDF80A102068C2EB8232C3EBEB
:109E200083339B0092008900E286218763870122A9
:109E30000A21FEF78FFF284605B030BD2DE9F0411D
:109E40004D4F97F8403182B043B14C4E96F81955BA
:109E5000012D04463BD0022D5AD015B102B0BDE809
:109E6000F081012280210068FEF774FF2068012242
:109E7000FF21FEF76FFF2A4629462068FEF76AFF9A
:109E800096F81A2520689121FEF764FF294620687C
:109E90000122FEF75FFF2A462068FF21FEF75AFFE6
:109EA0002A4620688021FEF755FF294620680122B6
:109EB000FEF750FF324B33491A6881F80001012345
:109EC000C6F81C2586F8193502B0BDE8F08101AA54
:109ED0000068DFF8B0800021FFF776FE9DF80430BF
:109EE00088F80001DA073ED5D6F82035002BB5D02A
:109EF000234AD6F81C15126892B2521A9342ADD278
:109F00004FF0FF320023C8F8042186F81935A5E781
:109F10000068DFF8708001AA1321FFF755FE9DF855
:109F2000043088F800015B07DED020682B4601AAC8
:109F30001E21FFF727F9BDF80430206801220B210C
:109F40005CBAFEF707FF104B88F80001A4B2A3FB30
:109F50000434E40801220023C8F8044187F84121B1
:109F600086F819357AE7064A02231268C6F81C25D6
:109F700086F8193572E700BF307E0020288F002058
:109F800050380020EC160020CDCCCCCC30B50446A7
:109F900000680379012B85B062D0022B03D0002525
:109FA000284605B030BD826802AD12F0010F18BF1F
:109FB00019462A4608BF8221FFF7B4FD0028EED0DB
:109FC0009DF80830DA07EAD52A46206807230321DE
:109FD000FFF7D8F805460028E1D0206811220A21B1
:109FE000FEF7B8FE9DF80E301B07D8D42A49BDF8FD
:109FF0000830B1F8242513FB02F3284A93423FDBD3
:10A00000B3F5000F3ADA002BB8BFFF331B125B42E7
:10A010001BB2BDF80A20E386B1F8263512FB03F324
:10A020001E4A934230DBB3F5000F31DA002BB8BF84
:10A03000FF3343F30F22BDF80C30B1F82815228707
:10A04000164A13FB01F393421CDBB3F5000F1DDA34
:10A05000002BB8BFFF331B125B421BB263879FE725
:10A06000826890F910C0417C02F0010202AD0192B9
:10A07000009560460222F9F73DFB9FE7084BC8E7D1
:10A08000084BC6E7074BE9E7064AD4E7044BE5E788
:10A0900047F6FF72CFE700BF288F002001FF7FFF48
:10A0A0000180FFFF0080FFFF10B5044686B0006806
:10A0B00000238DF80F300379012B31D0022B02D011
:10A0C000002006B010BD8368D9070DF10F024CBF08
:10A0D0002721A721FFF726FD0028F1D09DF80F309A
:10A0E0001B07EDD52068062304AA2821FFF74AF8AC
:10A0F00028B3BDF91030BDF91220002BB8BF0333CF
:10A100009B10E386BDF91430002AB8BF0332002B40
:10A11000B8BF033392109B102287638706B010BD2F
:10A12000826890F910C0417C02F0010201920DF1A9
:10A130000F02009260462722F9F7DCFACCE7C4F858
:10A14000360060870020BCE730B504464FF0000CB5
:10A150000068C4F836C0A4F83AC00379012B87B070
:10A160002AD0022B02D0002007B030BD8368D90767
:10A170000DF10F024CBF61468021FFF7D3FC002890
:10A18000F1D09DF80F301B07EDD52068062304AAF7
:10A190000121FEF7F7FF0028E5D0BDF81430BDF827
:10A1A0001010BDF812205BBA49BA52BA5B42E18680
:10A1B0002287638707B030BD8568417C90F9100025
:10A1C00005F0010501950DF10F0562460095F9F7BF
:10A1D00091FAD4E710B5044600230068C4F836307D
:10A1E00063870379012B86B023D0022B02D0002095
:10A1F00006B010BD8368D9070DF10F024CBF0621D0
:10A200008621FFF78FFC0028F1D09DF80F305B0707
:10A21000EDD52068062304AA0021FEF7B3FF00282D
:10A22000E5D0049ABDF81430C4F83620638706B030
:10A2300010BD826890F910C0417C02F001020192C9
:10A240000DF10F02009260460622F9F753FADAE7A1
:10A2500010B5044600230068C4F8363063870379DC
:10A26000012B86B012D0022B0DD18368DB070DF1D4
:10A270000B024CBF3421B421FFF754FC18B19DF9F7
:10A280000B30002B11DB002006B010BD826890F966
:10A2900010C0417C02F0010201920DF10B0200920C
:10A2A00060463422F9F726FAE8E72068092303AA72
:10A2B0002421FEF767FF0028E5D09DF810209DF8C7
:10A2C0000F109DF81330120442EA0162C2F30F42EC
:10A2D0009DF8121022871B049DF80D2043EA0163AC
:10A2E0009DF80C10120442EA0162C2F30F42C3F35C
:10A2F0000F43E286638706B010BD00BF2DE9F04131
:10A30000DFF8BC802C4E2D4D41F0010284B00021BD
:10A310000446FEF71FFDD8F80070C6F81C7519E05A
:10A32000022B3FD1A368DB070DF10F024FF01301A1
:10A3300020465EBF0DF10F0293212046FFF7F2FB8E
:10A340009DF80F3085F8000113F0070319D1D6F8F6
:10A3500020254ABB2379012BE2D1A268617C94F9C4
:10A36000100002F0010201920DF10F02009213227F
:10A37000F9F7C0F99DF80F3085F8000113F00703D5
:10A38000E5D001220B212046FEF7E4FC0022114615
:10A390002046FEF7DFFC012385F80001184604B0D3
:10A3A000BDE8F0810020CBE7D8F8001089B2C91BC6
:10A3B0008A42CFD2F2E700BF288F0020EC1600209F
:10A3C0005038002010B50368DA6B82B0044612B131
:10A3D000904740B123685B6B1BB1214601A89847A9
:10A3E00018B9FF23E38202B010BDBDF80630013B6F
:10A3F0009BB2F7E7F0B5044683B018460D46164603
:10A400001F4676F05DFB2844D4F800C0A073E673C5
:10A41000204600240094DCF814403B46324629468E
:10A42000A04703B0F0BD00BF38B58B68016004469B
:10A430000D46984700230B4A226123752B6B13B1FD
:10A44000204698472075084B93F82C351BB1237D87
:10A4500023F0010323750023E3822046BDE8384042
:10A46000B0E700BF0001FF00288F002010B5154B9A
:10A47000D3F8304584B084B12379012B10D0022B5E
:10A480000BD1A16811F00101024618BF80212046BE
:10A4900004B0BDE81040FEF707BC002004B010BDBA
:10A4A000A268617C8DF80F0002F0010294F910009F
:10A4B0000DF10F04CDE900428022F9F737FD04B019
:10A4C00010BD00BF288F0020F0B5294BD3F83055C0
:10A4D00085B09DB1B02280212846FEF73BFC40228A
:10A4E00080212846FEF736FC002280212846FEF710
:10A4F00031FC102280212846FEF72CFC4FF48064AA
:10A500002DB9013CA4B2002CFBD105B0F0BD002751
:10A510000DF10F062B79012B08D0022B04F1FF322D
:10A5200017D094B2002CF0D0012BF6D1AA6895F97F
:10A530001000697C8DF80F7002F00102013CCDE93A
:10A540000062A4B24022F9F7F1FC002CE2D105B080
:10A55000F0BDAA68013C12F0010218BF00224021A0
:10A560002846A4B2FEF7A0FB002CD3D105B0F0BD65
:10A57000288F00200B4B10B5D3F830458CB15038E4
:10A58000C2B280212046FEF7E5FB00228021204652
:10A59000FEF7E0FB20461022BDE810408021FEF7C8
:10A5A000D9BB10BD288F0020F0B5264B264CD3F820
:10A5B0003055203800EB8000661D85B00444064409
:10A5C00025B90134A642FCD105B0F0BD0DF10F074D
:10A5D0002B792278012B1BD0022B0AD00134A64202
:10A5E000F7D100224021284605B0BDE8F040FEF733
:10A5F000B1BBAB68DB074FF04001284619D50134E9
:10A60000FEF752FBA642E3D1002DEAD105B0F0BD22
:10A610008DF80F20AA6895F91000697C02F00102FC
:10A62000CDE9007201344022F9F780FCB442CFD169
:10A63000D7E70134FEF738FBB442C9D1002DE5D08D
:10A64000CFE700BF288F002088320808F0B5754B8F
:10A65000D3F8305585B0002D00F09680D4228021AB
:10A660002846FEF777FB802211462846FEF772FB4C
:10A67000A82280212846FEF76DFB3F228021284634
:10A68000FEF768FBD32280212846FEF763FB0022F9
:10A6900080212846FEF75EFB402280212846FEF7F7
:10A6A00059FB8D2280212846FEF754FB142280217D
:10A6B0002846FEF74FFBA12280212846FEF74AFBE1
:10A6C000C82280212846FEF745FBDA228021284651
:10A6D000FEF740FB122280212846FEF73BFB812239
:10A6E00080212846FEF736FBCF2280212846FEF740
:10A6F00031FBD92280212846FEF72CFBF122802154
:10A700002846FEF727FBDB2280212846FEF722FBA6
:10A71000402280212846FEF71DFBA42280212846E6
:10A72000FEF718FBA62280212846FEF713FBAF2276
:10A7300080212846FEF70EFBA62280212846FEF740
:10A7400009FBAE2280212846FEF704FB202280214F
:10A750002846FEF7FFFA002280212846FEF7FAFA83
:10A76000B02280212846FEF7F5FA402280212846B3
:10A77000FEF7F0FA002280212846FEF7EBFA1022BD
:10A7800080212846FEF7E6FA4FF4806435B9013C93
:10A79000A4B2002CFBD1012005B0F0BD00270DF1C3
:10A7A0000F062B79012B2AD0022B04F1FF3214D093
:10A7B00094B2002CF6D1812280212846FEF7CAFAF5
:10A7C000C82280212846FEF7C5FAAF2280212846FC
:10A7D000FEF7C0FA012005B0F0BDAA68013C12F0F6
:10A7E000010218BF002240212846A4B2FEF75CFAFD
:10A7F000002CD6D1002DDED1012005B0F0BDAA6815
:10A8000095F91000697C8DF80F7002F00102013C8F
:10A81000CDE90062A4B24022F9F788FB002CC0D138
:10A82000C9E700BF288F0020FDF7F4BFFDF7F2BF96
:10A83000FDF7F0BFFDF7EEBFFDF7ECBFFDF7EABF98
:10A8400038B52B4C2B483622002174F081F8D4F80F
:10A8500020320020984728B9D4F844329847012183
:10A8600008B938BD002124204A42234B234D024021
:10A8700000FB01441344C5F86C35D4F840229047DE
:10A88000836853B305F2345C048862466146002352
:10A890000878032801F1060121D00133092BF7D1F3
:10A8A000601E80B200231178022902F1060209D04D
:10A8B0000133092BF7D1D5F87035082B0DD05A1C70
:10A8C000C5F87025062202FB03CC022200238CF877
:10A8D0000020ACF80230ACF80400012038BD06219D
:10A8E00001FB0353B3F83605013880B2DAE700BF45
:10A8F000EC1600205C9400200C190020288F00200A
:10A9000001207047034620B1026812B1D26902B13A
:10A91000104793ED017A084BB8EEC77AD3ED016A80
:10A92000F6EE007AE7EE267AFDEEE77A17EE900A69
:10A9300000F30B00704700BF9C940020034620B139
:10A94000026812B1126A02B1104793ED027A084B05
:10A95000B8EEC77AD3ED026AF6EE007AE7EE267A11
:10A96000FDEEE77A17EE900A00F30B00704700BF88
:10A970009C940020034628B102681AB1516A09B1BB
:10A980009369184793ED037A074BB8EEC77AD3ED76
:10A99000036AF6EE007AE7EE267AFDEEE77A17EE26
:10A9A000900A00F30B0070479C94002038B504090E
:10A9B000013C042C1CD8104D05EB440200F00F03A1
:10A9C000B2F8BC0240FA03F212F0010212D00122E6
:10A9D00002FA03F3013B1840254477F011F895F88B
:10A9E000C832064A184400EB400002EB800038BD34
:10A9F000002038BD104638BD70320808482C0020B1
:10AA00002DE9F04F542204460021BE4895B073F062
:10AA10009FFFBD49621EE01C0C4612F8013F5D1EFF
:10AA2000052D88BF0023904244F8043BF5D1B74A76
:10AA3000A2F1100353F8040B012800F059819A4247
:10AA4000F8D151F8043B022B00F048819142F8D133
:10AA50000320FCF767FA0420FCF764FA0520FCF7F2
:10AA600061FA0620AA4FA74DFCF75CFA1A264FF0B0
:10AA7000000BA7F5347A2C7B002C41D02046FFF741
:10AA800095FF95F90D800246002800F0FF80D0F870
:10AA90000090C6710523837109F13F4303F57E03DE
:10AAA0000AEB9323CDE9022A187C0023137269F084
:10AAB00067FB029A928800231146012200924846C1
:10AAC000019303226CF060FC002317F83320A242AC
:10AAD0002ED00133102BF8D100218E4B296108EBC9
:10AAE000480803EBC8080122D8F87C322B751344C0
:10AAF000C8F87C320723AB756A7588F878229344CE
:10AB00000136F6B2202E05F10C05B4D1BBF1000FD1
:10AB10000BD0814D814F00262B7C7BB90136032E53
:10AB200005F1180507F58C77F6D115B0BDE8F08F63
:10AB3000039A02EBC309D9F8D412CEE7687969F019
:10AB40001FFB287969F01CFBD5F808904846F7F7F9
:10AB500041FFD5F814802C680797142303FB08F3F2
:10AB600009930023CDE91033CDE9123308930A93FA
:10AB7000EB68059304F14C034FF4806206934FF4A5
:10AB80000063CDE90B234FF400514FF48073CDE9FE
:10AB90000D1348464FF4003305A90F9369F0C4FA2A
:10ABA000D9F800205E495F4B42F00102C9F800204D
:10ABB0004A68134043F440334B606268B8F1010FB8
:10ABC00022F04072D4BF0023012322F4807242EAB3
:10ABD00003226260A168544A0A4042F00202A26065
:10ABE000E26A08F1FF33DBB222F4700242EA035357
:10ABF000E362444B4FF0010C03F148004FFA86FE2C
:10AC000002E00C33834230D05A7D002AF9D093F908
:10AC10000D207245F5D11A7C997D092A39D8D4F8CE
:10AC2000108002EB420A4FF0070909FA0AF901FA0B
:10AC30000AF128EA090841EA08012161BCF1060F7E
:10AC400039D80CF1FF31D4F8348001EB81014FF099
:10AC50001F098A4009FA01F128EA01010A436263E7
:10AC60000CF1010C5FFA8CFCCBE7A36843F4007392
:10AC7000A360A36843F48073A360A36843F0010357
:10AC8000A360A36843F08043A36047E7274B039387
:10AC90001AE7A2F10A08D4F80C9008EB48084FF024
:10ACA000070A01FA08F10AFA08F829EA080841EA4D
:10ACB0000801E160C2E7BCF10C0F3BD8ACF1070121
:10ACC000D4F8308001EB81014FF01F098A4009FA66
:10ACD00001F128EA01010A432263C1E7144B93F80A
:10ACE000B8202121013283F87C1083F8B820AFE628
:10ACF0000F4B93F8B8002024013083F8704083F89C
:10AD0000B8009EE68C8F0020307E0020407E002020
:10AD100040350808EC16002054190020E48F00206C
:10AD200000230140E030FCFFFDF7FFC0703208084F
:10AD3000288F0020ACF10D01D4F82C8001EB8101AB
:10AD40004FF01F098A4009FA01F128EA01010A437C
:10AD5000E26285E710B503681A79022A044603D037
:10AD600000232371236010BD987AFFF71FFE00288F
:10AD7000F6D040F61A610022C18002722021FDF750
:10AD8000F7FE00232371236010BD00BFF0B50668F5
:10AD9000194B144606F13F4202F57E0203EB922363
:10ADA000074683B0187C0D4669F0EAF9B988B1FA14
:10ADB00081F3C3F11F03C3F3CC0206EB820203F05D
:10ADC000070330469B00166A0F279C4007FA03F3DF
:10ADD00026EA03031362136A1C431462C5F30013CB
:10ADE0006A09CDE90032C5F3810305F003026CF076
:10ADF000CBFA03B0F0BD00BF703208082DE9F04F68
:10AE0000B44EB54CA64285B057D21D4602E00C3672
:10AE1000A64252D273798B42F9D13379834201D061
:10AE20000028F4D1F3799342F1D13468002C44D056
:10AE300000236360A360E36023616361A361E36156
:10AE400026603379237196F80690C4F80890327A18
:10AE5000E260012B33D0022B2FD1F07AFFF7A6FD51
:10AE600096F90970A061B07A2774FFF79FFD064636
:10AE70006061F8B1DFF880A207EB87030AEB830378
:10AE8000BA00D3F8CC810092B8F1000F12D093F839
:10AE9000DE21EAB10E220023F2713372B57109216D
:10AEA0003046FDF765FE3368B2881A83204605B048
:10AEB000BDE8F08F2046FFF74DFF0024F6E7F07A5B
:10AEC000FFF774FD727AB37A6374A0612274EDE7C0
:10AED00093F8D4B1584669F053F94FEA5B12012355
:10AEE0000BF01F0B023A03FA0BF3032A08D8DFE832
:10AEF00002F0ADA7B30279494A6922EA03034B6124
:10AF0000BB003B440AEB830393F8D101FFF74EFDEE
:10AF1000791C0246C9B218B140F60A330172C380E7
:10AF2000BB003B440AEB8303CDE9002193F8D30136
:10AF3000FFF73CFDDDE90021834620B1017240F6B8
:10AF40000A50ABF8060009F004030093BB0003EBC2
:10AF500007090AEB8909CDE9022199F8D201FFF727
:10AF600025FDDDE9022199F8D5910190002800F036
:10AF7000D580019B197240F60A41D980009B002BB5
:10AF800070D0002A00F0C58010464A214A46FFF7DB
:10AF9000FDFEBBF1000F04D058464A462A21FFF7B8
:10AFA000F5FE01984A460A21FFF7F0FEBB003B443C
:10AFB0000AEB830393F8D0B1BBF1000F6AD1484B81
:10AFC000984571D0474B984500F09880464B98457E
:10AFD00075D0464B984500F0BE80454B984500F033
:10AFE000AF80444B984500F0D180009BB8F800201A
:10AFF000002B02F441520CBF03230023134343F4FC
:10B000004573A8F80030B8F81C3023F400631B0423
:10B010001B0CA8F81C300723A8F81030B8F8003033
:10B020009BB243F04003A8F80030BBF1000F28D1D9
:10B03000BB003B440AEB8303012283F8DE2129E7AE
:10B0400026490A6A22EA03030B6259E723494A6A3E
:10B0500022EA03034B6253E720490A6922EA030309
:10B060000B614DE722B110460A214A46FFF78EFEDA
:10B07000BBF1000F95D058464A460A21FFF786FEDD
:10B080008FE75846FFF792FC0028D1D002688388EA
:10B090001383CDE75846FFF789FC00288FD04A4636
:10B0A0000921FFF773FE8AE703F584335A6A42F4F5
:10B0B00080525A625A6A22F480525A6295E703F526
:10B0C000FE331A6A42F400421A621A6A22F40042FB
:10B0D0001A628AE700610908B06209080038024074
:10B0E0000030014000380040003C00400034014086
:10B0F0000050014000540140EC16002003F50033DD
:10B100001A6A42F480421A621A6A22F480421A626F
:10B110006BE7BBF1000F7FF43FAF42E7009B2BB31F
:10B1200022B110464A214A46FFF730FEBBF1000F1C
:10B130003FF43CAF58464A462A21FFF727FE35E741
:10B1400003F568435A6A42F480125A625A6A22F43A
:10B1500080125A6249E703F582335A6A42F4005278
:10B160005A625A6A22F400525A623EE7CAB1104645
:10B170000A214A46FFF70AFEBBF1000F3FF416AF63
:10B1800058464A460A21FFF701FE0FE703F56443DC
:10B190005A6A42F400125A625A6A22F400125A623F
:10B1A00023E7BBF1000FEBD100E700BF2DE9F04F23
:10B1B00085B007460093BDF8383002939DF83C30C7
:10B1C00001938A469146FAF761FD002800F08181DB
:10B1D000C14E96F884450B2C00F276815C2202FB6E
:10B1E00004620021C2F8881582F88C15621C04EBF9
:10B1F0004401D2B2C4EBC101804606F5B16B387987
:10B2000086F8842503920BEB810BFFF7CFFB0546F5
:10B2100028B1039A0272022280F806A0C2715C2053
:10B2200000FB04600099C0F888854A464046F7F75D
:10B2300005FAD8F804309A7902F00201003918BFF3
:10B24000012112F0040210D149004FF4807C914694
:10B250004FF0010E58791B68032800F26F81DFE878
:10B2600010F0E500A2005F000C004FF0000C4A0057
:10B270004FF004096146E646ECE71A8C22F480524E
:10B280001204120C1A841A8C988822F400521204A8
:10B290004EEA010E120C42EA0E319A8BDFF840E2C0
:10B2A00022F4E6421204120C734580B242F4C0420A
:10B2B00000F025810EF5806E734500F020819880A6
:10B2C0009A83029A1A6419849A8B22F400621204F7
:10B2D000120C42F400629A83B3F844206FEA4242AF
:10B2E0006FEA524292B2A3F844201A8892B242F016
:10B2F000010223F8402B5C2202FB04660022C6F800
:10B3000090351A60019B002B00F0D08025B13A7A6D
:10B3100002212846FFF73AFD584605B0BDE8F08FF8
:10B320004EEA0100198C21F480710904090C19847A
:10B33000198C21F400710904090C41EA0021988854
:10B34000B3F81CE02EF0730E4FEA0E4E4FEA1E4E7D
:10B350004EF06008DFF888E1734580B200F0C280EB
:10B360000EF5806E734500F0BD80029A9880A3F8B8
:10B370001C80DA6319849A8B22F008021204120CE2
:10B3800042F008029A83B3F844206FEA42426FEA1F
:10B39000524292B2A3F844201A8892B242F00102BB
:10B3A00023F83C2BA7E74EEA0100198C21F010018D
:10B3B0000904090C1984198C21F020010904090CD5
:10B3C00041EA00119888B3F818E02EF4E64E4FEAEF
:10B3D0000E4E4FEA1E4E4EF4C048DFF804E17345AE
:10B3E00080B200F09E800EF5806E734500F099806B
:10B3F000029A9880A3F818809A6319841A8B22F411
:10B4000000621204120C42F400621A83B3F8442062
:10B410006FEA42426FEA524292B2A3F844201A887D
:10B4200092B242F0010223F8382B64E74EEA0100A1
:10B43000198C21F001010904090C1984198C21F0DF
:10B4400002010904090C01439888B3F818E02EF0B2
:10B45000730E4FEA0E4E4FEA1E4E4EF06008DFF8B4
:10B4600080E0734580B24FD00EF5806E73454BD0AF
:10B47000029A9880A3F818805A6319841A8B22F0D4
:10B4800008021204120C42F008021A83B3F8442096
:10B490006FEA42426FEA524292B2A3F844201A88FD
:10B4A00092B242F0010223F8342B24E711212846FE
:10B4B000FDF75EFB002D3FF42FAF2B68AA885A835F
:10B4C000584605B0BDE8F08F044A00210420FAF781
:10B4D0002DFB4FF0000B1FE7288F00201CE408080D
:10B4E0000000014021F4006141EA022121F4806161
:10B4F00020F4405041EA092140EA0C1035E720F4DD
:10B50000804040EA8C10DAE620F440704CEA0000FB
:10B510004FF6F37C01EA0C0C4CEA020C49EA0C01F0
:10B52000A6E721F0800141EA021121F0400120F458
:10B53000406041EA091140EA8C0059E7B3F8442021
:10B540006FEA42426FEA524292B2A3F844201A884C
:10B550005C20002100FB046092B242F001021A80DC
:10B56000C0F890150960FFDE30B50368284D294CFE
:10B570002DED028BAB42246883B0F0EE408AB0EE32
:10B58000608A10D005F58065AB420CD005F570558A
:10B59000AB4208D005F58065AB4204D005F5806567
:10B5A000AB4218BF6408B4FBF1F303F57F43FF33EC
:10B5B0001B0CB4FBF3F40023B4FBF1F501920093F0
:10B5C0002246ABB20221FFF7F1FDE0B1B5EE408AB1
:10B5D00007EE904AF1EE10FAF8EE677A0ABF07EE2E
:10B5E000105A28EE278AB8EE478A9FED0B7AC8EEEC
:10B5F000076A0123037127EE667AC0ED046AA8EE9C
:10B60000A77A80ED037A03B0BDEC028B30BD00BF9A
:10B6100000000140300C002000007A44074B53F832
:10B62000203021B14BB11A689B8853837047002B9F
:10B63000FCD01A689B8813837047704764320808EF
:10B640002DE9F04F864FA7B000210A260C4607F6D9
:10B65000D8154FF0050B01968BE0BAF1000F19D108
:10B6600043F04003BEF18C0F87F8DC3D00F2E4802C
:10B6700004F1010C98340DEB040A0CF198040DEB65
:10B68000040C74464FF0040E0AF88CEC0CF88C3C59
:10B6900004F1020EBEF18C0F42F0020C00F2CC80DD
:10B6A00004F198036B4403F88BCC04F1040CBCF157
:10B6B0008C0F03F88CBC00F2BF800EF198060DEBE6
:10B6C000060E4FF0060A0EF88CAC04EB0A0E4FEA99
:10B6D0008909BEF18C0F5FFA89F603F8890C00F234
:10B6E000AB8004F19C0CEC444FF007090CF88C9CE7
:10B6F00004F1080CBCF18C0F03F8876C00F29C80FD
:10B700000EF198060DEB060E0EF88CBC03F8852C96
:10B7100004F10A028C2A00F28F8004F1A0060DEBDE
:10B72000060C0CF88CAC03F8830C04F10C008C288C
:10B7300000F2828004F1A20204F1A3036A446B4484
:10B7400002F88C9C044603F88C8C480901F01F0C0D
:10B7500055F82030012202FA0CF223EA020345F8E0
:10B760002030019B013B01936ED00131B1F5F07F98
:10B770006AD23C222846F9F7ABFC011E5FDB07EBDF
:10B78000410297F8DC3DB2F814CA1CF0040FC1F373
:10B790000722C8B25FFA8CF94FEA1C2803F0400A6E
:10B7A00004F1020E7FF459AFBAF1000F03D103F098
:10B7B000380CCC4519D003F0870343EA0903BEF1E6
:10B7C0008C0F87F8DC3D37D804F1010C0CF198069A
:10B7D00098346C440DEB060C4FF0040904F88C9C73
:10B7E00074460CF88C3C0EF1020EBEF18C0F23D87F
:10B7F00004F198030DEB030C231D8C2B0CF88B2C00
:10B800000CF88CBC18D80EF198020DEB020E062233
:10B810000EF88C2C0CF8890CA0188C280CD804F18C
:10B820009C0304F19D026B446A44072403F88C4C8A
:10B83000044602F88C8C88E76FF0004485E72046C8
:10B8400014B927B0BDE8F08FD7F8D40D234603AA6A
:10B8500000216CF077F8012027B0BDE8F08F00BF21
:10B86000288F0020F0B5284CD4F8D40D83B010B147
:10B8700094F8DA3D0BB103B0F0BD01230DF10702DE
:10B88000842184F8DA3DFEF79FF994F8DC2DD4F892
:10B89000D40D04210A43FDF75DFAD4F8D40D0DF15F
:10B8A00007028421FEF790F99DF8073013F0040693
:10B8B000F3D1164D84F8DC3D3C223146284673F026
:10B8C00047F83246124E05F13A0005F2FA374FF0CA
:10B8D000010E30F8023F334002F01F019BB24FEAE5
:10B8E000521C0EFA01F1013223B155F82C300B43F2
:10B8F00045F82C30B842ECD1FFF7A2FE0028FBD16E
:10B9000084F8DA0D03B0F0BD288F002000990020E4
:10B9100004DFFFFF70B5414DD5F8D44D82B09CB324
:10B9200095F8D83D012B43D0022B2FD1082194F953
:10B9300010303B4A85F8DB1D03EB830302EB8303E6
:10B94000A2688DF80510002040F2044192078DF89E
:10B950000400ADF80610D3F8CC0142D504230DEB5A
:10B96000030200216BF050FFA3689B0722D52D48EE
:10B970003C22FF2172F0ECFF95F8D93D23B9FFF787
:10B9800071FF012385F8D93D02B070BD0DF10302AE
:10B99000A0212046FEF718F99DF8033003F00503B7
:10B9A000012B37D0002B2FD1D5F8D44D0821BEE77D
:10B9B0004821BCE71C4B1D491A681D4B48684FF4D1
:10B9C000FA7606FB02F2A3FB023292094B681B1ABD
:10B9D0009A42FBD26369002BC9D01A689B881383F3
:10B9E000C5E7636913B11A689B8853830E4B0F49EF
:10B9F0001A680F4B4E68D200A3FB023292094B68C3
:10BA00009B1B9A42FBD2A9E70A4A126840F2DC5318
:10BA10009A42B9D9D5F8D44D482188E7288F00201B
:10BA2000EC1600200099002074390020001000E07E
:10BA3000D34D6210503800202DE9F041334D95F878
:10BA4000DA3D82B003B1FEE7012285F8DA2D95F8E0
:10BA5000DB2D044602F0F702D5F8D40D85F8DB2D76
:10BA60000E461946FDF776F9E2B207460921D5F8E8
:10BA7000D40DFDF76FF9B4F5807F3FD0D5F8D40D24
:10BA8000DFF88C8050220821FDF764F9D5F8D40D39
:10BA90000DF10702A021FEF797F848B9D8F88C31CC
:10BAA000B8F8902159690A4214BF5A831A83EDE706
:10BAB0009DF8074014F02004F0D1E2B20A21D5F835
:10BAC000D40DFDF747F93219D5F8D40DC021013452
:10BAD000FEF77AF8362CF0D157B995F8DB2DD5F86A
:10BAE000D40D02F0F702394685F8DB2DFDF732F967
:10BAF000002385F8DA3D02B0BDE8F081D5F8D40D19
:10BB000040220A21FDF726F9B8E700BF288F002060
:10BB1000482C00202DE9F04F604D95F8DA7DC3B038
:10BB200007B1FEE795F8DB2D044602F0F70201238A
:10BB3000D5F8D40D85F8DB2D0E46394685F8DA3D6B
:10BB4000FDF708F9FF2C4FF009038DF8054088BF79
:10BB5000A40801AA8CBF04F0C008B84602204FF028
:10BB6000000C4FF00A0B0DF1050A4FF00B09137092
:10BB700014E0B1F5827F02F800B00AF8003016F840
:10BB80000C3017D80CF1010CBCF1360F02F80790FD
:10BB900004F1060402F80E30084614D0871C48EA67
:10BBA0000C03B7F5827F00F104010446DBB200F11B
:10BBB000030EDED90CF1010C6FF00041BCF1360F21
:10BBC000374C0846EAD1B4F5827F63D80823535432
:10BBD0000DF10503A0211954831CD5F8D44D314E25
:10BBE00094F9101001EB810106EB8101D1F8CC0131
:10BBF000A168890722D500216BF006FEA3689B0788
:10BC000031D5294CD5F8D40D0DF10302A021FDF753
:10BC1000DBFF48B9D4F88C31B4F8902159690A4255
:10BC200014BF5A831A83EDE79DF8033013F0200305
:10BC3000F0D185F8DA3D43B0BDE8F08F616911B10C
:10BC40000E68898871831949194F0E681949D7F808
:10BC500004C0F600A1FB0616B6097968A1EB0C0139
:10BC60008E42FAD2C7E7114B11491A68114B486846
:10BC70004FF4FA7606FB02F2A3FB023292094B68FC
:10BC80001B1A9A42FBD26369002BBAD01A689B88B0
:10BC90001383B6E76FF000439FE700BF288F0020B3
:10BCA00001000080EC160020482C00207439002090
:10BCB000001000E0D34D621038B5837913F0010F06
:10BCC000044603F02002C36B406B1FD0002A5D685E
:10BCD0000CBF4221022110B12A7AFFF757F8012345
:10BCE00084F86032A4F85C326A790C482968104400
:10BCF0000A8C90F8500383409BB292B222EA03026E
:10BD00000A840A8C92B213430B8438BD002A5D6802
:10BD10000CBF222102210028DED1E0E770320808A2
:10BD2000F8B583681C686579A80744D4ED0700D48A
:10BD3000F8BD94F85C32002BFAD194F85D320133EF
:10BD4000DBB2092B84F85D3277D00A2BF0D194F85E
:10BD50005F52B4F86632002D00F08D80980502D451
:10BD6000DA0700F1F580B4F86A320133A4F86A32D8
:10BD700001239D42A4F85C32DAD1E66BA17900235D
:10BD800084F85F3201F00101304668F043F97268CF
:10BD9000764B5079116803440A8C93F8503305FAB6
:10BDA00003F39BB292B222EA03020A840A8C92B293
:10BDB00013430B84F8BD94F86112002934D1A26AB0
:10BDC000636A94F86002934200F09180531CA66964
:10BDD000A362B65C2269A779934228BF002376004C
:10BDE000A3620A2346F4007684F862320123A4F8A1
:10BDF000646284F8613208B13A074CD47B0695D569
:10BE00000922402087EA06037608A4F86462DE0768
:10BE1000A16B2AD411B10B688988598384F86222F6
:10BE2000002883D02AB181E794F96222002A40F0E9
:10BE30009580002384F8613278E794F85F32002B14
:10BE40007FF476AF94F85E32082B3FF671AFB4F80A
:10BE50006622012000FA03F101330A43D9B208290E
:10BE600092B2F7D9A4F86622F8BD0029D6D00B68A3
:10BE700089881983D2E743F001009905A4F8660286
:10BE80004AD4E36A4008002B53D0216BC0B29847D4
:10BE900094F85F526CE7E26BD2F804E0334A9EF804
:10BEA0000500DEF800C00244606B92F85023934016
:10BEB000BCF8202092B222EA0303ACF82030BCF890
:10BEC00020309BB2ACF8203018B19EF80820FEF765
:10BED0005DFF002384F86032236CA06B2BB35B689A
:10BEE0001A7A00288AD00121FEF750FF86E7002841
:10BEF0007FF41CAFA37919077FF518AF216CA36BF2
:10BF000041B32BB14A680146127A1846FEF73EFF4C
:10BF10002046FFF7D1FE09E7B4F86A320122134444
:10BF2000A4F85C22A4F86A32F8BD0121FCF720FED7
:10BF300064E7E3696269C0B2D054E369E26894F8E7
:10BF40005F520133B3FBF2F102FB1133E3610FE700
:10BF5000184696E71846FCF70BFED9E7A779B4F820
:10BF60006462013A07F0400052B24BE770320808B1
:10BF700038B504464068304B0568304A9D42126827
:10BF8000084610D003F580639D420CD003F5705332
:10BF90009D4208D003F580639D4204D003F5806381
:10BFA0009D4218BF52081346B3FBF0F1B1F5803F34
:10BFB0000FD289B22046F6F741FB23681A685379FD
:10BFC000DBB993794BB92B889BB243F001032B80EB
:10BFD00038BD012BEAD95B08E6E71A061ED41849DA
:10BFE000CA18302082F800035809012203F01F0309
:10BFF00002FA03F341F82030E5E7190615D410489A
:10C000005C0900EB030C012103F01F0301FA03F3A9
:10C0100030218CF8001340F82430D2E7094A03F0AD
:10C020000F031A4430231376CDE7064903F00F03BC
:10C03000194430230B76C4E700000140300C002087
:10C0400000E100E0FCEC00E00346C06B99608FE784
:10C05000002ABCBF80185242002B30B503EB01050B
:10C0600003DA0C465B42294625460028B7BF121A60
:10C07000841814460020A4F11D0C0029BCBF2B46D7
:10C080000021BCF1000FC4BFA2EB0C021418A5F1F3
:10C090000F02002AC4BF9B1A5D1884421EDBC1F147
:10C0A000010C0F4AAC44C1EB0113CCEB0C1C00EBB0
:10C0B000430301344FEA4C0C02EB43024FF0200ED5
:10C0C0008D42A8BF002304DB22F813E01E339C45F9
:10C0D000FAD10130A04202F10202F1D130BD00BF1D
:10C0E0003C9900201B4B1C48196C1C4A10B441F0B1
:10C0F00080510124196404625321FF24CA20546230
:10C10000506251625B6FDB0085B013D40023144989
:10C1100002930291029A134804320292029A136027
:10C1200003930391039B0393039B186005B05DF891
:10C13000044B70470A4B002201920193019B01932B
:10C14000019A084B12689A42E0D105B05DF8044BA1
:10C15000704700BF0038024000000E420028004037
:10C160005028004076614E692DE9F04F2DED028B8D
:10C17000AC4BAD4E1B78AD4DDFF8D0A2B1B000276F
:10C180000293B146BB46A6F11008D9F8004000233F
:10C1900055F83320944203D001330E2BF8D1FF23FE
:10C1A000534493F8E03D022B00F0BD80032B00F0D8
:10C1B000B180012B09D1D9F80C3023F0807323F022
:10C1C000080343F00403C9F80C304846FBF7F2F8C3
:10C1D00048B90BEB8B0308EB8303D96901F00C031F
:10C1E000042B00F0AB800BF1010BBBF10C0F09F13C
:10C1F0001409CAD1DDF8088006F1F005344608E0DC
:10C200002068E260FBF7D6F94844C7B21434A5426F
:10C210001FD02046FBF7CEF80028F7D1E368590776
:10C2200003F00C02F2D5042AF0D023F0080242F009
:10C230000402781CB84511465FFA80F923F0040324
:10C24000DED82068E36019461434FBF7B3F9A54241
:10C25000DFD10023764FDFF8F8911D461C46984643
:10C260009B463046FBF7A6F8002840F0AA80F0680D
:10C2700043076BD5029B57F80C2C434500F2A8806E
:10C28000030765D4002D57F80C3C40F3BF8023A969
:10C2900000229C4602E0AA4200F0B78051F8043F19
:10C2A0001B689C4502F10102F5D1C30165D40BF175
:10C2B000010BBBF10C0F06F1140607F11407D0D1E6
:10C2C000584B029593F80090B9F10C0F00F36B8274
:10C2D000584B594A1B791370032B40F2BB801A1F2D
:10C2E000022A00F29482052B00F08282062B0CBFFA
:10C2F0004FF47A564FF47A665049514800224A600A
:10C300000027504AB2FBF6F200260A60C0E9006737
:10C310004D4AA0E0D9F80C3023F00C0343F08073B1
:10C32000C9F80C3051E7D9F80C3023F0807323F0B2
:10C33000040343F00803C9F80C3046E72046FBF736
:10C3400039F90137FFB20744FFB24CE70207ACD519
:10C35000002C57F80C3C4CDD17A900229C4601E04C
:10C36000A24245D051F8043F1B689C4502F10102EE
:10C37000F6D1420786D4C30199D5002C57F80C3C5E
:10C380000ADD17A9002251F8040F0068834202F168
:10C3900001028CD0A242F6D1002D0BDD23A9002290
:10C3A00051F8040F0068834202F101023FF47FAFAD
:10C3B000AA42F5D14FF080711846F160FBF7FAF808
:10C3C00075E75B464A4601210420F9F7AFFB6EE7AB
:10C3D00020F00801F1601046FBF7ECF8F06808F176
:10C3E000010801075FFA88F8B2D44207C3D549E7CC
:10C3F0006346184630AB03EB85020821F16042F832
:10C40000306C0135FBF7D6F851E76346184630AB80
:10C4100003EB84020421F16042F8606C0134FBF705
:10C42000C9F844E7A4000010FC16002048250808BD
:10C43000081700202C410020A23F0020A83F002028
:10C44000B03F002040420F00F1750008288F002007
:10C4500058E408087F4ACAF8F02D7F4A12F81330D2
:10C46000002B00F0CE81A14500F3D381B9F1000F7C
:10C470005CD09FED7A8ADFF828B2794E0DF15C0826
:10C480000024784BDBF804201B7858F8040FC2F323
:10C490000072062B00F21F82DFE803F06C635A374C
:10C4A00004040400052B00F08A816F496F4D062BB0
:10C4B00008BF29460025019200950A46142302214F
:10C4C000FEF774FE0390002800F07B81039AD2F8F7
:10C4D00000C0DCF804E02B46DEF80070DEF81050F7
:10C4E000590106EB431072586A4012F47C5F03F165
:10C4F000010300F0D780102BF2D10023CCF80C30D0
:10C500005B4B039A43F834200DE0DFED5A0A5A4B97
:10C51000B0EE600A5988FFF727F8554B43F834000E
:10C52000002800F051810134A145AAD19AF8F43DC8
:10C530004BBB524A02210420F9F7F8FA9AF8EE0DA3
:10C54000B0FA80F0400931B0BDEC028BBDE8F08F4D
:10C55000DFED4B0A9FED4B0A4FF4FA61FFF704F849
:10C56000DBE7DFED490A4FF47A71B0EE600AFEF7BF
:10C57000FBFFD2E79FED390AF0EE480A4FF4C8718D
:10C58000FEF7F2FFC9E79AF8F58D9AF8F63D08F143
:10C590000108A8EB0308B8F1120F0BDD12230221EA
:10C5A00000933A4A8AF8EE1D434600210420F9F729
:10C5B000BDFAC3E79AF8003E012B00F01E81022B62
:10C5C00040F00C8168F0A8FE314A9AF8003ECAF8A3
:10C5D000042E002B00F00F81022B40F00381029B00
:10C5E000122BB8BF12239BB2984500F31681029B11
:10C5F0009845A8BF9846B8F1000F9FDD254EDFF89B
:10C60000A0B0254F23AD002404E00134444546F892
:10C61000040B93D0DBF80430BAF8F81DC3F30072B2
:10C62000BAF8FA3D01920091B7FBF3F31A4A55F8B4
:10C63000040F9BB20321FEF7B9FD0028E5D10525C3
:10C640000146164A8AF8EE5D23460420F9F76EFA91
:10C6500074E700BF7D8A0008382508086F12833A06
:10C66000340C0020A23F0020C0C62D00001BB700E4
:10C67000E83F0020000000002C41002020E50808D1
:10C68000ACC5A737ACC5A7366F1203393CE508081F
:10C6900009760008287F002040420F00DCE50808EA
:10C6A000AC000010037FCCF80C00002B7FF428AF07
:10C6B000B7F844306FEA43436FEA53439BB2A7F89D
:10C6C00044303B889BB243F080033B809EF80520BA
:10C6D000834B9EF806E004929A181EF0040F92F81D
:10C6E0005023B7F820E014BF0423012393409BB2EA
:10C6F0001FFA8EFE2EEA030EA7F820E03A8C92B2C3
:10C7000013433B843B8842689BB243F001033B8068
:10C71000744B9A4200F09380734B74481A6B42F446
:10C7200080021A6301F118024FF0070E20F802E0B0
:10C730001A6B42F480021A6372186D4892F9143031
:10C74000C2F818C0002BD06072DB6A4A580902EBAD
:10C75000030C4FF0010E03F01F030EFA03F34FF02A
:10C76000300E8CF800E342F8203031448B6805939A
:10C770001846F6F72FF9059B1A6822F001021A6095
:10C780001846F6F727F9DDE904130022CDE9122255
:10C79000CDE914220C921092032900F29A80DFE86E
:10C7A00001F096949260544ACDF800B001218AF8C5
:10C7B000EE1D4B4600210420F9F7B8F9B6E64F49C3
:10C7C00078E64F4B43F8340005218AF8EE1D4D4AB8
:10C7D000234600210420F9F7A9F9A7E64A4ACAF836
:10C7E000042E43B1494A02210420F9F79FF9A5E636
:10C7F0004FF4FA5680E5029BF5E668F08DFD444A59
:10C80000E3E6444A02210420F9F790F98EE6424A11
:10C8100021E6424A00940321C9E7029B00930420C9
:10C820003F4A8AF8EE0D43460021F9F77FF985E685
:10C830003C4A03F00F031A443023137695E7A3F51F
:10C8400020532A481A6B42F400121A6301F11802AD
:10C850004FF0070E20F802E01A6B42F400121A6340
:10C860006AE740371E4A0897EDB202EB8502039F44
:10C87000D2F85423079212220B924FF480624FF4A5
:10C88000804C0D924FF48052CDE90E2C4022184678
:10C8900007F114050A9207A94FF40032119203938D
:10C8A000099567F041FC039B1A6842F010021A6078
:10C8B00028464822002172F04BF801233B71104BAF
:10C8C00043F834702FE63C37CCE73837CAE73437C3
:10C8D000C8E70027C6E70A4A002342F8343073E766
:10C8E000703208080060024000380240380C002016
:10C8F000D102000800E100E070E40808808D5B00D0
:10C90000E83F0020F8E408082576000868E50808F4
:10C910006D8A03089CE40808ED750008BCE408086B
:10C92000A4E50808FCEC00E010B5104CD4E90423A1
:10C93000A16882B002FB03F38B428DF8070012D08E
:10C940006368E0680DF10701184470F0E9FB636863
:10C950002269A16813446269B3FBF1F0013201FB63
:10C9600010336360626102B010BD00BFC03F0020A1
:10C9700010B50379012B84B00C4627D0022B23D1AC
:10C980008368DB070DF10F024CBF01218121FDF708
:10C99000C9F89DF80F300022C3F3001161F30702BC
:10C9A000C3F3800161F30F220F49C3F3C00C6CF392
:10C9B000174281F80001C3F3801161F31F62DB09A4
:10C9C0002260237104B010BD0020E2E782680DF1FF
:10C9D0000F0102F00102CDE900121A46417C90F9E4
:10C9E0001000F6F787FED4E7EC1600202DE9F041A1
:10C9F00082B014460E4601AA50210546FDF7E4F820
:10CA00009DF80430DFF8F080394F01335B00DBB272
:10CA10004621238001AA2846FDF7D6F823789DF801
:10CA2000042008FB03F303F5FA73A7FB0313013299
:10CA30009909DB0902FB0133A280A7FB03239B09B1
:10CA400001AAE360512102232846FCF79BFB2378CF
:10CA5000BDF8040008FB03F340BA03F5FA73A7FB23
:10CA60000323C2B2C0F307208240013292B2980978
:10CA7000DB0902FB0033A7FB03739B097021E280F3
:10CA8000238201AA2846FDF79FF89DF80430013360
:10CA90005B00DBB201AA6380712102232846FCF708
:10CAA00071FBBDF80430134AF17882F800015BBADB
:10CAB000DAB2C3F307239A40013292B2228119B14C
:10CAC000E388D21A92B222810B48A378084900FB6E
:10CAD00003F303F5FA73A1FB03039809DB0902FBD7
:10CAE0000033A1FB03139B09638202B0BDE8F08110
:10CAF000D34D6210EC160020002F3A002DE9F04FC4
:10CB0000DFF89C82DFF89C92DFF89CA2A34F8DB0E7
:10CB1000054600264FF4FA7307AA89210068C8F871
:10CB2000203589F84061FDF74FF89DF81C202868F2
:10CB3000892142F00102FCF70DF93246882128686C
:10CB4000FCF708F9012280212868FCF703F901228B
:10CB5000FF212868FCF7FEF8324631462868FCF7CA
:10CB6000F9F807AA91212868FDF72EF89DF81C30E6
:10CB7000286888F81A3531460122FCF7EBF832466E
:10CB8000FF212868FCF7E6F8324680212868FCF788
:10CB9000E1F807AA60212868FDF716F89DF81C2027
:10CBA0002868602142F01202FCF7D4F84FF40053D9
:10CBB000ADF81C3007AA022344212868FCF7ECF9E1
:10CBC000FF2201212868FCF7C5F82C68012280218A
:10CBD0002046FCF7BFF80122FF212046FCF7BAF8F7
:10CBE000324631462046FCF7B5F80622FF212046A2
:10CBF000FCF7B0F807AA83212046FCF7E5FF9DF873
:10CC00001C20832142F004022046FCF7A3F80722EF
:10CC1000FF212046FCF79EF8012281212046FCF7E7
:10CC200099F8012280212046FCF794F86B22942188
:10CC30002046FCF78FF8324683212046FCF78AF81D
:10CC4000DAF80060C8F81C652379012B00F09880A1
:10CC5000022B0FD000209DF81C3087F80001DBB9B3
:10CC6000DAF800309BB29B1BB3F5FA7FECD90DB01C
:10CC7000BDE8F08FA368DB0707AA4FF083012046C9
:10CC80005EBF07AA83212046FCF74CFF9DF81C30AD
:10CC900087F80001002BE3D0012283212046FCF716
:10CCA00059F807AA92212046FCF78EFF0022812125
:10CCB00020469DF81CB0FCF74DF80622FF212046C7
:10CCC000FCF748F807AA83212046FCF77DFF9DF872
:10CCD0001C20832102F0FB022046FCF73BF80122D6
:10CCE000FF212046FCF736F8012200212046FCF700
:10CCF00031F80022FF212046FCF72CF820460022C4
:10CD00008021FCF727F80623B02105AA2868FCF744
:10CD100039FA0122FF212868FCF71CF800224F2174
:10CD20002868FCF717F82C224E212868FCF712F827
:10CD30000022FF212868FCF70DF84FEADB1628686F
:10CD4000B422B621FCF706F80024002E18BF0C26EA
:10CD50000BF07F0BA2464FF0010EC4F3C403303337
:10CD60006B44E2B213F81C0C04F0070C0EFA0CF141
:10CD7000964220EA010119D903F81C1C0134ECE7A2
:10CD8000A268617C94F9100002F00102019207AAE6
:10CD900000928322F6F7AEFC5DE700BFEC160020A0
:10CDA000288F0020307E002050380020DA4540FADD
:10CDB0000CF200F01183D30744BF0AF1010A5FFAB5
:10CDC0008AFA0134302CC8D1062305AAB02128687C
:10CDD000FCF7E2F80122FF212868FBF7BBFF0022E5
:10CDE00011462868FBF7B6FF0022FF212868FBF7F1
:10CDF000B1FF002209212868FBF7ACFF00221021B7
:10CE00002868FBF7A7FF002211212868FBF7A2FF83
:10CE1000012224212868FBF79DFFFF222521286895
:10CE2000FBF798FF002275212868FBF793FF01228A
:10CE3000FF212868FBF78EFF2C224E212868FBF784
:10CE400089FF002248212868FBF784FF2146202221
:10CE50002868FBF77FFF0022FF212868FBF77AFF95
:10CE6000214609222868FBF775FF00225421286813
:10CE7000FBF770FF042231212868FBF76BFF0322C8
:10CE800032212868FBF766FF832240212868FBF7E0
:10CE900061FF252246212868FBF75CFF0022602104
:10CEA0002868FBF757FF002227212868FBF752FF6D
:10CEB000062250212868FBF74DFF002251212868E7
:10CEC000FBF748FF962252212868FBF743FF082210
:10CED00056212868FBF73EFF224657212868FBF7BA
:10CEE00039FF002261212868FBF734FF002262210C
:10CEF0002868FBF72FFF002264212868FBF72AFF30
:10CF0000002265212868FBF725FFA02266212868FA
:10CF1000FBF720FF0122FF212868FBF71BFF3222CD
:10CF200022212868FBF716FF142247212868FBF707
:10CF300011FFFF2249212868FBF70CFF00224A213C
:10CF40002868FBF707FF0022FF212868FBF702FF94
:10CF50000A227A212868FBF7FDFE00227B2128683F
:10CF6000FBF7F8FE212278212868FBF7F3FE012267
:10CF7000FF212868FBF7EEFE342223212868FBF707
:10CF8000E9FE002242212868FBF7E4FEFF2244214B
:10CF90002868FBF7DFFE262245212868FBF7DAFE2A
:10CFA000052246212868FBF7D5FE40221146286855
:10CFB000FBF7D0FE06220E212868FBF7CBFE1A22D3
:10CFC00020212868FBF7C6FE402243212868FBF792
:10CFD000C1FE0022FF212868FBF7BCFE032234219A
:10CFE0002868FBF7B7FE442235212868FBF7B2FE1C
:10CFF0000122FF212868FBF7ADFE042231212868B9
:10D00000FBF7A8FE09224B212868FBF7A3FE0522A7
:10D010004C212868FBF79EFE04224D212868FBF76F
:10D0200099FE0022FF212868FBF794FE002244218C
:10D030002868FBF78FFE202245212868FBF78AFE2F
:10D04000082247212868FBF785FE28224821286806
:10D05000FBF780FE002267212868FBF77BFE042295
:10D0600070212868FBF776FE012271212868FBF702
:10D0700071FEFE2272212868FBF76CFE00227621E9
:10D080002868FBF767FE002277212868FBF762FE1D
:10D090000122FF212868FBF75DFE01220D2128688F
:10D0A000FBF758FE0022FF212868FBF753FE012200
:10D0B00080212868FBF74EFEF82201212868FBF743
:10D0C00049FE0122FF212868FBF744FE01228E2140
:10D0D0002868FBF73FFE012200212868FBF73AFE93
:10D0E0000022FF212868FBF735FE002280212868F6
:10D0F000FBF730FE04220A212868FBF72BFE2C6880
:10D10000842107AA2046FCF75FFD9DF81C202046DD
:10D1100002F0EF028421FBF71DFE01220B2128689B
:10D12000FBF718FE2C6803A92046FFF721FC07AA8D
:10D1300003A92046FFF75AFC9DF80C30002B00F0A5
:10D140005C810A9C04F684549DF80E30002B00F09C
:10D150004A810A9B03F2B22304EB43049DF80F308B
:10D1600023B1BDF82C3003F525731C449DF8103015
:10D1700023B1BDF82E3003F226231C44E8220121FE
:10D180002868C8F8084EFBF7E5FD2868214668F0D6
:10D19000EFFB012211462868FBF7DCFD402187F8F0
:10D1A00000012868FDF7AAF800283FF460AD0121CE
:10D1B00028680222FBF7CEFD002187F800012868CD
:10D1C000FDF79CF800283FF452ADE82201212868C1
:10D1D000FBF7C0FD4FF4005307AAADF81C30442103
:10D1E00002232868FBF7D8FE2C6803A92046FFF726
:10D1F000BFFB07AA03A92046FFF7F8FB50225721DF
:10D200002046FBF7A7FD082256212046FBF7A2FD8A
:10D21000082250212046FBF79DFDBDF82C204FF43D
:10D220007A7148F20E6301FB0233794A934240F26D
:10D23000EB80784AA2FB0332120C013AFF2A4FF02E
:10D24000000306DD52080133FF2A9BB2FAD81B0205
:10D250009BB21343C3F30722DBB28DF808208DF88D
:10D26000093002AA022351212046FBF795FE0A9AB3
:10D270004FF47A7148F20E6301FB0233664A93421F
:10D2800000F2C080634AA2FB0332120C013AD2B210
:10D2900046212046FBF75EFD2046D8F8081E68F0C0
:10D2A00067FB02AA01212046FCF78EFC02229DF8B2
:10D2B000086001212046FBF74DFD00212046FDF7C7
:10D2C0001DF8324620460121FBF744FD2C6803A9D6
:10D2D0002046FFF74DFB07AA03A92046FFF786FB70
:10D2E000482211462046FBF735FD082247212046FB
:10D2F000FBF730FD032232212046FBF72BFD0722EE
:10D3000030212046FBF726FD0122FF212046FBF7B6
:10D3100021FD202230212046FBF71CFD0022FF21A9
:10D320002046FBF717FD062270212046FBF712FD71
:10D33000BDF82E10394A4FF47A7046F6440300FBCC
:10D340000133A2FB03239DF80F201B0B1AB1BDF87C
:10D35000222013449BB2002B52D05A1EFF2A4FF0BA
:10D36000000306DD52080133FF2A9BB2FAD81B02E4
:10D370009BB21343C3F30722DBB28DF808208DF86C
:10D38000093002AA022371212046FBF705FED8F8D6
:10D39000081E204668F0ECFA02AA01212046FCF79C
:10D3A00013FC9DF80850022201212046FBF7D2FC15
:10D3B00000212046FCF7A2FF2A4620460121FBF768
:10D3C000C9FC6422012387F80001C8F8202589F8E8
:10D3D00040310DB0BDE8F08F0EFA0CFC20EA0C00D5
:10D3E00003F81C0CEDE49DF80D30002B3FF4B6AEB5
:10D3F0000A9B03F525731C44B0E640F63634A3E6D9
:10D400001A46BAE7FF2243E700231A4625E700BF82
:10D410001B0C0100950370F41B280D014963A41334
:10D4200010B5174C84F80514017952BAA4F80624F3
:10D4300001294FF0000282B084F8042410D00229A0
:10D4400003D06FF00C0002B010BD042304F20442BC
:10D45000FF21FBF749FD0028F3D0002002B010BDEA
:10D460008268417C90F9100004F2044402F0010249
:10D47000CDE900420423FF22F6F758FDEBE700BF99
:10D48000288F00202DE9F04F9E4F9F4B9F4D06683F
:10D490003C464FF0000885B0834683F842815B37F5
:10D4A000C4F12D0905F2044A13E0022B0FD1B26832
:10D4B00012F0010F4FF0030352464FF0FF013046C8
:10D4C00001BF03235246FF213046FBF70DFDA74263
:10D4D0001AD0337985F8048409EB0401012B14F880
:10D4E000012F85F8051485F80624DED1B368717C18
:10D4F00096F9100003F00103CDE900A3FF220323F6
:10D50000F6F714FDA742E4D14FF40743A5F804341D
:10D51000402385F8063452460323FF213046FBF7AB
:10D520003BFD00238DF80E300DF10E01304668F002
:10D53000E9F99DF80E30002BF6D04FF40643A5F81C
:10D5400004340123724A85F80634FF210323304650
:10D55000FBF722FD4FF407436D4AA5F8043400247D
:10D560000323FF21304685F80644FBF715FD4FF4F1
:10D570000063A5F804340923654A85F80634FF21C1
:10D5800003233046FBF708FD4FF43063A5F804345D
:10D590005F4A85F8064430460323FF21FBF7FCFC75
:10D5A000002800F0AD80DBF800400DF10E025E2196
:10D5B0002046FBF7CDFEBDF80E30B3F5D77F00F067
:10D5C0008D806BD8512B00F0858079D81D2B7FD1B1
:10D5D0000F2608BB0A224B212046FBF7FFFC0F2237
:10D5E00060212046FBF7FAFC0D2263212046FBF761
:10D5F000F5FCB82269212046FBF7F0FC40F60D72DD
:10D6000078212046FFF70CFF40F60E627A21204673
:10D61000FFF706FF00286ED0DBF80000212168F03C
:10D62000C7F8DBF800400DF10E02DE212046FBF7C3
:10D630008FFEBDF80E309FED377AC3F3090303EB7D
:10D640008303DB0007EE903AF8EEE77A4FF4D84315
:10D6500067EE877AA5F80434FCEEE77A524617EEB7
:10D66000903A1BBAC5F80634FF2106232046FBF783
:10D6700093FC4FF40743DBF80000A5F80434402383
:10D6800085F8063452460323FF21FBF785FCB8B327
:10D690001D4B83F8420105B0BDE8F08F40F2E13246
:10D6A000934219D01CD840F2D922934214D040F2B0
:10D6B000E122934202D0B3F5E67FADD1642688E73C
:10D6C000AD2B0BD0D62B01D0602BA5D1212680E726
:10D6D0001E2BA1D114267CE7C8267AE7322678E7EC
:10D6E00040F28F42934203D040F29152934293D141
:10D6F0004FF4FA766DE73146204668F059F88BE72B
:10D700000020C5E7E3350808307E0020288F002080
:10D710002C9300209A99893F03682DE9F0411F6AF4
:10D720001FB13B46BDE8F0411847002A164611DDFF
:10D7300004460D460E4400E023689B682046984747
:10D740000028F9D0236815F8011B1B68204698476C
:10D75000B542F1D1BDE8F081DEE700BFBFF34F8FE6
:10D760000549064BCA6802F4E0621343CB60BFF37D
:10D770004F8F00BFFDE700BF00ED00E00400FA0599
:10D7800008B572B600224FF0FF31930003F16043F9
:10D7900003F561430132082AC3F88010C3F88011F1
:10D7A000F3D1FFF7DBFF00BF012108B50846F6F70C
:10D7B00027FFFFF7E5FF00BF00B583B00D4900224A
:10D7C00000920091009B04330093009B1B68012B87
:10D7D00002D003B05DF804FB01920191019B064960
:10D7E00004330193019B1A600B6883F308884B682C
:10D7F0009847FEE7502800400000FF1F10B4EFF3E9
:10D800001183102282F31288094C0A4822684FF0D3
:10D81000E021013222608A69C0F80C2E0022C0F893
:10D82000102E0A69DBB283F311885DF8044B704750
:10D8300050380020288F002030B4EFF311821023DD
:10D8400083F312884FF0E023D2B29969186910F47B
:10D85000803F0D481EBF0121C0F8101E99690B4B77
:10D860001D68D0F8103E82F31188094804684FF40F
:10D870007A7202FB04F02B44401A0021B0FBF4F052
:10D8800030BCE3FB02017047288F00205038002095
:10D8900074390020124B5B68C3F30803FBB9EFF344
:10D8A0001183E3B930B40F4A0F4C4FF0E02C1368EA
:10D8B000DCF8180011688B42F9D1D4F80C1E8842AC
:10D8C000F5D80A4A15684FF47A7404FB05F2002172
:10D8D000101AB0FBF5F0E3FB040130BC7047ABE776
:10D8E00000ED00E050380020288F0020743900201F
:10D8F00090B170B5461EFFF7CDFF04460D46FFF709
:10D90000C9FF001B61EB0501B0F57A7F71F10001E1
:10D91000F5D3013EEFD270BD704700BF2DE9F04155
:10D92000076888B08046B6227E213846FBF712FA97
:10D930006426FFF7AFFF04460D46FFF7ABFF001B61
:10D9400061EB0501B0F57A7F71F10001F5D3013E7D
:10D95000EFD102213846FBF753F97B6913B11A68FE
:10D960009B885383FFF796FF04460D46FFF792FF0F
:10D97000001B61EB0501B0F57A7F71F10001F5D371
:10D980007B6913B11A689B8813830A26FFF782FF0D
:10D9900004460D46FFF77EFF001B61EB0501B0F565
:10D9A0007A7F71F10001F5D3013EEFD132467C213F
:10D9B0003846FBF7CFF9FFF76DFF04460D46FFF73A
:10D9C00069FF001B61EB0501B0F57A7F71F1000181
:10D9D000F5D3002259213846FBF7BCF9FFF75AFF6F
:10D9E00004460D46FFF756FF001B61EB0501B0F53D
:10D9F0007A7F71F10001F5D35E22002371498DF821
:10DA000007200DF10702CDE902320122CDE90531EF
:10DA1000049202A94FF4A4723846079269F044FFB9
:10DA20000A26FFF737FF04460D46FFF733FF001BBA
:10DA300061EB0501B0F57A7F71F10001F5D3013E8C
:10DA4000EFD1012259213846FBF784F9FFF722FF75
:10DA500004460D46FFF71EFF001B61EB0501B0F504
:10DA60007A7F71F10001F5D38C2240213846FBF713
:10DA700071F9FFF70FFF04460D46FFF70BFF001B80
:10DA800061EB0501B0F57A7F71F10001F5D3032256
:10DA900041213846FBF75EF9FFF7FCFE04460D46D0
:10DAA000FFF7F8FE001B61EB0501B0F57A7F71F11D
:10DAB0000001F5D3444CD8F8382098F83500B4FB71
:10DAC000F2F2032391B2414AF9F7CEF94388B4FB4D
:10DAD000F3F4C8F840400279422142F0C0023846CF
:10DAE000FBF738F9FFF7D6FE04460D46FFF7D2FEE6
:10DAF000001B61EB0501B0F57A7F71F10001F5D3F0
:10DB0000082243213846FBF725F9FFF7C3FE0446F8
:10DB10000D46FFF7BFFE001B61EB0501B0F57A7FF4
:10DB200071F10001F5D3042258213846FBF712F9B0
:10DB3000FFF7B0FE04460D46FFF7ACFE001B61EB9D
:10DB40000501B0F57A7F71F10001F5D30A22532166
:10DB50003846FBF7FFF8FFF79DFE04460D46FFF73A
:10DB600099FE001B61EB0501B0F57A7F71F10001B0
:10DB7000F5D300227C213846FBF7ECF8FFF78AFE4C
:10DB800004460D46FFF786FE001B61EB0501B0F56C
:10DB90007A7F71F10001F5D306227D213846FBF72B
:10DBA000D9F8FFF777FE04460D46FFF773FE001B1A
:10DBB00061EB0501B0F57A7F71F10001F5D308B092
:10DBC000BDE8F0814036080840420F008837080859
:10DBD0002DE9F043836B0768A04AA14CB4FBF3F135
:10DBE00083B08046052389B290F83500F9F73CF9F7
:10DBF00000214388B4FBF3F48146C8F8404038461E
:10DC0000FAF7FEFF002276213846FBF7A3F80F2231
:10DC10004E213846FBF79EF80F26FFF73BFE0446E1
:10DC20000D46FFF737FE001B61EB0501B0F57A7F6B
:10DC300071F10001F5D3013EEFD199F805204F2194
:10DC400002F00F023846FBF785F80F26FFF722FE99
:10DC500004460D46FFF71EFE001B61EB0501B0F503
:10DC60007A7F71F10001F5D3013EEFD199F80520DB
:10DC7000502102F00F023846FBF76CF80F26FFF731
:10DC800009FE04460D46FFF705FE001B61EB05018A
:10DC9000B0F57A7F71F10001F5D3013EEFD1FF229B
:10DCA00052213846FBF756F80F26FFF7F3FD0446DE
:10DCB0000D46FFF7EFFD001B61EB0501B0F57A7F24
:10DCC00071F10001F5D3013EEFD198F83510072925
:10DCD00041D0644D95F85001F9F724FD0446012226
:10DCE00076213846FBF736F8A2780C213846FBF748
:10DCF00031F822790D213846FBF72CF8A279A38858
:10DD0000120142EA1322D2B20E213846FBF722F862
:10DD10004FF4807195F85001F9F704FD0446022292
:10DD200076213846FBF716F8A2785200032102F05C
:10DD3000FE023846FBF70EF8227904213846FBF73D
:10DD400009F8A279A388120142EA13220521D2B26E
:10DD50003846FAF7FFFF002276213846FAF7FAFF35
:10DD6000032214213846FAF7F5FF0F26FFF792FD3C
:10DD700004460D46FFF78EFD001B61EB0501B0F573
:10DD80007A7F71F10001F5D3013EEFD13246632174
:10DD90003846FAF7DFFF6426FFF77CFD04460D46A0
:10DDA000FFF778FD001B61EB0501B0F57A7F71F19B
:10DDB0000001F5D3013EEFD1082265213846FAF77C
:10DDC000C9FF64210DF107023846FBF7FDFE9DF8FF
:10DDD000072022F0100242F06002642138468DF8DC
:10DDE0000720FAF7B7FF0F26FFF754FD04460D464C
:10DDF000FFF750FD001B61EB0501B0F57A7F71F173
:10DE00000001F5D3013EEFD10DF106024D21384658
:10DE1000FBF7DAFE9DF8062002F03F0242F04002D6
:10DE20004D2138468DF80620FAF794FF0F26FFF7AC
:10DE300031FD04460D46FFF72DFD001B61EB05018A
:10DE4000B0F57A7F71F10001F5D3013EEFD10321E6
:10DE50003846FAF7D5FE03B0BDE8F0839C370808D2
:10DE600040420F00307E0020F0B5002283B007460C
:10DE70000A210068FAF76EFF1426FFF70BFD04462F
:10DE80000D46FFF707FD001B61EB0501B0F57A7F3A
:10DE900071F10001F5D3013EEFD138680F220A215C
:10DEA000FAF758FF0A26FFF7F5FC04460D46FFF780
:10DEB000F1FC001B61EB0501B0F57A7F71F1000107
:10DEC000F5D3013EEFD13868032301AA1021FBF7F7
:10DED00059F90A26FFF7DEFC04460D46FFF7DAFC87
:10DEE000001B61EB0501B0F57A7F71F10001F5D3FC
:10DEF000013EEFD19DF804209DF805009DF8061025
:10DF0000194B803280308031A3F82425A3F82605F0
:10DF10003246A3F8281538680A21FAF71BFF0A26AB
:10DF2000FFF7B8FC04460D46FFF7B4FC001B61EB9D
:10DF30000501B0F57A7F71F10001F5D3013EEFD113
:10DF40000DF1030238680221FBF73EFE0DF10302DA
:10DF500038680921FBF738FE386811220A21FAF7E0
:10DF6000F9FE012003B0F0BD288F0020F0B500229B
:10DF700083B007460A210068FAF7ECFE1426FFF783
:10DF800089FC04460D46FFF785FC001B61EB05018B
:10DF9000B0F57A7F71F10001F5D3013EEFD1386819
:10DFA0000F220A21FAF7D6FE0A26FFF773FC044671
:10DFB0000D46FFF76FFC001B61EB0501B0F57A7FA2
:10DFC00071F10001F5D3013EEFD13868032301AAB6
:10DFD0001021FBF7D7F80A26FFF75CFC04460D4634
:10DFE000FFF758FC001B61EB0501B0F57A7F71F17A
:10DFF0000001F5D3013EEFD1324638680A21FAF725
:10E00000A9FE0A26FFF746FC04460D46FFF742FC30
:10E01000001B61EB0501B0F57A7F71F10001F5D3CA
:10E02000013EEFD10DF1030238680221FBF7CCFD70
:10E030000DF1030238680921FBF7C6FD386801229B
:10E040000A21FAF787FE012003B0F0BDF8B5782267
:10E05000074600210068FAF77DFE0526FFF71AFC47
:10E0600004460D46FFF716FC001B61EB0501B0F5F9
:10E070007A7F71F10001F5D3013EEFD1386820229B
:10E080000121FAF767FE0526FFF704FC04460D465A
:10E09000FFF700FC001B61EB0501B0F57A7F71F121
:10E0A0000001F5D3013EEFD1324638680221FAF77C
:10E0B00051FE6426FFF7EEFB04460D46FFF7EAFB30
:10E0C000001B61EB0501B0F57A7F71F10001F5D31A
:10E0D000013EEFD10120F8BD70B524220446412154
:10E0E0000068FAF737FE90B90526FFF7D3FB044620
:10E0F0000D46FFF7CFFB001B61EB0501B0F57A7F02
:10E1000071F10001F5D3013EEFD1012070BD20680F
:10E1100020223021FAF71EFE0028E5D020680622D2
:10E120003121FAF717FE0028DED0206800223421C2
:10E13000FAF710FED8E700BFF8B5072207460A2114
:10E140000068FAF707FE0526FFF7A4FB04460D4614
:10E15000FFF7A0FB001B61EB0501B0F57A7F71F1C1
:10E160000001F5D3013EEFD1386824224121FAF7AE
:10E17000F1FD0526FFF78EFB04460D46FFF78AFBEF
:10E18000001B61EB0501B0F57A7F71F10001F5D359
:10E19000013EEFD13868C0224221FAF7DBFD0526A7
:10E1A000FFF778FB04460D46FFF774FB001B61EB9D
:10E1B0000501B0F57A7F71F10001F5D3013EEFD191
:10E1C0000120F8BDF8B50122074610210068FAF7D2
:10E1D000C1FD00B9F8BD1426FFF75CFB04460D46EF
:10E1E000FFF758FB001B61EB0501B0F57A7F71F179
:10E1F0000001F5D3013EEFD13868A022BDE8F84018
:10E200001121FAF7A7BD00BFF0B583B00023074680
:10E210008DF802301426FFF73DFB04460D46FFF74C
:10E2200039FB001B61EB0501B0F57A7F71F100014C
:10E23000F5D3013EEFD131460DF102023868FBF70C
:10E24000C3FC0DF1020280213868FBF7BDFC4FF4DE
:10E25000F842ADF8042038688DF80660032301AA5F
:10E260006021FAF799FE1426FFF714FB04460D46C9
:10E27000FFF710FB001B61EB0501B0F57A7F71F130
:10E280000001F5D3013EEFD131460DF103023868AC
:10E290008DF80360FBF798FC4CF26243ADF8043054
:10E2A00004238DF806303868032301AA6021FAF7A9
:10E2B00073FE1426FFF7EEFA04460D46FFF7EAFA5E
:10E2C000001B61EB0501B0F57A7F71F10001F5D318
:10E2D000013EEFD131460DF1030238688DF803603D
:10E2E000FBF772FC4FF4E853ADF8043008238DF8C7
:10E2F0000630386801AA03236021FAF74DFE142680
:10E30000FFF7C8FA04460D46FFF7C4FA001B61EB9D
:10E310000501B0F57A7F71F10001F5D3013EEFD12F
:10E320000DF10302314638688DF80360FBF74CFCB1
:10E3300038680DF102021E21FBF746FC012003B0F4
:10E34000F0BD00BF2DE9F047C2B282B00E233221EA
:10E350000220FCF753FDDFF85CA10746CAF8540120
:10E36000002864D00321FAF74BFC4FF00008C146A7
:10E370003226FFF78FFA04460D46FFF78BFA001B93
:10E3800061EB0501B0F57A7F71F10001F5D3013E33
:10E39000EFD19F23019397F91030404C8DF8016025
:10E3A00003EB830304EB8303D3F8CC01BB689A0728
:10E3B00058D504230DEB0302694669F025FABB68C2
:10E3C0009B0738D59DF802109DF80130344A0902A8
:10E3D000002741EA03419DF803302780C4E9017713
:10E3E0001943304BA781994204D1B2F80480B2F8A6
:10E3F0000690012752F8083F002BF4D1002F44D09B
:10E40000A4F80080A4F80C90B8F1000F3DD04FEABA
:10E410000922A37302FB08F3C4E90123B3F1807F4F
:10E420004FF48072628032D801238AF8583138461E
:10E4300002B0BDE8F0871C4B1C491A681C4B4FF416
:10E44000FA7000FB02F2A3FB0232486892094B68A3
:10E450001B1A9A42FBD27B69002BB3D01A689B88A7
:10E460001383AFE77B6913B11A689B8853830E4B04
:10E470000E491A680E4B4D68D200A3FB0232920976
:10E480004B685B1B9A42FBD293E70027CFE701233F
:10E49000B7208AF86031F9F74FFAC5E7EC1600208B
:10E4A000BC3708081620C20074390020001000E0B4
:10E4B000D34D6210307E00202DE9F041C2B282B00F
:10E4C0000E2333210220FCF799FCDFF8A4800746D5
:10E4D000C8F8640168B3002301933226FFF7DAF924
:10E4E00004460D46FFF7D6F9001B61EB0501B0F5B8
:10E4F0007A7F71F10001F5D3013EEFD104230DEBDA
:10E5000003029F213846FAF73DFE9DF806309DF83C
:10E510000510154A1B0243EA01439DF807100B43FF
:10E52000934209D0C8E91F66A8F87860A8F884600B
:10E53000304602B0BDE8F0810C4BC8F878300126B7
:10E5400040214FF400324FF00063C8E91F23A8F8C0
:10E55000841088F8866088F86861F9F751FD3046C4
:10E5600002B0BDE8F08100BF21AAEF00000400085E
:10E57000307E002010B5044630B1036823B1DB685B
:10E5800013B1BDE810401847FFF784F9D4E904231C
:10E590009042994134BF0120002010BD70B5006841
:10E5A00001220921FAF7D6FB6426FFF773F9044626
:10E5B0000D46FFF76FF9001B61EB0501B0F57A7F9F
:10E5C00071F10001F5D3013EEFD170BD2DE9804816
:10E5D00083B0431C0193DFF830810A230093D8F8FD
:10E5E0008011D8F88C31B8F88401B8F89021DDF8A2
:10E5F00004B048834FF0320A1A834FF00509D8F867
:10E600008031B8F8842159690A4214BF5A831A83A9
:10E61000D8F88C31B8F8902159690A4214BF5A834E
:10E620001A8356465746FFF735F904460D46FFF75D
:10E6300031F9001B61EB0501B0F57A7F71F1000142
:10E64000F5D3013FEFD1D8F88031B8F8842159696A
:10E650000A4214BF5A831A83D8F88C31B8F8902133
:10E6600059690A4214BF5A831A83FFF713F9044603
:10E670000D46FFF70FF9001B61EB0501B0F57A7F3E
:10E6800071F10001F5D3013EEFD1B9F1000F1CD0BB
:10E69000B9F10109B3D14FF4FA76FFF7FBF804465C
:10E6A0000D46FFF7F7F8001B61EB0501B0F57A7F27
:10E6B00071F10001F5D3013EEFD14FF0FA0ABBF141
:10E6C000000F07D04FF0000999E70BF1FF3BBBF1BA
:10E6D000000FF7D14FF47A76FFF7DCF804460D46C9
:10E6E000FFF7D8F8001B61EB0501B0F57A7F71F1F7
:10E6F0000001F5D3013EEFD1009B013B00937FF475
:10E700006EAFFFF751F800BF482C0020437A5A1C27
:10E710000344D2B242729972037A934200D970478D
:10E72000002AFCD010B5044604F10A01D0E90030FB
:10E7300098470023637210BD2E4E3568F06880B58F
:10E740002EF0FEFA28462EF0FBFAF76879798B074F
:10E7500047D500210846FCF761FF00210120FCF7A6
:10E760005DFF254C3B6838465B68984758B92B6875
:10E7700028465B689847F8B9F7683B6838465B6895
:10E7800098470028F3D0F068D4F88C210368B4F8D7
:10E790009011DB68518398472B6801461B68284617
:10E7A0009847D4F88C31B4F890211A832B68284606
:10E7B0005B6898470028DFD0D4F880212B68B4F834
:10E7C0008411DB685183284698470146F068036846
:10E7D0001B689847D4F88031B4F88421F7681A830D
:10E7E000C0E73B6838469B6941F002019847F768EB
:10E7F000AFE700BFB0A40020482C00200FB410B534
:10E8000082B004AB0B4C53F8042BA06B0A49019364
:10E8100069F022F9A46B627A32B1D4E9003004F1D4
:10E820000A0198470023637202B0BDE8104004B0AB
:10E83000704700BFB0A400200DE70008F8B50446FB
:10E840000F46164600252046202171F0F9FF0446A8
:10E85000C8B10378202B03D114F8013F202BFBD043
:10E860002046F7F721FEB0F5617F10DB40F6340358
:10E87000984211DD30231A46C5B17B7033780133DD
:10E8800033702046F8BD002DFBD10125DBE70023C6
:10E890001A46002DF1D109E0074AA0F56173A2FBE9
:10E8A0000323DA08C3F3C703002DE6D13A703378A7
:10E8B00001333370E9E700BF1F85EB5170B50546A2
:10E8C00008460E4672F0FCF83146044602462846D9
:10E8D000F7F7CEFA68B92B5DA3F13002092A00D808
:10E8E00070BD23F02003413B192BF9D901342819BD
:10E8F00070BD002070BD00BF18B103685B6903B133
:10E900001847704718B103681B6A03B11847002005
:10E91000704700BF38B50B4D0C4620B10368DB6A69
:10E920000BB1984760B90020C4E90000C4E90200B7
:10E93000C4E906552D2230232061227584F8203049
:10E9400038BD00BFC04209080178F1B1F8B50F4FDA
:10E950000546002602E015F8011FA9B1BC6B637AD9
:10E960005A1C2344D2B262729972237A9342F2D82B
:10E9700004F10A01002AEED0D4E90030984766720B
:10E9800015F8011F0029E9D1F8BD7047B0A4002097
:10E9900070B504460E48FFF7D7FF2046FFF7D4FFB7
:10E9A0000C48FFF7D1FF0C4B9E8F16B970BD013E8E
:10E9B000FCD0FEF76FFF04460D46FEF76BFF001B11
:10E9C00061EB0501B0F57A7F71F10001F5D3EEE757
:10E9D00004E6080818E70808B0A4002070B5114C38
:10E9E00005460E461048FFF7AFFF2A460F49A06BB9
:10E9F000334669F031F8A56B6A7A32B12B686868E2
:10EA000005F10A01984700236B7294F83E303BB140
:10EA100094F840300122134484F83F2084F84030B9
:10EA200070BD00BFB0A400200CE608080DE7000888
:10EA30000FB470B582B006A951F8040B0191FFF72D
:10EA4000CDFF0E48FFF780FF0D4B9E8F36B902B009
:10EA5000BDE8704004B07047013EF8D0FEF71AFFE1
:10EA600004460D46FEF716FF001B61EB0501B0F5ED
:10EA70007A7F71F10001F5D3EEE700BF18E70808CF
:10EA8000B0A4002070B5C379044603F007008CB031
:10EA90001546062800F29680DFE800F00924333599
:10EAA000384004004C480CB0BDE87040A6E60E7833
:10EAB00013F0C0031BD0402B21D13146237A4A2BBF
:10EAC0005DD8464A02EBC30393F8B821914256D26F
:10EAD000D3F8B43153F82100002850D00CB0BDE871
:10EAE00070408BE613F0C00391F90060E3D13C481D
:10EAF0003146FFF783FE15B1E3793F2B4DD90CB0BA
:10EB000070BD0E88D4E7B1F90060D1E7096813F051
:10EB1000C0030E463DD0402BD0D0F0E791ED000A67
:10EB20006846F7F79DFB01462B48FFF767FE002D6F
:10EB3000E5D0E3793F2BE2D8237A284D35F923300D
:10EB400000EE103A6846B8EEC00AF7F789FB0146B6
:10EB50002448FFF753FEE37903F0C003402B28D08D
:10EB6000637A05EB830393ED000AB8EE400A68462A
:10EB7000F7F776FB01461B48FFF740FEBFE7694603
:10EB8000204621F0D1FE18486A463146FFF750FF73
:10EB9000B5E71648FFF732FEADE7104B627A217AEF
:10EBA00053F8222033F9211011480CB0BDE8704011
:10EBB00024E6237A05EBC30595F8B831013B00EE56
:10EBC000103AD2E713F0C00304D0402B97D10021B4
:10EBD0000E4673E71E468AE7A8F508089C38080821
:10EBE000A8F308080823090820E6080824EC080808
:10EBF00018E60808D8B10378CBB12DE9F04F87B0FB
:10EC0000704905AA6EF018FA8246002800F0CE80FE
:10EC10000024DFF8ECB16B4EA1462546A0464FF02C
:10EC2000FF37032C32D8DFE804F0676C2104664814
:10EC3000FEE6504671F044FF032867D19AF80020A1
:10EC4000382A63D19AF80120452A00F081804E2AA3
:10EC50005CD100229AF80230312B00F08980322BEF
:10EC600054D149EA020242F002090FE059465046E7
:10EC700071F030FD002874D045F00105534950462D
:10EC800071F028FD002865D045F0020505AA31463F
:10EC900000206EF0D1F9013482460028C1D178B24B
:10ECA0004B4A002392F90010814232D00133072BE6
:10ECB00002F10C02F6D1B8F1000F5CD0002D08BFB4
:10ECC00003250023EDB2CDE90085CDF808901A4662
:10ECD00019462DF0D1FD064600286ED03D483E4C29
:10ECE00042463946F6F7E8FE39463C48F6F7E4FE78
:10ECF0002068314664F0EEF95046F7F7D5FB074639
:10ED0000C4E75046F7F7D0FB8046BFE74FF0FF0956
:10ED1000BCE7314C03EB430304EB83039E6C002EF2
:10ED2000C9D02F483946F6F7C7FE15B17179A94207
:10ED300028D1B9F1000F02D0B17949452CD1F36A3D
:10ED4000002BD1D02748F6F7B7FE0023F362CBE7BC
:10ED500004227FE72449504671F0BCFC002893D17F
:10ED600094E72249504671F0B5FC002884D185E72C
:10ED700049EA02098AE71E483946F6F79DFE07B0C0
:10ED8000BDE8F08F2A461B48F6F796FE3368E9B2D5
:10ED90009B6930469847CCE74A461748F6F78CFE01
:10EDA00033684946DB6930469847C8E781464FF0EB
:10EDB000FF305546D046074672E739460F48F6F70A
:10EDC0007BFEDCE71846090840E6080850E608081C
:10EDD000F4A40020A0E60808B0A4002034E7080846
:10EDE000C0E608081CE7080854E60808CC0E090825
:10EDF00058E60808D8E60808F8E6080880E6080893
:10EE00004CE60808A0B32DE9F04F037887B005461B
:10EE10003BB300F10040514C0138294603E09F42CA
:10EE20002AD1814212D011F8013BA3F14102192AE3
:10EE300014F8012BA2F1410698BF2033192E02F1DC
:10EE40002007ECD99A4217D1002BEAD1444B00227B
:10EE5000C3F8242E83F82D2EA3F82B2E07B0BDE87F
:10EE6000F08F0021012007B0BDE8F04F64F08CB9AD
:10EE70000021012064F088B93A4C294603E09F4202
:10EE80001AD1814212D011F8013BA3F14102192A93
:10EE900014F8012BA2F1410698BF2033192E02F17C
:10EEA0002007ECD99A4207D1002BEAD1012007B004
:10EEB000BDE8F04F54F07ABF2B4C294603E09F4247
:10EEC00058D1814212D011F8013BA3F14102192A15
:10EED00014F8012BA2F1410698BF2033192E02F13C
:10EEE0002007ECD99A4245D1002BEAD11C4B0022D5
:10EEF00093F92B4E83F8242E1846164693F8D61411
:10EF00000129A1F1030509D0052D07D90EB180F81B
:10EF10002B4E164807B0BDE8F04F89E593F8D7149B
:10EF2000A52903F1140303D00132782AE6D1EDE7D5
:10EF3000012C03D0013C64B20126F5E70C4980F8AE
:10EF4000244E0023013280F8252E81F8983080F875
:10EF50002B3E07B0BDE8F04F54F08ABF64E70808C5
:10EF6000F07F00206CE708082CFB080840E6080842
:10EF7000B0A40020DFF8C8B22846F7F795FA9BF94D
:10EF800098A00AFA80F6772E074600F2DB80284622
:10EF9000202171F055FC0446002800F02A810378F6
:10EFA000202B03D114F8013F202BFBD02046F7F78C
:10EFB0007BFA01255FFA80F82046202171F040FCA1
:10EFC0000446002800F013810378202B03D114F8A5
:10EFD000013F202BFBD02046F7F766FA0135019060
:10EFE000EDB22046202171F02BFC0446002800F0F1
:10EFF000FC800378202B03D114F8013F202BFBD099
:10F000002046F7F751FA01350290EDB22046202153
:10F0100071F016FC0446002800F0E5800378202BF0
:10F0200003D114F8013F202BFBD02046F7F73CFA20
:10F0300001350390EDB22046202171F001FC044619
:10F04000002800F0CE800378202B03D114F8013F74
:10F05000202BFBD02046F7F727FA013503B20493A3
:10F06000EDB22046202171F0EBFB0446002800F0B1
:10F07000B0800378202B03D114F8013F202BFBD064
:10F080002046F7F711FA20210346204605931CB2CB
:10F0900071F0D6FB0135059BEDB20246002859D030
:10F0A0001378202B03D112F8013F202BFBD0104600
:10F0B0000592F7F7F9F9059A0FFA80F92021104621
:10F0C00071F0BEFB00284CD00378202B03D110F840
:10F0D000013F202BFBD0F7F7E7F905F0FD05042DE4
:10F0E00008BFC3B27FF415AFB8F1010F0AD9B8F168
:10F0F000040F07D0A8F10502032A03D9B8F1030FC2
:10F100007FF407AF23B1A52B44D0482B7FF401AF88
:10F11000002E39D1474A82F82B6E82F8D6840199A5
:10F12000C2F8C4140299C2F8C8140399C2F8CC14E6
:10F130000499A2F8D014A2F8D244A2F8D49482F888
:10F14000D7348BE63C493D487723002207B0BDE821
:10F15000F04F6DE4062D7FF4DCAE8146DBB2044651
:10F16000C2E7052D7FF4D5AEB8F1010F0AD9B8F189
:10F17000040F07D0A8F10503032B03D9B8F1030F3F
:10F180007FF4C7AE0346C3E72A4A06EB860602EBC6
:10F190008602C2E786BB2748019AC0F8C424029AB7
:10F1A000C0F8C824039AC0F8CC24049A80F8D73455
:10F1B00080F8D684A0F8D024A0F8D244A0F8D49443
:10F1C00001230AF101023A448BF8982080F82B3E83
:10F1D00044E6202171F034FB024600287FF460AF42
:10F1E00097E604903DE7039025E702900EE7019033
:10F1F000F7E605468046DFE60E48019906EB8606EF
:10F2000000EB8602C2F8C41482F8D734029990F851
:10F210002B3EC2F8C8140399C2F8CC1401330499E8
:10F2200082F8D684A2F8D014A2F8D244A2F8D494DA
:10F230005BB2C6E7F07F002074E7080880E70808A3
:10F24000B0A400202DE9F04782B03C4901AA6DF03E
:10F25000F3FE002863D04FF0000A4FF0FF34374D23
:10F26000D1465646D0462746BAF1040F37D8DFE8D4
:10F270000AF0423C310B03000378482B41D0562B57
:10F280002DD14FF0010904E0F7F70EF93F280646AB
:10F2900025D8002001AA29460AF1010A6DF0CCFE0A
:10F2A0000028E1D1BAF1040F2ED0BAF1050F40D1F8
:10F2B000234AB301A72103F47C6308F03F0801FB54
:10F2C000074443EA080302EB440243EA4933A2F845
:10F2D0009C3007E0F7F7E8F83F288046D9D919486D
:10F2E000FFF7A6FB02B0BDE8F087F7F7DDF8A62828
:10F2F0000446CED9F3E7F7F7D7F803280746C8D96D
:10F30000EDE74FF00009C4E70D4AA72303FB0743CD
:10F3100002EB4303B3F89C90C9F34039C9E74FF0BF
:10F32000FF373C46084923463A46012063F0B8FFC0
:10F33000D8E7BAF1030FD2D0F4E700BF18460908A6
:10F34000B0A4002040E608084CA500202DE9F04FAD
:10F350008FB0DFF8A4829C4E9C4C0091074603E0DE
:10F360000C34444500F0AC80B56B6A7A32B12B683E
:10F37000686805F10A01984700236B72E27902F090
:10F380003803BB42ECD1914BA4EB030C904B4FEAFA
:10F39000AC0C03FB0CFC1FFA8CFCBCF11B0F40F205
:10F3A00006818C4D01201C2302E0342800F0D3801C
:10F3B00015F8011F0B449BB29C45014600F101006A
:10F3C000F3D2854B03EB4103B3F80C548348844BD1
:10F3D000834204D3F4E01433834280F0F18019882F
:10F3E000C1F30B01A942F6D12046D3F808B001922F
:10F3F00021F014FB81460BEB000A204621F066FB4E
:10F40000019A0146009802F0070300F02005062B40
:10F4100014D8DFE803F07F87776E58049000D1EDB1
:10F42000007A9AED007AB4EE677AF1EE10FA0CBF2A
:10F4300001230023002D4FD0002B91D102AD29468E
:10F44000204621F071FA009B5A0613D565482946DB
:10F45000FFF7D4F92B68644A93427FD000225146CB
:10F460002046FFF70FFB6148FFF76EFAB38F002BC2
:10F4700040F088805E482946FFF7C0F900225146D7
:10F480002046FFF7FFFA5948FFF75EFAB38F002BCB
:10F490003FF466AF9A46FEF7FDF905468946FEF74A
:10F4A000F9F9401B61EB0901B0F57A7F71F10001B8
:10F4B000F5D3BAF1010AEED10C3444457FF454AFD0
:10F4C0000FB0BDE8F08F0A685BF809309B1AB3FAF9
:10F4D00083F35B09002DAFD102AD2946204601938D
:10F4E00021F022FA009B5B06C4D5019B002BC1D101
:10F4F000ACE7B1F900203BF909309B1AB3FA83F36A
:10F500005B0997E70A883BF809309B1AB3FA83F343
:10F510005B098FE70A781BF809309B1AB3FA83F36B
:10F520005B0987E791F900201BF909309B1AB3FAB0
:10F5300083F35B097EE702F0C002402A264B38D0F5
:10F54000627A53F82220013250466EF023F9B0FA65
:10F5500080F35B096EE74FF6FF7537E72B79002BD9
:10F560007FF47CAF1BF80930202B7FF477AF214864
:10F570005146FFF743F91D48FFF7E6F9B38F002B1B
:10F580003FF478AF9B460194FEF784F90446894620
:10F59000FEF780F9001B61EB0901B0F57A7F71F18C
:10F5A0000001F5D3BBF1010BEED1019C62E70A2506
:10F5B0000CE7227A03EBC20393F8B821013AC2E7C1
:10F5C00000239B68FFDE00BFB0A40020644E080843
:10F5D000ABAAAAAA103D08089C380808EC5B0908E9
:10F5E00088560908ACE708086E616D6518E70808D9
:10F5F000A0E70808B8E70808A06C080880B5184814
:10F60000184DFFF7A1F91848FFF79EF9AC6B627A25
:10F6100032B12146606851F80A3B98470023637273
:10F620002F683B6838465B699847B0B90A26FEF7F1
:10F6300031F904460D46FEF72DF9001B61EB050379
:10F64000B0F57A7F73F10003F5D3013EEFD13B684B
:10F6500038465B6998470028E8D0012007F0B6FDDE
:10F66000C0E70808B0A40020DCE70808174B93F8AF
:10F67000D425012A00D0704710B593F8D925062A61
:10F6800084B00FD00A2A07D134F016F8104804B01D
:10F69000BDE81040FFF758B90E4804B0BDE810406F
:10F6A000FFF752B9D3F8F4454CB10B4A07CA01AB86
:10F6B00003C301A91A7020460922FEF72DF8074856
:10F6C00004B0BDE81040FFF73FB900BFB0A4002070
:10F6D000F8E70808E8E7080830E8080814E8080828
:10F6E00080B52D482D4FFFF72FF92D48FFF72CF946
:10F6F000BE8F002E40D1BC6B627A32B12146606869
:10F7000051F80A3B984700236372264B00251D7071
:10F7100087F8F855C7F8385623F0C0FB2248FFF7A2
:10F7200013F9BC6B627A2AB12146606851F80A3B32
:10F73000984765723F683B6838465B699847B0B93F
:10F740000A26FEF7A7F804460D46FEF7A3F8001BAD
:10F7500061EB0503B0F57A7F73F10003F5D3013E49
:10F76000EFD13B6838465B6998470028E8D0002015
:10F7700007F02CFD013EBED0FEF78CF804460D4686
:10F78000FEF788F8001B61EB0501B0F57A7F71F197
:10F790000001F5D3EEE700BF3CE80808B0A4002064
:10F7A00018E70808B87E0020DCE70808F0B5374CF9
:10F7B00094F83E3091B01BB194F83F30002B4FD1FC
:10F7C0003348FFF7C1F8012384F83F3684F87836D0
:10F7D000F7F750F940B9F7F74DF928B9F7F74AF9B3
:10F7E00010B90520FEF7F2FEF7F7D0F80028F8D0A0
:10F7F000284B29481A68C4F84C260026012384F8AF
:10F80000786684F83F6684F86E36FFF79DF8A56B3E
:10F810006A7A2AB1D5E9003005F10A0198476E727B
:10F8200027683B6838465B699847B0B90A26FEF7F7
:10F8300031F804460D46FEF72DF8001B61EB05017B
:10F84000B0F57A7F71F10001F5D3013EEFD13B684D
:10F8500038465B6998470028E8D0002007F0B6FCDE
:10F8600094F840200D4901A8F6F748F901A8FFF7E0
:10F87000DFF80B48FFF7DCF8002384F83E3084F80B
:10F880003F3084F8403011B0F0BD00BFB0A400207C
:10F89000CCE8080850380020DCE7080868E80808C9
:10F8A000ACE80808F8B52C4C05462C48FFF74CF896
:10F8B00006F0A8F8012384F83F3684F87836F7F785
:10F8C000D9F840B9F7F7D6F828B9F7F7D3F810B94F
:10F8D0000520FEF77BFEF7F759F80028F8D0204AFC
:10F8E0001168C4F84C160023012228461D4984F8EB
:10F8F000783684F83F3684F86E2684F83F30FEF779
:10F90000DDFF054600B1F8BD1748FFF71DF8A66BEF
:10F91000727A2AB1D6E9003006F10A019847757269
:10F9200027683B6838465B69984788B90A26FDF71F
:10F93000B1FF04460D46FDF7ADFF001B61EB05016D
:10F94000B0F57A7F71F10001F5D3013EEFD1E8E720
:10F95000002007F03BFC00BFB0A40020D4E808085A
:10F9600050380020ECE80808DCE70808F8B5394B07
:10F97000394F1B68D7F87C46002B69D01B6A984723
:10F98000A28861884468521A02FB0444002C4AD0C1
:10F990003248FEF7D9FF3248FEF7D6FF3148FEF76E
:10F9A000D3FFBE8F86BB3048FEF7CEFFBC6B627ABA
:10F9B000002A45D14FF47A76FDF76CFF04460D46D8
:10F9C000FDF768FF001B61EB0501B0F57A7F71F16F
:10F9D0000001F5D3013EEFD138682DF0B1F9234B8A
:10F9E0001A784AB12249304651F836300BB19B683B
:10F9F000186001369642F7D102210120F4F700FE8B
:10FA0000FDF7BEFE013ECED0FDF744FF04460D4695
:10FA1000FDF740FF001B61EB0501B0F57A7F71F146
:10FA20000001F5D3EEE71348FEF78EFFBD6B6A7A4F
:10FA30002AB12B68686805F10A0198476C72F8BD15
:10FA40002368606804F10A01984700236372B1E7F4
:10FA5000094895E794940020B0A4002004E6080823
:10FA6000F8E8080818E70808DCE70808A400001010
:10FA7000E83F002018E908089CA400202DE9F84F71
:10FA80001A4FDFF870A0DFF870B0DFF8709007F55C
:10FA90004C7802E01037474526D03868FEF754FF0F
:10FAA000796811B15846FEF7A9FEB96811B110483E
:10FAB000FEF7A4FE4846FEF747FFBAF83C60002E6A
:10FAC000E8D0FDF7E7FE04460D46FDF7E3FE001B18
:10FAD00061EB0501B0F57A7F71F10001F5D3013ECC
:10FAE000EFD110374745D8D1BDE8F88F443D08081D
:10FAF00050E90808B0A4002048E9080818E70808F9
:10FB000070B50C48FEF720FF0B4B9E8F16B970BDE9
:10FB1000013EFCD0FDF7BEFE04460D46FDF7BAFEE1
:10FB2000001B61EB0501B0F57A7F71F10001F5D39F
:10FB3000EEE700BF18E70808B0A400202DE9F04167
:10FB4000304F3B68002B5BD01B6A98478368002BC3
:10FB500050D02D48DFF8C480FEF7F6FE2B48FEF7A4
:10FB6000F3FEB8F83C60D6B93FF066F83B6813B1D5
:10FB70005B68984710BB6426FDF78CFE04460D4673
:10FB8000FDF788FE001B61EB0501B0F57A7F71F18E
:10FB90000001F5D3013EEFD1E8E7013EE4D0FDF7E7
:10FBA00079FE04460D46FDF775FE001B61EB05016D
:10FBB000B0F57A7F71F10001F5D3EEE71448FEF756
:10FBC000C3FE1248FEF7C0FEB8F83C601EB9BDE89F
:10FBD000F081013EFBD0FDF75DFE04460D46FDF7CA
:10FBE00059FE001B61EB0501B0F57A7F71F1000150
:10FBF000F5D3EEE70748FEF7A7FEBDE8F0417FE743
:10FC00000548A3E7949400206CE9080818E7080861
:10FC100078E9080858E908089CA40020B0A400204E
:10FC200070B52C4990B00522044670F007FF30BB38
:10FC3000294C94F83E30D3B12848FEF785FE284879
:10FC4000FEF782FEA68F1EB910B070BD013EFBD03C
:10FC5000FDF720FE04460D46FDF71CFE001B61EB80
:10FC60000501B0F57A7F71F10001F5D3EEE70122CD
:10FC700084F83E2084F83F3084F84030DCE71949AE
:10FC80000322204670F0DAFEF0B9134C94F83E30AF
:10FC900013B194F83F306BB91348FEF755FEFFF7E8
:10FCA0002FFF002384F83E3084F83F3084F8403042
:10FCB00010B070BD94F840200C4901A8F5F71EFF64
:10FCC00001A8FEF7B5FEECE7094810B0BDE87040AA
:10FCD000FEF7AEBE80E90808B0A4002088E9080855
:10FCE00018E7080800040908A0E9080868E80808F7
:10FCF000B4E90808800601D5002930D10CB470B5EC
:10FD0000184C1949A06B82B007AB069A019367F0B3
:10FD1000A3FEA56B6A7A32B12B68686805F10A0107
:10FD2000984700236B721148FEF70EFEA68F3EB96E
:10FD3000012002B0BDE8704002B07047013EF7D02C
:10FD4000FDF7A8FD04460D46FDF7A4FD001B61EB81
:10FD50000501B0F57A7F71F10001F5D3EEE70020DF
:10FD6000704700BFB0A400200DE7000818E708089E
:10FD7000F0B5054683B060B304785CB300F1004E83
:10FD8000444C0EF1FF3E014603E0984236D17145E6
:10FD900013D011F8013BA3F14102192A14F8012BE9
:10FDA000A2F1410C98BF2033BCF1190F02F12000E1
:10FDB000EBD99A4222D1002BE9D1374B374AC3F80D
:10FDC0008026C3F88426C3F88826C3F88C2603B09F
:10FDD000F0BD0446324D334E35F8243005EB840235
:10FDE000002152880120CDE90032234632460134F9
:10FDF000FFF780FF042CEFD103B0F0BD2846F6F7E3
:10FE000053FB0328064639D82021284670F018FDF8
:10FE1000044600283BD00378202B03D114F8013F7F
:10FE2000202BFBD02046F6F73FFB0127054620217B
:10FE3000204670F005FDD8B10378202B03D110F8CF
:10FE4000013F202BFBD0F6F72FFB8FB1A5F2EE225E
:10FE500040F2DC539A420BD8A0F2EE229A4207D825
:10FE60000D4B03EB8603A3F88056A3F88206AEE79A
:10FE70000D4803B0BDE8F040FEF7DABD0B490C4871
:10FE80000323002203B0BDE8F040FEF7D1BD0546D4
:10FE90000746CCE764E70808B0A40020E803D007D1
:10FEA00030AB0020C4E9080840E60808D8E9080893
:10FEB00080E708082DE9F04385B040B30378064693
:10FEC0002BB300F1004C574C0CF1FF3C014603E012
:10FED000984232D1614512D011F8013BA3F14102A1
:10FEE000192A14F8012BA2F1410598BF2033192DCE
:10FEF00002F12000ECD99A421FD1002BEAD14A48E6
:10FF00006022002105B0BDE8F0436EF021BD464DF2
:10FF1000464E0024D5E9012115F80C3B0093CDE9AC
:10FF2000012123463246002101200134FFF7E2FE81
:10FF3000082CEFD105B0BDE8F0833046F6F7B4FAEF
:10FF4000C3B2072B054657D82021304670F078FC05
:10FF50000446002859D00378202B03D114F8013F20
:10FF6000202BFBD02046F6F79FFA071E18BF01276B
:10FF700001262046202170F063FC044600284ED064
:10FF80000378202B03D114F8013F202BFBD020460F
:10FF9000F6F78AFA01368046F6B22046202170F044
:10FFA0004FFC0446A0B30378202B03D114F8013F83
:10FFB000202BFBD02046F6F777FA01368146202128
:10FFC0002046F6B270F03CFC08B10136F6B2032EC2
:10FFD00005D0174805B0BDE8F043FEF729BD154B25
:10FFE0006DB205EB450503EB850383F89076C3F806
:10FFF0009486C3F898969DE70F491048072300227E
:020000040801F1
:1000000005B0BDE8F043FEF713BD06460746B0E76E
:10001000202170F015FCA1460028D6D1D9E78046F2
:10002000BBE700BF64E7080840AB0020E0E9080830
:1000300040E60808B0A40020F8E9080880E70808AE
:1000400070B588B0002841D003780446002B3DD01D
:1000500000252D2B54D0A3F13002092A50D9202B92
:1000600062D163780134002BF3D1052DBDF9143032
:100070005AD19AB2112A57D8BDF91610A1F5FA72C1
:1000800092B2B2F5FA6F4FD8BDF91800A0F5FA7226
:1000900092B2B2F5FA6F47D8BDF91A40A14243DCDB
:1000A000A04241DBBDF91C5005F17D0292B2FA2A53
:1000B0003AD8204A02EBC303A3F8F016A3F8F206DD
:1000C000A3F8F44683F8F65608B070BD1A4C1B4EE0
:1000D000002594F90600B4F90410B4F9022034F9AB
:1000E000083BCDE90210CDE9003200212B46324613
:1000F00001200135FFF7FEFD122DEAD108B070BDD9
:10010000042D11DC2046F6F7CFF908AB03EB4503CD
:10011000013523F80C0C14F8013FA3F13002092A31
:10012000F9D9002B95D1A0E7054808B0BDE870408B
:10013000FEF77EBCB0A40020A0AB002008EA0808AF
:1001400040E6080870B58AB0064670F0B9FC10F0B9
:10015000FF0414D13B4D3C4EAB68D5E90021012092
:10016000CDE9012100933246234600210134FFF7F7
:10017000C1FD082C05F10C05EED10AB070BD334C61
:1001800006F1050C314603E098422AD1614512D0B0
:1001900011F8013BA3F14102192A14F8012BA2F135
:1001A000410598BF2033192D02F12000ECD99A4265
:1001B00017D1002BEAD12648264A904238BF40F298
:1001C000FF3103D3D9E714309042D6D20388C3F36A
:1001D0000B038B42F7D11B490AB0BDE87040F6F71C
:1001E0001FBE1D4905AA30466CF026FF78B11A4E95
:1001F00006AD0024F6F758F905AA45F8040B314678
:10020000002001346CF018FF30B1042CF2D11348F7
:10021000FEF70EFC0AB070BD042CF8D1069B072B2C
:10022000F5D80849DDE9074003EB430301EB8302FE
:1002300041F823009460099B09485360FFF782FF4F
:100240009BE700BF30AC002020EA080864E70808FC
:1002500088560908EC5B09081846090840E60808B2
:10026000C84C09082DE9F04184B0654903AA6CF037
:10027000E3FE002870D0F6F717F90D2805462AD8B6
:100280005F4903AA00206CF0D7FE002866D05D49C4
:100290005D4E044603E09E4523D1B14213D011F8D0
:1002A000013BA3F14102192A14F8012BA2F1410CE0
:1002B00098BF2033BCF1190F02F1200EEBD99A42FE
:1002C0000FD1002BE9D100244D4903AA00206CF086
:1002D000B3FE00287BD04D48FEF7AAFB04B0BDE872
:1002E000F0814B494B4F044603E09C4516D1B9427F
:1002F00012D011F8013BA3F14102192A14F8012B85
:10030000A2F1410698BF2033192E02F1200CECD93E
:100310009A4203D1002BEAD10124D5E73E49DFF808
:1003200010C1044603E09F4235D1614512D011F857
:10033000013BA3F14102192A14F8012BA2F1410655
:1003400098BF2033192E02F12007ECD99A4222D10E
:10035000002BEAD10224B7E74FF0FF35DFF8CC805D
:100360002E4F2F4E00240EE03B5D08EB83033246F8
:10037000D3F8D83700930021234601200134FFF73A
:10038000B9FC0E2CAAD06B1CEED0AC42ECD00134E0
:100390000E2CFAD1A2E72349234F03E09E429AD1C3
:1003A000B94212D011F8013BA3F14102192A10F809
:1003B000012BA2F1410498BF2033192C02F1200631
:1003C000ECD99A4287D1002BEAD103247CE7134E63
:1003D000164FDFF84C8074550446AC420BD1335DA8
:1003E00007EB83034246D3F8D83700930021234616
:1003F0000120FFF77FFC01340E2CEED16EE700BF29
:100400001846090834EA080833EA088840E608086C
:100410003CEA08083BEA0888543C0908089D00208B
:1004200044EA080878380908773809889C380808A9
:10043000533C098810F040002FD00CB470B50C4626
:1004400082B029B1002002B0BDE8704002B0704710
:10045000174EB56B6B7A5A1C2B44D2B223216A72A9
:1004600099722B7A934219D9069A124907AB2846FA
:10047000019367F0F1FAB46B627A32B1D4E90030DB
:1004800004F10A01984700236372FFF739FB01204A
:1004900002B0BDE8704002B070477047002AE3D058
:1004A000D5E9003005F10A0198476C72B56BDBE7BE
:1004B000B0A400200DE700082DE9F04FDFF8F0A010
:1004C00087B0934681460D46164600270AF2EC7423
:1004D0004FF0190895F800C0BBF1000F52D03078EA
:1004E000604551D00021002302E001333D2B5AD05A
:1004F00004EBC3024FEAC30C12798242F5D1F378C0
:1005000005914FF4617218FB03230393B378D4442D
:1005100018FB032302939CF8F13772784846CDE923
:100520000032224A3B46FFF785FF95F800C0059947
:10053000002302E001333D2B35D004EBC302D80089
:1005400012796245F6D1EB784FF4617218FB032300
:100550000393AB78504418FB032302936A7890F816
:10056000F1374846CDE900323B46104A0137FFF7E4
:10057000C1FB282F05F1040506F10406AAD107B036
:10058000BDE8F08F5946D3E76A7873789A42A9D1CB
:10059000AA78B3789A42A5D1E978F378C91AB1FA62
:1005A00081F149099FE700235B79FFDE5CEA0808D7
:1005B0009C380808002871D0F0B5037883B0044651
:1005C000002B43D0F5F770FF272805466ADC00238F
:1005D000601C20218DF8073070F032F9AE0004461F
:1005E00058B10378202B03D114F8013F202BFBD006
:1005F0002046F5F759FF002834DA2046202170F014
:100600001FF90446A0B10378202B03D114F8013F51
:10061000202BFBD02046F5F747FF1D2808D8264B96
:10062000334483F8E1079DF8073001338DF8073034
:10063000224FB11C0DF1070239442046FEF7FEF8A7
:100640009DF80730042B08D103B0F0BD1B490022F0
:10065000012003B0BDE8F0402EE7002347F8253025
:1006600003B0F0BD164FC2B2002307F2EC7001E0F8
:100670003D2BC2D000EBC3014FEAC30C4979914234
:1006800003F10103F4D101238DF807300A4B6744CD
:10069000334497F8F02783F8E027AEE707490022B4
:1006A000012009E7074908482723002203B0BDE8D5
:1006B000F040FEF7BDB900BFB0A4002090AC002010
:1006C0009C38080810ED080880E708082DE9F04F6D
:1006D00089B0434E434F079092460C46154602F1AF
:1006E000540894F90430404A92F90010994202F1FA
:1006F0000C0209D09642F7D10C35454504F10C04A3
:10070000EFD109B0BDE8F08FBAF1000F51D095F9E3
:1007100004E0D5F800B06A79A879297A95F807C07D
:10072000734548D04FF0000907EB8C0C07EB8101B3
:10073000DCF8D439049307EB8000D1F8D439039363
:1007400007EB8202D0F8D4390293D2F8D43901935E
:10075000264A0798CDF800B073464946FFF76AFE6F
:1007600094F90430E279D4F800C007EB82024946DC
:10077000D2F8D4290492227A07EB82020C35D2F8FF
:10078000D4290392A27907EB82020C34D2F8D4293F
:10079000029214F8070C154ACDF800C007EB800050
:1007A000D0F8D40901900798FFF7A4FA454598D1ED
:1007B000A7E7D146D6E723685B45B3D16379934277
:1007C000B0D1A3798342ADD1237A8B42AAD194F8D8
:1007D0000790A9EB0C09B9FA89F94FEA5919A3E76F
:1007E00048A500209C380808F4A4002070EA0808F6
:1007F000D8B10278CAB12DE9F04F87B0451CF5F7A2
:1008000053FE5A4C014647B22246002392F9046037
:10081000BE4202F10C020CD00133072BF6D1544832
:1008200007B0BDE8F04FFEF703B9504900220120A0
:100830004CE703EB430304EB830494E8070003AEA7
:1008400086E807000746202128466FF0F9FF834617
:1008500000287DD00278202A03D11BF8012F202AFE
:10086000FBD02B2A39D02D2A66D05846F5F71CFE2E
:10087000022307460093E37994F8059094F80680E4
:1008800094F808A001930025584620216FF0D8FF66
:100890008346002845D00278202A03D11BF8012F77
:1008A000202AFBD05846F5F7FFFD002203461146EB
:1008B000304804E00132112A1AD050F8041F99423E
:1008C000F8D1022D5FFA82FC16D0032D16D0012D2F
:1008D00014BFE146E0460135D6E70BF1010B58465F
:1008E000F5F7E2FD01228240022317430093C2E79D
:1008F000BBB9022D9C46E8D1E246ECE7002369F340
:10090000070368F30F236CF317436AF31F6303971E
:10091000CDF8113096E8070084E8070007B0BDE87D
:10092000F08F009B2B44DBB2012B14D1124807B08F
:10093000BDE8F04FFEF77CB80BF1010B5846F5F718
:10094000B3FD01228240022327EA0207009392E7C7
:10095000012300938FE70023019A69F3070368F3EB
:100960000F2362F317436AF31F63D0E7D07E0020A2
:1009700090EA08087042080840E608082DE9F04FA0
:1009800089B0DFF8D0A0079281460C4615460026B4
:100990004FF019084FF461773AE0A97894F802B063
:1009A0002B786A78E87895F804C095F805E08B45CF
:1009B00034D04FF0000B18FB027218FB0373CDE923
:1009C0000232CDE9040CCDE900E1334652465946E6
:1009D0004846FFF72FFD23790593E3780493627867
:1009E000237818FB027218FB0373CDE90232A37857
:1009F000019363790093524633465946484601367F
:100A0000FFF778F9142E04F1060405F106051ED04F
:100A1000079B002BC1D1DDF81CB0DCE794F800B0D7
:100A20009B45C6D194F801B09345C2D194F803B068
:100A30008345BED194F804B0E345BAD194F805B02B
:100A4000ABEB0E0BBBFA8BFB4FEA5B1BB3E709B0BA
:100A5000BDE8F08FA4EA0808002800F0AD802DE979
:100A6000F047037882B00446002B71D0F5F71CFDE7
:100A70001328054600F3A48000EB40060023601C09
:100A800020218DF807306FF0DBFEDFF850814FEA50
:100A900046096F0008EB4606044658B10378202B40
:100AA00003D114F8013F202BFBD02046F5F7FCFCC6
:100AB000032877D9204620216FF0C2FE044658B1A2
:100AC0000378202B03D114F8013F202BFBD02046C4
:100AD000F5F7EAFC1D2859D920460DF107023146E9
:100AE000FDF7ACFE20216FF0ABFE0446002870D06D
:100AF0000378202B03D114F8013F202BFBD0204694
:100B0000F5F7D2FC3C289DF807A032D920462021D9
:100B10006FF096FEB0B10378202B03D110F8013F9F
:100B2000202BFBD0F5F7C0FC1D280BD82A4B2F44F7
:100B30000AF1010A03EB47035FFA8AFA8DF807A06E
:100B400083F88408BAF1060F09D102B0BDE8F08736
:100B500022490022012002B0BDE8F0470EE72048FC
:100B6000002348F80930B38002B0BDE8F047FDF734
:100B70005FBF194B7A190AF1010A03EB42035FFACE
:100B80008AFA8DF807A083F88308BFE79DF807204D
:100B9000114B01328DF807207A1903EB420383F8D9
:100BA000820899E70C4B7A1903EB420383F8850816
:100BB00001238DF807307DE7084900220120DDE69A
:100BC000084909481323002202B0BDE8F047FDF7A9
:100BD0002FBF9DF807A099E7B0A4002030AD0020FA
:100BE00040E6080810ED080880E708082DE9F04FF6
:100BF0002DED088B99B082460C46154600260792CB
:100C00005DE0F4EE4A8AF1EE10FA74D1B4EE6A9A1D
:100C1000F1EE10FA6FD1F4EE4B9AF1EE10FA0CBF30
:100C20000121002114A80691F5F71AFBB0EE4A0A3B
:100C3000074610A8F5F714FB0DF130098346B0EE16
:100C40006A0A4846F5F70CFB0DF120080590B0EE56
:100C50004B0A4046F5F704FB059A0390CDE901B233
:100C600006992B4A009733465046FFF7E3FBB0EE58
:100C7000480A14A8F5F7F4FAB0EE680A074610A877
:100C8000F5F7EEFAB0EE490A83464846F5F7E8FA7A
:100C9000B0EE690A81464046F5F7E2FA3346CDE9FF
:100CA0000290CDE9007B1A4A002150460136FFF739
:100CB00021F80C2E04F1100405F1100522D094ED5A
:100CC000008AB5EE408AF1EE10FA1BD0079BD4EDF6
:100CD000018A94ED029AD4ED039A73B195ED000A5E
:100CE00095ED01AAD5ED02AA95ED03BAB4EE408ABE
:100CF000F1EE10FA85D0002194E70DF130090DF1E5
:100D00002008B4E719B0BDEC088BBDE8F08F00BF38
:100D1000C4EA08082DE9F04198B30378054683B387
:100D20006D4C00F1050E014603E0984237D1714544
:100D300013D011F8013BA3F14102192A14F8012B39
:100D4000A2F1410C98BF2033BCF1190F02F1200031
:100D5000EBD99A4223D1002BE9D1604A92F84A1C80
:100D60004FF4D47000FB01F102F6F80302F6B8125A
:100D70000B440A44002143F8101F9342FBD1BDE805
:100D8000F081564991F84A3C4FF4D47000FB0311AE
:100D9000BDE8F041002201F60811012026E72846AF
:100DA000F5F782FB0B28064600F28B8020212846AF
:100DB0006FF046FD0446002800F08B800378202B5E
:100DC00003D114F8013F202BFBD02046F5F7B8FAE9
:100DD000424B93F84A2C4FF4D470711C00FB02F282
:100DE00003F6F80302EB0112134483ED000A012518
:100DF000204620216FF024FD0446C8B10378202B43
:100E000003D114F8013F202BFBD02046F5F798FAC8
:100E1000324B03F6F80293F84A3C4FF4D47101FBCD
:100E200003F3711C03EB01131344013583ED010A35
:100E3000204620216FF004FD0446C0B10378202B2A
:100E400003D114F8013F202BFBD02046F5F778FAA8
:100E5000224B03F6F80293F84A3C4FF4D47101FB9D
:100E600003F303EB06131344013583ED060A202137
:100E700020466FF0E5FCC0B10378202B03D110F8B9
:100E8000013F202BFBD0154C94F84A7CF5F758FA1B
:100E90004FF4D47307FB03F304F6F80403EB0616D0
:100EA0002644032D86ED070A04D0BDE8F0410C4826
:100EB000FDF7BEBD1033E1180022BDE8F04101206E
:100EC00094E6BDE8F041074907480B230022FDF7EF
:100ED000AFBD05468CE700BF64E70808B0A400205A
:100EE00040E6080810ED080880E708082DE9F04FF3
:100EF00091B0DFF834B1079282460C469046002547
:100F000009AF0BAE3AE01A4643493046F4F7F6FD16
:100F1000079B002B49D098F800C02378634547D041
:100F20004FF000093D4B059300230493B8F91230AC
:100F30000393B8F910303A4A02930192CDF800C0F9
:100F40002B465A4649465046FFF774FA0597237DCB
:100F50000493B4F912300393B4F9102014F8203B31
:100F60000093CDE901622B465A4649465046013569
:100F7000FEF7C0FE082D08F120084AD004F115093B
:100F80000422494638466FF007FE0022A3688DF818
:100F90002820E268082B72F10001B4D321493046C1
:100FA000F4F7ACFD079B002BB5D1DDF81C90CDE725
:100FB000D4E90202D8E902139A4208BF8842AFD1AD
:100FC000227D98F814309A42AAD199F8002098F816
:100FD00015309A42A4D199F8012098F816309A4217
:100FE00009F101099CD119F8012F98F817309A429C
:100FF00096D199F8012098F818309A4290D1226938
:10100000D8F81030A2EB0309B9FA89F94FEA591957
:1010100088E711B0BDE8F08FA8F30808C84C0908AC
:1010200090E00808D8EA0808E4EA080898B32DE92F
:10103000F04F037883B0804633B300F1004CA34DEA
:101040000CF1FF3C014603E0984228D1614512D0E3
:1010500011F8013BA3F14102192A15F8012BA2F165
:10106000410798BF2033192F02F12000ECD99A4292
:1010700015D1002BEAD196484FF48072002103B0BD
:10108000BDE8F04F6DF064BC91490022012003B02F
:10109000BDE8F04F2AE78E490022012026E74046AE
:1010A000F5F702FA83B2072B074600F2EA80202107
:1010B00040466FF0C5FB8146002800F0F4800378BD
:1010C000202B03D119F8013F202BFBD04846F5F720
:1010D000EBF901250FFA80F8202148466FF0B0FBAC
:1010E000002800F0E3800378202B03D110F8013FA3
:1010F000202BFBD0002B00F0E3800026014600F1FE
:10110000100C3446A3F13002D2B2092AA3F1610EC9
:101110000CD9BEF1050FA3F15702A3F1410E04D97A
:10112000BEF1050F11D8A3F13702D2B211F8013F79
:10113000240144EA167442EA0616002B00F0B0803F
:10114000202B00F0AD806145DCD1002301930135F7
:10115000EDB220216FF074FB8246002800F0AE80D3
:101160000378202B03D11AF8013F202BFBD05046E7
:10117000F5F79AF901350FFA80F9EDB250462021C2
:101180006FF05EFB8346002800F096800378202BEA
:1011900003D11BF8013F202BFBD05846F5F784F90B
:1011A00001350FFA80FAEDB2584620216FF048FB66
:1011B000834600287ED00278202A03D11BF8012F15
:1011C000202AFBD05846F5F76FF9013543B200935A
:1011D000EDB2584620216FF033FB0346002867D05C
:1011E0000278202A03D113F8012F202AFBD00135E1
:1011F000EDB2032D4ED91FFA88F2022A4AD809F21D
:10120000262292B2B2F5E16F44D80AF2262292B2B7
:10121000B2F5E16F3ED89DF800B0BBF1060F39D8AA
:10122000184600936FF04CFC042833D8019B8BB315
:101230002849009B28483FB201F5476201EB47115E
:1012400081F8708CA1F8809CA1F882AC81F884BCF4
:1012500002EB47110A46C1E902641432591E0333F6
:1012600011F8014F055D05F00305022D08BF203C74
:1012700002F8014F0C780CB19942F1D103B0BDE8EE
:10128000F08F164916480723002203B0BDE8F04F3F
:10129000FDF7CEBB134803B0BDE8F04FFDF7C8BB68
:1012A0000123019353E70546804615E7019050E777
:1012B0000D4B9EE700908CE7824675E781465DE71F
:1012C0001E461C460123019341E700BF64E708085E
:1012D00020B10020B0A4002021DD080808EB080898
:1012E00080E7080840E60808C84C09082DE9F04FD7
:1012F000DFF8AC9087B0924680460C461546002633
:10130000BAF1000F35D06B7A617AB5F90AC0B5F938
:101310000CE095F808B09942D5E900202BD00027C1
:10132000CDE90020CDE9023CCDE904EB33464A4645
:1013300039464046FFF77EF8237A0593B4F90C301E
:101340000493B4F90A300393637A0293626854F801
:10135000103B3946CDE90032404633464A46013615
:10136000FEF7C8FC112E05F11005C9D107B0BDE884
:10137000F08F5746E0E721689142D0D16168814201
:10138000CDD1B4F90A106145C9D1B4F90C10714539
:10139000C5D1277AA7EB0B07B7FA87F77F09BFE715
:1013A00018EB0808A0B32DE9F04F037883B0054689
:1013B0003BB300F1004E804C0EF1FF3E014603E0CE
:1013C000984229D1714513D011F8013BA3F1410294
:1013D000192A14F8012BA2F1410C98BF2033BCF15B
:1013E000190F02F12000EBD99A4215D1002BE9D157
:1013F00072484FF48872002103B0BDE8F04F6DF0E1
:10140000A7BA6E490022012003B0BDE8F04F6DE796
:101410006A490022012069E72846F5F745F8C3B27A
:10142000102B064600F2AC80202128466FF008FA07
:101430000446002800F0B1800378202B03D114F873
:10144000013F202BFBD02046F5F72EF8012507465B
:10145000204620216FF0F4F90446002800F09B801C
:101460000378202B03D114F8013F202BFBD020461A
:10147000F5F71AF801358046EDB2204620216FF0CD
:10148000DFF90446002800F084800378202B03D184
:1014900014F8013F202BFBD02046F5F705F8012872
:1014A000814667D80135EDB2204620216FF0C8F99A
:1014B0000446002874D00378202B03D114F8013F90
:1014C000202BFBD02046F4F7EFFF00F5B473B3F503
:1014D000347F82464ED80135EDB2204620216FF090
:1014E000AFF9834600285DD00378202B03D11BF889
:1014F000013F202BFBD05846F4F7D6FF00F5B4731C
:10150000B3F5347F044635D80135EDB25846202175
:101510006FF096F98346002846D00378202B03D13C
:101520001BF8013F202BFBD05846F4F7BDFF031EEC
:1015300018BF01230135584620210193EDB26FF009
:101540007FF908B10135EDB2062D13D11C4B019A7C
:1015500076B203EB0613C3F8707DC3F8748D83F87D
:10156000799DA3F87AADA3F87C4D83F8782D03B06C
:10157000BDE8F08F134803B0BDE8F04FFDF758BA4F
:10158000114912481023002203B0BDE8F04FFDF7C7
:101590004FBA814688E780466FE70546074657E71A
:1015A00082469AE70446B1E720216FF049F9002806
:1015B000E0D0CDF804B0C5E764E7080820B2002009
:1015C000B0A4002040E6080838EB080880E70808C7
:1015D0002DE9F047DFF8B4A088B0904681460C466C
:1015E00015460026B8F1000F34D098F80D20637B23
:1015F0009A4231D00027AB7B05936B7B04932B7B06
:101600000393AB6802936B6801936A782B7800921E
:10161000394652464846FEF70DFFA37B0693637B8F
:101620000593237B0493A368039363680293627812
:1016300014F8103B3946CDE900324846334652464D
:101640000136FEF757FB3F2E05F11005CAD108B051
:10165000BDE8F0874746E0E72288B8F800309A42B4
:10166000C8D1A268D8F808309A42C3D16268D8F8C5
:1016700004309A42BED1E368D8F80C20534033F0CE
:101680007F430CBF01270027B5E700BF4CEB0808DC
:101690002DE9F04F8FB00C460992079015460026B1
:1016A00030E02868BDF828100C9080B2AB88ADF807
:1016B00034308142B5F9023095F801C095F804E064
:1016C0002A7834D00021CDE9023ECDE9002C0798DC
:1016D0001E4ACDF8108033460891FEF7ABFE0899FC
:1016E0001A4A0798CDF800903346CDE903B8CDE902
:1016F00001A70136FEF7FEFA242E04F1060405F1D7
:1017000006051FD0B4F90270A388206894F801A0E0
:1017100094F804B094F9058094F800900A90ADF81C
:101720002C307FB1099B002BBBD10999D8E79F4290
:10173000C8D1BDF82C10BDF83400091AB1FA81F1F6
:101740004909C0E70FB0BDE8F08F00BF6CEB080897
:10175000F0B589B006466FF0B3F910F0FF020DD175
:10176000474991F84A3C4FF4D47000FB031101F64D
:10177000C811012009B0BDE8F04089E7414C751D52
:10178000314603E09E452AD1A94213D011F8013B0E
:10179000A3F14102192A14F8012BA2F1410C98BFC0
:1017A0002033BCF1190F02F1200EEBD99A4216D169
:1017B000002BE9D1324A344B92F84A1C4FF4D470D2
:1017C00000FB01221868998802F6C81302F52A6204
:1017D0001860998006339A42FAD109B0F0BD2B49BE
:1017E00001AA30466BF028FC4FF0FF33079380B11D
:1017F000264E02AD0024F4F757FE034645F8043B9D
:10180000002001AA314601346BF016FC30B1062CE1
:10181000F1D11F48FDF70CF909B0F0BD042CF8DD3B
:10182000029B232BF5D8039A112AF2D8049C3B2C57
:10183000EFD8059F07F57A71B1F5FA6FE9D8069EE2
:10184000FF2EE6D8079D691C4029E2D80C4991F883
:101850004A0C4FF4D47E0EFB00F04FF0060E0EFB48
:1018600003030B440B4883F8C82983F8C949A3F83C
:10187000CA7983F8CC6983F8CD59FFF769FFACE7E3
:10188000B0A4002064E70808B44208081846090814
:1018900040E60808C84C09082DE9F04F9FB098466B
:1018A0000F908B4692464FF0000910920AE0C8450F
:1018B0000BD009F10109B9F1400F0BF1140B0AF13A
:1018C000140A7AD0B8F1FF3FF1D15D460FCD14ACC8
:1018D0000FC42B6823609BF813300B939BF81030D8
:1018E0000C939BF911300D939BF81230DBF8082014
:1018F0000E93109B0A929BF80C209BF804700890A2
:101900000992002B46D0DAF800301193DAF808304B
:10191000129356469AF8133013930FCE19AD0FC594
:10192000189C33689AF804C09AF80CE02B605C406D
:1019300034F07F442CD167452ED00B9B07930A9B34
:101940000693099B0593089B1D4A0F98CDE90373E5
:101950000E9B02930D9B01930C9B009321464B46DB
:10196000FEF768FD0B9B07930A9B0693099B059363
:10197000089B134A0F98CDE903730E9B02930D9BAE
:1019800001930C9B009321464B46FEF7B3F990E779
:101990000024D2E7109CE5E7089B8342CDD1099B48
:1019A0007345CAD10A9B129A9342C6D10B9B139AD4
:1019B0009C1AB4FA84F46409BFE71FB0BDE8F08F45
:1019C00084EB08082DE9F0418AB005460C466FF01B
:1019D00077F810F0FF0011D1524991F83E2022B162
:1019E000631C3BD10AB0BDE8F0814FF0FF3301F535
:1019F000686101200AB0BDE8F0414DE74A4C681D1E
:101A0000294603E09E452CD1884213D011F8013BB2
:101A1000A3F14102192A14F8012BA2F1410C98BF3D
:101A20002033BCF1190F02F1200EEBD99A4218D1E4
:101A3000002BE9D13D483E4A904203D3D2E714300F
:101A40009042CFD20388C3F30B03B3F57E7FF6D168
:101A500038490AB0BDE8F041F5F7E2B9234602463D
:101A6000C5E735496A4628466BF0E6FA78B1324E4A
:101A70006D460024F4F718FD6A4645F8040F314618
:101A8000002001346BF0D8FA38B1092CF2D12B4880
:101A9000FCF7CEFF0AB0BDE8F081092CF7D101991F
:101AA0003F29F4D8029B012BF1D80398421C402A0D
:101AB000EDD8049F362FEAD8DDF814E0BEF1070F09
:101AC000E5D8DDF818C01E4C0CF5742202F5107232
:101AD000A242DCD8079E072ED9D8089D05F57422AE
:101AE00002F51072A242D2D8099CFF2CCFD80D4A21
:101AF0004FF0140808FB012209B282F8910E114838
:101B000082F8903E82F8927E82F884EEC2F880CE0F
:101B100082F88C6EC2F8885E82F8934EFFF752FF0F
:101B200060E700BFB0A4002064E7080888560908F1
:101B3000EC5B090830B300201846090840E60808A5
:101B400080841E00C84C09084FF0FF313AE700BFFF
:101B50002DE9F04FA5B08B46119092464FF0000949
:101B60001292DBF808300C939BF80C300B93BBF807
:101B700010300D93BBF812300E93BBF814300F9356
:101B80005D46BBF8163010930FCD16AC0FC495E828
:101B90000700129BDBF800709BF804809BF818602C
:101BA00084E80700002B4DD0DAF800301393DAF800
:101BB0000830159355469AF80C3014930FCD1DAC90
:101BC0000FC495E807009AF818E09AF804C0B645E3
:101BD00084E8070038D00024109B08930F9B0793DC
:101BE0000E9B06930D9B05930C9B04930B9B214A24
:101BF0001198CDE90273CDE900684B462146FEF706
:101C000019FC109B08930F9B07930E9B06930D9B4B
:101C100005930C9B04930B9B164A1198CDE9027314
:101C2000CDE900684B46214609F10109FEF762F84B
:101C3000B9F1040F0BF11C0B0AF11C0A91D125B06C
